:100000000C94CE0F0C94FF0F0C94FF0F0C94FF0F69
:100010000C94FF0F0C94FF0F0C94FF0F0C94FF0F28
:100020000C94FF0F0C94FF0F0C94FF0F0C94FF0F18
:100030000C94FF0F0C94FF0F0C94FF0F0C947E7622
:100040000C94FF0F0C94FF0F0C94FF0F0C94FF0FF8
:100050000C94FF0F0C94FF0F0C94FF0F0C94D1B570
:100060000C94FF0F0C943FB80C9415B80C94FF0F30
:100070000C94FF0F0C94FF0F0C94FF0F0C94FF0FC8
:100080000C94FF0F0C94FF0F0C94FF0F0C94FF0FB8
:100090000C947DA60C94EDA50C9434A60C941E45EE
:1000A0000C94FF0F0C94FF0F0C94FF0F0C94FF0F98
:1000B0000C94FF0F0C94FF0F0C94FF0F0C94FF0F88
:1000C0000C94FF0F0C94FF0F0C94FF0F0C94EBB7E4
:1000D0000C94C1B70C94FF0F0C9497B70C946DB7A8
:1000E0000C94FF0F7617DC18AA17C617DC18E81750
:1000F000DC181C1838185A189118AD1851196219C3
:10010000541954196219571962195A195A195A1956
:100110005A195A195419B21EA51E0A1F0A1F0A1F7E
:100120000A1F0A1F0A1F0A1F0A1F0A1F381BE21D87
:10013000E51DEF1D051E2F1EFE1D0A1F0A1F0A1FAB
:100140000A1F0A1FD21EE41EFF1E0525F924F924EA
:1001500005250525E024ED24ED24052505255D294B
:100160005D290D2C0D2C0D2CB92994299429942945
:1001700075297529B52CED2C822CF12CF12C552CE0
:10018000252CF12CB52CB52CFE4CFE4CFE4CF04C25
:10019000694D694D694D694D694D694D1D4D0C4D58
:1001A0002D4D494D3F4DB74FA64FA94FB14FB14FC0
:1001B000A94FA64FB14FB14FB14FA64FA64FA64F73
:1001C000B14FB14FB14FB14FB14FB14FB14FB14F2F
:1001D000B14FB14FB74F68597559795979599459F9
:1001E000945983597D598A591D62F2612D632D639B
:1001F0002D632D63BD62FF622D632D632D632D631F
:10020000066320630D632C624B62AB62AB624B6290
:100210002C62AB62AB62AB62816276626C629762A7
:100220008C624A634D63F2612D632D632D632D63F0
:10023000BD62FF622D632D632D632D632D632D63DE
:100240001963B26DD86D0B6E146E176E0B6EE86D80
:100250000B6E226E256EF96D316E346EA787FD86AA
:10026000FD86B68754885188A787C087C087C08716
:10027000A787A78770876387278710870D8745879C
:1002800075879787978732873287DD870C88208824
:100290000C880C88D087FC87FC87FC87E287EE8778
:1002A0007688AA8876886588658876887688FF8AC1
:1002B000FF8A76887688C79729986D98CA98DF98BC
:1002C0000098799879987998F497E097FC98BF9B73
:1002D000BF9BCE9BA79BA79BAE9BC79BC79BC79B68
:1002E000A79BA79BEB9BEB9B049CE69BE69BF79B4A
:1002F000F09BF09BF09BE69BE69BEEA1EEA1EEA1AE
:10030000EEA1EBA1EBA1F2A1F2A1F2A1F2A1F2A167
:10031000F2A1F2A1F2A1EBA1EBA1F2A1F2A1F2A153
:10032000F2A1F2A1F0A1EEA148A84BA863A87AA877
:10033000C4A8D7A8F7A81AAA1DAA0CAA10AA16AA78
:1003400054AA21AA25AA2BAA2FAA33AA39AA3DAAC0
:1003500041AA54AA47AA4BAA4FAAE9AAEEAAF3AA0D
:10036000FDAA07AB80AB11AB19AB21AB2BAB35AB07
:100370003FAB4EAB58AB80AB62AB6CAB76AB0763BD
:100380004236B79BD8A71A39685618AEBAAB558C07
:100390001D3CB7CC5763BD6DEDFD753EF617723150
:1003A000BF000000803F08000000BE922449123EBA
:1003B000ABAAAA2ABECDCCCC4C3E00000080BEAB7E
:1003C000AAAAAA3E00000000BF000000803F000073
:1003D000000000084178D3BB4387D1133D190E3C80
:1003E000C3BD4282AD2B3E68EC8276BED98FE1A9B7
:1003F0003E4C80EFFFBE01C4FF7F3F0000000000C5
:100400000C94FE430C9460B50C94B14F0C94B92934
:100410000C9427870C9441330C94E86D0C944B6238
:100420000C94047C0C94F09B0C94D0870C9439AA07
:100430000C94AA880C94AC320C94D6670C94358238
:100440000C9423440C94FF620C94B38B0C9497622D
:100450000C94617A0C9416AA0C947C5A0C94507BE0
:100460000C94DF670C94F1350C9422930C9448A8FB
:100470000C942B5B0C94BF9B0C94BA750C941D626E
:100480000C9426610C940C880C942D630C94E78BCF
:100490000C94C28B0C94FDAA0C9428B50C94BB123E
:1004A0000C940F440C944A630C94557A0C94E87A9B
:1004B0000C94E98B0C94FC980C9480120C9463A817
:1004C0000C94A79B0C941C970C9457800C940110CF
:1004D0000C94C4840C94E1B80C9477120C94FF90A3
:1004E0000C9421610C946B800C94CE9B0C94E2874D
:1004F0000C945A180C949E740C94562F0C942FAA9A
:100500000C9403110C943C800C94F79B0C94878002
:100510000C94DF980C94F3B80C9441AA0C94D6BCBC
:100520000C94DA820C94A51E0C9475590C947ABF25
:100530000C94715A0C941C180C943EC10C94E86BEA
:100540000C94B21E0C9425AA0C9479590C9475291C
:100550000C94AE9B0C9438660C9411AB0C94D96738
:100560000C9494290C9422B90C94ABBE0C94638720
:100570000C94F96D0C944D630C946D980C94D567A4
:100580000C94F0120C9453800C943F4D0C944587BE
:100590000C948C620C941BB90C94049C0C9476AB58
:1005A0000C944BA80C9479980C94D86D0C94D2BCF4
:1005B0000C94735A0C9474800C94D18D0C94DCB907
:1005C0000C9421AB0C947FB90C94D7A80C94EEAA90
:1005D0000C94FE1D0C9400440C9452130C94C08790
:1005E0000C9462190C940A1F0C942D4D0C947D5997
:1005F0000C9400980C9412360C94DC180C9488809F
:100600000C9468590C9480AB0C9443810C9435ABDA
:100610000C945D290C9462AB0C94CCBC0C94694D89
:100620000C940A9C0C94A8B80C947AA80C94176E9D
:100630000C94EE870C94F2610C94F0350C94572FC7
:100640000C941DAA0C94C6170C94FF8A0C941D4D93
:100650000C9404BE0C94C4A80C9446BE0C9427823F
:100660000C9408360C94FA8B0C94E51D0C945E6384
:100670000C9451880C948FB90C94EBA10C947E745B
:100680000C94E8790C944FAA0C940D750C94E3BC6F
:100690000C94552C0C9487BF0C9432870C941AAA96
:1006A0000C94AA320C9458AB0C94256E0C94D21E68
:1006B0000C9465880C9419630C9497870C945B7A5E
:1006C0000C94226E0C94FD860C9417970C94146E67
:1006D0000C940D870C94ED2C0C945A2F0C94F2A1D1
:1006E0000C94CDBC0C940D630C94AD180C94DBB43D
:1006F0000C948A590C94AA170C94427C0C9456685A
:100700000C94FF1E0C94CB8C0C9419AB0C942063AE
:100710000C9414B50C94F12C0C94051E0C94E58BE0
:100720000C94F3740C9457A40C94DE8B0C942B440F
:100730000C94E5BC0C94E9AA0C940C4D0C94381B59
:100740000C9421AA0C9407AB0C9472830C94B8B649
:100750000C9405250C9460840C94E8170C94FE4CC2
:100760000C942F1E0C94B6B80C94BEBD0C940CAA1D
:100770000C944BAA0C94B08B0C9415100C945488C8
:100780000C9454AA0C94073D0C9448A40C942BABE5
:100790000C942BAA0C944EAB0C94F4970C947617F3
:1007A0000C94E0240C94CC740C9410360C94EF1D33
:1007B0000C9457190C94C7970C94CE800C94511933
:1007C0000C9462B50C945F2F0C9491830C943FAB06
:1007D0000C94A37A0C94D3BC0C9491180C946C6276
:1007E0000C940B6E0C941F390C94E69B0C94E41E35
:1007F0000C94822C0C9477A40C94A94F0C948C111B
:100800000C94AFB50C94ED240C9498440C9433AA3A
:100810000C94EB8D0C94E0970C9438180C940663B0
:100820000C94252C0C94C38B0C940B940C9494591D
:100830000C947F800C94316E0C94E0C50C94BD62D6
:100840000C94FC870C94C79B0C9432800C94F0A100
:100850000C949B610C941A610C94E38B0C9420888B
:100860000C94B26D0C9410870C94EF740C94AB62E2
:100870000C9481620C9462B90C9458440C941B97AC
:100880000C94F9240C9470870C94EEA10C94299884
:100890000C9433840C943D800C94E21D0C94758769
:1008A0000C9436B50C94A7870C94A64F0C943DAAD3
:1008B0000C9454190C94AF8B0C94DF8F0C9486B865
:1008C0000C945DBB0C9469B80C9498910C94346EA4
:1008D0000C94EB9B0C940D8C0C94F3AA0C94766204
:1008E0000C9447AA0C94BA830C94A0740C94FF4304
:1008F0000C94B6870C946CAB0C9433610C942C6202
:100900000C945A190C945B800C9487440C94338596
:100910000C94C07A0C94B74F0C9494740C942F756B
:100920000C94F7A80C943F5B0C94CA980C94E96B58
:100930000C940D2C0C94DD870C9483590C9410AA04
:100940000C94E7BC0C9451B90C940B360C94B52C58
:100950000C9476880C94DC670C9420330C9405B5C9
:100960000C94F04C0C94D2C80C9458680C94494DDB
:100970000C94537A6364696E6F70737578585B007A
:10098000556E6B6E6F776E207375666669782000A2
:10099000556E6B6E6F776E20636D642000636C72B2
:1009A0004374723A20002F00496E3A200000002064
:1009B000002300260029002C002F00320000010037
:1009C000000301060109013D00494E3A00476F74DA
:1009D00020495020616464726573733A002769701E
:1009E000205B69705B2C646E735B2C67775B2C7388
:1009F00075626E65745D5D5D5D27202D2073657485
:100A0000207374617469632049500A004661696CFF
:100A1000656420746F20636F6E6669677572652008
:100A200045746865726E6574207573696E672044DD
:100A30004843502E20596F752063616E2073657492
:100A4000206970206D616E75616C6C7921000A758A
:100A500073657320444843500A00204D41534B3A7C
:100A6000002047573A0020444E533A004C6F6164CF
:100A700065642066726F6D20666C617368204950F2
:100A80003A005374617274696E67206C616E002461
:100A90006E6F6465730024666F726D617400246408
:100AA0006174617479706500302D31303000696E89
:100AB00074656765720068737600636F6C6F7200AF
:100AC0004F4E2C4F46462C48414C542C52455354C3
:100AD0002C584F4E2C584F46462C544F47474C45A8
:100AE00000656E756D00666C6F617400332E302E7C
:100AF000310024686F6D696500757074696D652CCF
:100B000066726565686561700030656232393234DD
:100B10005F323032312D30342D3132004C6967680C
:100B2000744875622000246E616D650072656164B1
:100B300079002074727920616761696E20696E2086
:100B400035207365636F6E6473006661696C6564FC
:100B50002C2072633D004177616974696E6720667D
:100B60006F722072657461696E656420746F70695C
:100B7000637300636F6E6E656374656420617320D8
:100B800000202E2E2E0020757365723A003A000A5E
:100B9000417474656D7074696E67204D51545420B2
:100BA000636F6E6E656374696F6E20746F200024CE
:100BB000737461746500646973636F6E6E656374EA
:100BC0006564005573696E67204D515454207061FF
:100BD0007373776F72642066726F6D20636F6E66D9
:100BE0006967004E3A00446576696365204E616D21
:100BF000653A00526562696E64207375636365735C
:100C0000732E20495020616464726573733A004505
:100C100072726F723A20726562696E6420666169F1
:100C20006C0052656E6577656420737563636573E8
:100C3000732E20495020616464726573733A0045D5
:100C400072726F723A2072656E65776564206661B4
:100C5000696C000A4E6F206C696E6B0041636365BE
:100C60007074696E6720636F6D6D616E64732E2E94
:100C70002E0A004452590046414E5F4F4E4C5900D7
:100C8000584F4E0048414C54002054533A002054D1
:100C90003A003D0050696E3A0044726976657220F0
:100CA0005265733A00416C72656164792048616CE9
:100CB0007465640A00416C726561647920496E61F3
:100CC00063746976650A00416C72656164792041DC
:100CD00063746976650A005475726E696E67205890
:100CE0004F4E0A00584F464620736B69707065641A
:100CF0002E205072657620636D643A005475726ED2
:100D00006564206F66662066726F6D3A0052657387
:100D1000746F7265642066726F6D3A004E6F207357
:100D2000746F7265642076616C756573202D206424
:100D3000656661756C743A200049676E6F72656410
:100D40002C206368616E6E656C20636D643D004F9E
:100D500075744F664D656D6F7279210A003B2000F6
:100D600020436D643D00205375623D002049746549
:100D70006D3D0052414D3D002064656C74613A0048
:100D80002D3E002F002056616C3A00496E3A004D0E
:100D90006F746F722074696D656F757400556E6B3A
:100DA0006E6F776E20636D6400466F7263656420BA
:100DB000657865637574696F6E00496E76616C69FC
:100DC000642050494420706172616D2061727261CB
:100DD000792E002C002C002C002C005049443A2085
:100DE000636F6E666967206661696C65643A00507E
:100DF000494420636F6E666967206C6F6164656447
:100E0000200050494420636F6E66696720657272E6
:100E10006F72005049443A204F7574206F66206D00
:100E2000656D6F72790053686F770020636D643D64
:100E3000002D00312D7769726520636F756E743AED
:100E4000200020416464723A0064657623002061CA
:100E50006C69766500204E6F64653A005365617277
:100E60006368696E6700312D776972652073686FFA
:100E700072746564005265747279696E6720646982
:100E80006D6D657220434D440A004D6F6462757349
:100E900020706F6C6C696E67206572726F723D00B6
:100EA0002056616C3A20004D423A20004E6F74206B
:100EB000737570706F7274656420726567207479E1
:100EC00070650A00496C6C6567616C2061726775BA
:100ED0006D656E74730A005265747279696E67206D
:100EE000564320434D440A004D6F64627573207071
:100EF0006F6C6C696E67206572726F723D002D00B9
:100F00002050492056616C203A004D6F6462757321
:100F100020706F6C6C696E67206572726F723D0035
:100F20002D0020464D2056616C203A0052657472A7
:100F300079696E672056432074656D7020434D4477
:100F40000A00696E00735F6F7574006D79686F6D6C
:100F50006500202D3E2000202D3E2000202D3E202B
:100F60000020696E61637469766520002061637496
:100F700069766520002076616C75652069732000B4
:100F800020756E6B6E6F776E0A00204772703A00A4
:100F900020696E76616C69640053746174757320A6
:100FA00064656666657265640A002D3E0050756270
:100FB0003A2000636D6400434F4F4C004845415454
:100FC000004155544F002D3E005075623A20007389
:100FD0006574002D3E005075623A20002D3E005091
:100FE00075623A2000556E6B6E6F776E20636D648C
:100FF000200A004F4646004F4E004D6F64627573E5
:10100000206F70206661696C65640A004D42206F34
:101010006B003D005643230020636D643D003D009E
:1010200056435F6865617423006931360001693396
:1010300032000275313600037533320004693868B6
:10104000000569386C0006753868000775386C0053
:101050000878313000094164642040533A20003A56
:10106000002066726F6D20004D4220676F74200073
:1010700000002100240027002A002D00300033004A
:1010800001010000040107010A01010210202008EB
:1010900008102040102040800201020108040201D3
:1010A0000102040810204080804020100804020142
:1010B000800402018040201008040201080402019B
:1010C0000102040810204080010204081020408022
:1010D00005050505070508080808020202020A0AB4
:1010E00008080404040401010101010101010303D2
:1010F000030303030303040707070C0C0C0C0C0C7D
:101100000C0C0202020206060606060606060B0B79
:101110000B0B0B0B0B0B3E003C00543A004375725B
:1011200072656E74204C414E20636F6E666967284D
:1011300069702C646E732C67772C7375626E65749E
:10114000293A000A55736520746865736520636FDA
:101150006D6D616E64733A202768656C7027202D71
:10116000207468697320746578740A276D61632040
:1011700064653A61643A62653A65663A66653A3032
:1011800030272073657420616E642073746F7265FC
:10119000204D41432D6164647265737320696E2034
:1011A000454550524F4D0A276970205B69705B2C92
:1011B000646E735B2C67775B2C7375626E65745D10
:1011C0005D5D5D27202D20736574207374617469E3
:1011D000632049500A277361766527202D207361AB
:1011E000766520636F6E66696720696E204E565281
:1011F000414D0A2767657427205B636F6E666967D8
:1012000020616464725D27202D2067657420636F00
:101210006E6669672066726F6D207072652D636FF0
:101220006E666967757265642055524C20616E6404
:101230002073746F726520616464720A276C6F6139
:101240006427202D206C6F616420636F6E66696770
:101250002066726F6D204E5652414D0A277077649A
:1012600027202D20646566696E65204D51545420F9
:1012700070617373776F72640A276B696C6C2720D7
:101280002D2074657374207761746368646F670AD6
:1012900027636C65617227202D20636C6561722065
:1012A000454550524F4D0A277265626F6F74272073
:1012B0002D207265626F6F7420636F6E74726F6C35
:1012C0006C657200536F6674207265626F6F74692B
:1012D0006E672E2E2E00444D58696E20427566664C
:1012E000657220616C6C6F632065727200496E6973
:1012F0007420696E2063683A00444D584F75742E0F
:1013000020467265653A000944533234383220650C
:1013100072726F720009526573657420646F6E6536
:101320000009436865636B696E6720666F722031E0
:101330002D5769726520646576696365732E2E2E5C
:10134000004453323438322D31303020707265739E
:10135000656E74004572726F7220312D7720696E50
:10136000697420233220467265653A007773746190
:10137000742E20467265653A005465726D2E2046C3
:101380007265653A004572726F7220312D7720695F
:101390006E697420233100467265653A0044533209
:1013A0003438325F3130305F4932435F544F5F3100
:1013B000575F42524944474520696E697400204195
:1013C0006464723A00646576230052414D3D000A20
:1013D000312D7769726520000A6D71747420000ADE
:1013E0006D6F64627573207632000A6D6F6462758A
:1013F0007320763120282B29000A696E707574736A
:1014000020000A6974656D7320000A436F6E666977
:1014100067757265643A003B003D0050696E3A00A2
:101420003B003D4C4F5700546865726D6F3A004F5A
:101430006E6520776972652052656164790A00469D
:101440007265653A00444D58206F7574207374615D
:10145000727465642E204368616E6E656C733A2009
:1014600000444D5820696E20737461727465642E57
:10147000204368616E6E656C733A00636373383144
:10148000313A2064617461206E6F74206176616905
:101490006C61626C6500636373383131206E6F7408
:1014A00020696E697469616C697A6564004552529D
:1014B000004C4F57004D454449554D004849474859
:1014C0000046414E5F4F4E4C59004452590048452A
:1014D000415400434F4F4C004155544F00726177C7
:1014E000007175656974007377696E67006C6F636E
:1014F0006B002D3E002000230050656E6465642063
:101500007374617465207265747269657665643A96
:10151000003D004C454741435920494E3A00766111
:101520006C0074656D7000736174006875650066A9
:10153000616E0052474200485356006D6F6465006B
:10154000536574436D643A00536574466C61673A41
:1015500000436C72466C61673A0053746F72656445
:10156000204558543A00737566666978436F646520
:101570003A000000000000000000004F4E00000094
:10158000000000004F464600000000000052455396
:10159000540000000000544F47474C4500000048ED
:1015A000414C540000000000584F4E000000000065
:1015B00000584F46460000000000494E4352454146
:1015C0005345004445435245415345004845415425
:1015D0000000000000434F4F4C0000000000415548
:1015E000544F000000000046414E5F4F4E4C5900E2
:1015F00044525900000000000053544F50000000B6
:1016000000004849474800000000004D4544495546
:101610004D0000004C4F5700000000000054525590
:1016200045000000000046414C53450000000045C5
:101630004E41424C4544000044495341424C4544CC
:1016400000524742000000000000485356000000CE
:1016500000000054787432436D643A00005EBCE2CE
:10166000613FDD83C29C7E20A3FD1F419DC3217F7E
:10167000FCA2401E5F01E3BD3E6082DC237D9FC172
:10168000421CFEA0E1BF5D0380DE3C62BEE0025C66
:10169000DF81633D7C22C09E1D43A1FF4618FAA452
:1016A00027799BC584DA3866E5BB5907DB8567393E
:1016B000BAE406581947A5FB7826C49A653BD98732
:1016C000045AB8E6A7F91B45C6987A24F8A6441A26
:1016D00099C7257B3A6486D85B05E7B98CD2306E12
:1016E000EDB3510F4E10F2AC2F7193CD114FADF3FE
:1016F000702ECC92D38D6F31B2EC0E50AFF1134DF2
:10170000CE90722C6D33D18F0C52B0EE326C8ED0E5
:10171000530DEFB1F0AE4C1291CF2D73CA947628D1
:10172000ABF517490856B4EA6937D58B5709EBB5BD
:1017300036688AD495CB2977F4AA4816E9B7550BB1
:1017400088D6346A2B7597C94A14F6A8742AC896A5
:10175000154BA9F7B6E80A54D7896B35436F6E6EFF
:1017600065637465642E00436F6E6E2E2061626F38
:1017700072746564004C6F61646564006C6F6164D1
:10178000206661696C6564004E6F2073746F7265CA
:101790006420636F6E666967004C6F6164696E6791
:1017A00020436F6E6669672066726F6D20454550F5
:1017B000524F4D000A72657175657374204D515416
:1017C0005420436F6E6669670053617665642074C8
:1017D0006F20454550524F4D00536176696E67202A
:1017E000636F6E66696720746F20454550524F4D98
:1017F0002E2E0053617665640A0053657420647967
:101800006E616D69632049500A00454550524F4D45
:1018100020636C65617265640A0050617373776F51
:10182000726420757064617465640A00636F756C1E
:1018300064206E6F742070617273653A2000557079
:1018400064617465640A002B002D00485454502FC5
:10185000312E312025690020485454502F312E312B
:101860000D0A486F73743A2025730D0A416363654E
:1018700070743A202A2F2A0D0A436F6E6E656374C6
:10188000696F6E3A20636C6F73650D0A00257300F3
:1018900020000D0A00474554006661696C656420AC
:1018A000746F20636F6E6E6563740A004552524F09
:1018B000523A205365727665722072657475726E45
:1018C00065642000446F6E652E0A004170706C796B
:1018D000696E672E0A00436F6E66696720706172D9
:1018E00073696E67206661696C65640A00676F746E
:1018F00020436F6E6669670A00436F6E66696720F2
:101900005552493A20687474703A2F2F002044656C
:101910006661756C7420636F6E66696720736572AB
:1019200076657220757365643A20006C617A796817
:101930006F6D652E727500205361766564000A280C
:101940002D295359534C4F47000A282B29504944FD
:10195000000A282D294D43503233303137000A28F0
:101960002D294152544E4554000A282D294F5441E7
:10197000000A282B29535049204C4544000A282BA3
:10198000294D4F544F5220435452000A282B2941CD
:1019900043204841494552000A282B2943435338E4
:1019A000313120262048444331303830000A282D78
:1019B00029524553544152545F4C414E5F4F4E5F44
:1019C0004D5154545F4552524F5253000A282D290D
:1019D0004841524452455345542C207573696E67F3
:1019E00020736F6674000A282D29434F554E5445C5
:1019F00052000A282D29444854000A282B294F5701
:101A0000495245000A282B294D4F44425553000A9C
:101A1000282B294144414652554954204C45440005
:101A20000A282B29444D58000A282B2957697A6E19
:101A3000657435313030000A282B2944533234384C
:101A4000322D313030000A282D29467265655261E9
:101A50006D207072696E74696E670064653A6164C6
:101A60003A62653A65663A66653A3037000A466911
:101A7000726D77617265204D4143204164647265E7
:101A8000737320006C617A79686F6D652E727500D2
:101A90000A436F6E666967207365727665723A00F5
:101AA0000A282B295741544348444F47000A282B02
:101AB00029434F4E54524F4C4C494E4F0032303117
:101AC0003130334C0020432B2B2076657273696FC5
:101AD0006E3A00306562323932345F323032312D45
:101AE00030342D3132000A4C617A79686F6D652E81
:101AF0007275204C6967687448756220636F6E74F4
:101B0000726F6C6C657220004E6F7420737570700C
:101B10006F727465642072656720747970650A005D
:101B2000293A0028543A003D3E0020002D3E004353
:101B30006F6E76657274696E6720002D3E00577275
:101B40006F6E672041737369676E6D656E742000F8
:101B5000524742783A200020764C6576656C3A0010
:101B600020436F6E76563A0020436F6E76533A00EC
:101B700020486F743A00436F6C643A0020436F6EE4
:101B800076657274656420563A00436F6E766572AE
:101B900074656420533A002D3E0057726F6E6720C3
:101BA00041737369676E6D656E7420002D3E00573A
:101BB000726F6E672041737369676E6D656E742016
:101BC00000444D582D4F757420496E697400444D82
:101BD000582D4F75742073746F700041737369676B
:101BE0006E65643A00444D58206374726C3A20006C
:101BF00044656661756C742073657269616C206DF3
:101C00006F6465204E383120757365640038453146
:101C1000002600384E31000600384532002E0038CC
:101C20004E32000E00384F31003600384F32003E41
:101C300000374531002400374E310004003745326B
:101C4000002C00374E32000C00374F310034003783
:101C50004F32003C00203D3E004D6F6462757320A2
:101C600074656D706C617465206E6F7420666F753D
:101C70006E643A2000496E76616C69642074656D0B
:101C8000706C6174652E002C002C002C002C004D13
:101C90004255533A20636F6E666967206661696CCE
:101CA00065643A004D6F6462757320636F6E666998
:101CB00067206572726F72004D6F64627573206386
:101CC0006F6E666967206C6F6164656420004D42C9
:101CD00055533A204F7574206F66206D656D6F7295
:101CE00079004D4255533A20506F6C6C696E6720F5
:101CF0006572726F7220004E6F7420737570706F12
:101D0000727465642072656720747970650A006575
:101D10006E64506F6C6C20002D2D2D00506F6C6C1C
:101D20002000556E6B6E6F776E20737566666978EE
:101D30002000556E6B6E6F776E20636D64200046D9
:101D40006F7263656420657865637574696F6E0092
:101D5000204F464600204F4E00757074696D650037
:101D600066726565686561700024737461747300E0
:101D700020457870697265640A00202D746172676D
:101D80006574207A6F6E652D0020416C61726D2044
:101D9000457870697265640A0020636D643A0020BA
:101DA0004375723A00205365743A006363733831A7
:101DB0003120697320616C726561647920696E6994
:101DC0007469616C697A65640068646331303830C5
:101DD00020697320616C726561647920696E697431
:101DE00069616C697A656400484443313038302059
:101DF0006E6F7420696E697469616C697A656400DC
:101E000053617665643A0020537566663A00204156
:101E1000543A00206973200044656C6574696E67EC
:101E200020636F6E662E2052414D207761733A0019
:101E300053746F707065640053746F7070696E676F
:101E4000206368616E6E656C73202E2E2E00556EB9
:101E50006C6F636B696E6720636F6E666967202EB7
:101E60002E2E00536B697070696E672E2E004F75B1
:101E7000744F664D656D6F727921005D20000A5BBD
:101E8000003A004D41433A003E3E2000496E7661E3
:101E90006C696420636F6D6D616E640000002200E8
:101EA000250028002B002E00310034000201000024
:101EB000050108010B0100000A0B02090C0D0E08B8
:101EC0000703040100000000000000000000000003
:101ED0000000000000000000000000000000000002
:101EE00000001211100000000000000000000000BF
:101EF0000000000000000000000000002C20002E68
:101F0000003E3E3E004E6F204D414320636F6E66A3
:101F10006967757265643A20736574206669726DCD
:101F2000776172652773204D41430A00556E6B6ED1
:101F30006F776E207375666669782000556E6B6EDC
:101F40006F776E20636D642000536574706F696EE7
:101F5000743A00496E7075742076616C75653A004C
:101F600050574D2D4F757420496E69740050574D70
:101F70002D4F75742073746F700052474220505774
:101F80004D002050574D00524742572050574D00AA
:101F90003D0050696E3A0000E0C5D2C811241FBE52
:101FA000CFEFD1E2DEBFCDBF00E00CBF1AE0A0E072
:101FB000B2E0E4EBF5EB01E00BBF02C007900D923D
:101FC000A034B107D9F721E1A0E4BAE001C01D9225
:101FD000AC3BB207E1F71FE0CDECDFE000E006C06C
:101FE00021970109802FFE010E9466D6CC3CD107C3
:101FF00080E00807A9F70E94D8C80C94C8DA0C94AE
:102000000000FC0122813381232B49F086819781D6
:102010008130910549F01CF00397029718F080E099
:1020200090E0089582E090E00895CF93DF93CDB7DC
:10203000DEB760970FB6F894DEBF0FBECDBF198232
:102040001A821B821C821D821E821F8218868B812F
:102050008F7080618B836FEF3E819F81888529819E
:102060007A815B814C814C873E87888B372F452F47
:102070005C857E85892F988960960FB6F894DEBFBF
:102080000FBECDBFDF91CF9108958F929F92AF92F7
:10209000BF92CF92DF92EF92FF920F931F93CF9355
:1020A000DF93E0919610F0919710309709F469C092
:1020B000812EF02E932EC22EA52ED42EB72EE62ED4
:1020C000BC01CF010E94565AEC01892B09F45CC077
:1020D00088858F70853009F057C060E0CE010E947E
:1020E0001B9F8C0161E0CE010E941B9FFC01C185FA
:1020F000D285D80119962D913C911A97213031053E
:1021000071F034F4232B09F03FC06F2DCE0118C0BD
:102110002230310549F027303105A9F035C06F2D47
:10212000CE0103960E946A776E2DCE010E946A77D7
:102130006D2DCE0101960E946A776C2DCE0102961C
:102140000E946A7721C0892BF9F080858F708530D5
:10215000D9F4C681D7812097B9F088858F708430F3
:1021600061F40F2D182D2C2D392D4D2D5A2D6E2D3E
:102170007B2D89859A850E9445100A80DB81C02DC0
:10218000EACF80E090E002C081E090E0DF91CF9163
:102190001F910F91FF90EF90DF90CF90BF90AF9085
:1021A0009F908F900895CF92DF92EF92FF920F93BE
:1021B0001F93CF93DF93E091CB0FF091CC0F30972B
:1021C000C9F090859F709530A9F469017A01EB01FF
:1021D000682FCF010E941B9FFC0190859F70943057
:1021E00049F481859285009729F09601A701BE01E7
:1021F0000E944510DF91CF911F910F91FF90EF90BA
:10220000DF90CF900895AF92BF92CF92DF92EF927E
:10221000FF920F931F93CF93DF938091C80F9091FC
:10222000C90F892B09F46DC0E1E0F0E0C0E0D0E017
:10223000CC24C394D12CB6010C2E02C0660F771F9C
:102240000A94E2F74091440A5091450A7F0184E0E4
:10225000E80EF11CCF01B12C9C01A0912E02B0918F
:102260002F02A817B90720F420912E0230912F02D7
:10227000A0914710B0914810A20FB31FAC90A0914D
:10228000C80FB091C90F9C0121503109A20FB31F93
:102290000A2D10E02C9130E00217130729F0462B8D
:1022A000572BAC92BB24B3940196E816F906A1F61D
:1022B0005093450A4093440ABB20E9F08091C80F2F
:1022C0009091C90FE80FF91F028110E0218130E0E1
:1022D000408150E03197608170E0CE010E94D310C0
:1022E00080E00E946C486093400A7093410A80939A
:1022F000420A9093430A2196F701C430D10509F0B0
:102300009ACFDF91CF911F910F91FF90EF90DF90C7
:10231000CF90BF90AF900895AF92BF92CF92EF92BF
:10232000FF920F931F93CF93DF93CDB7DEB728971C
:102330000FB6F894DEBF0FBECDBF5C0109831A83D0
:102340002B833C834D835E836F8378876DE979E0CF
:1023500089EF9EE00E9422B6CE0101960E94449928
:102360006981611114C00B810F70013081F030F070
:10237000023031F0053021F010E06EC0CC24C3945F
:10238000D501ED91FC91068CF78DE02D45C0F5014E
:10239000828193810E940B6A19811130A9F0123059
:1023A00009F047C01D821E821F821886D501ED915B
:1023B000FC91068CF78DE02DCC24C39402E01A81A9
:1023C0002B813C8140E02DC0CE0101960E94289FC8
:1023D0004997D4F459C0873008F065C081508230E5
:1023E00010F486E68D83D50112966D917C9113973A
:1023F00040E0CE0101960E94969960E07AE0F501F6
:10240000828193810E942A4FD501ED91FC91068C27
:10241000F78DE02DCC24C39409811A812B813C8156
:102420004D815E816F817885C501199581E090E0CD
:102430004EC060E979E089EF9EE00E9422B64AE052
:1024400050E0612F89EF9EE00E94B1B689EF9EE0D7
:102450000E9449B701E010E060E879E089EF9EE072
:102460000E9422B64AE050E0B80189EF9EE00E9447
:1024700042B789EF9EE00E9449B7CE0101960E94C3
:10248000449980E090E023C08B8182958F708630E4
:1024900009F0A1CF8CEF93E0A0E0B0E08D839E83A4
:1024A000AF83B887A0CF873049F480E090E0ACECF0
:1024B000B2E48D839E83AF83B88795CF8A508230F4
:1024C00008F091CF86E690E0A0E0B0E0E7CF289654
:1024D0000FB6F894DEBF0FBECDBFDF91CF911F9135
:1024E0000F91FF90EF90CF90BF90AF900895FC01B7
:1024F00082819381009719F062E00E940B6A08952F
:102500000F931F93CF93DF93CDB7DEB728970FB606
:10251000F894DEBF0FBECDBF19821A821B821C82C7
:102520001D821E821F8218862B812F702B83198299
:10253000FC0102811381C8010E94366A823071F069
:10254000853061F040E0B801CE0101960E94EE991D
:1025500060E0CE0101960E94D19A02C080E090E036
:1025600028960FB6F894DEBF0FBECDBFDF91CF9196
:102570001F910F910895CF92DF92EF92FF920F93E8
:102580001F93CF93DF93CDB7DEB760970FB6F89464
:10259000DEBF0FBECDBF7C016B01CA01B901AE0128
:1025A0004F5F5F4F0E94D249D701ED91FC910288A5
:1025B000F389E02D9801AE014F5F5F4FB601C7016F
:1025C000199560960FB6F894DEBF0FBECDBFDF91B0
:1025D000CF911F910F91FF90EF90DF90CF900895D2
:1025E000CF92DF92EF92FF920F931F93CF93DF93DF
:1025F000CDB7DEB7C054D1090FB6F894DEBF0FBE19
:10260000CDBF8091941090919510059789F1611537
:10261000710571F169017A018B0140E450E0CE014E
:1026200001960E9417DA6FE270E0CE0101960E94D7
:10263000DED9892B41F4980143E050E060E4CE01FB
:1026400001960E94384940E450E0B601CE0101965F
:102650000E94F9D90E94DD9D882351F08091941049
:1026600090919510069721F48091DC0A882319F047
:1026700080E090E007C0B701CE0101960E94FF9E66
:1026800081E090E0C05CDF4F0FB6F894DEBF0FBE74
:10269000CDBFDF91CF911F910F91FF90EF90DF9011
:1026A000CF900895CF92DF92EF92FF920F931F93F6
:1026B000CF93DF93CDB7DEB760970FB6F894DEBF48
:1026C0000FBECDBF7C016B01BA01A901CE010196FD
:1026D0000E94DD48D701ED91FC910288F389E02D3D
:1026E0009801AE014F5F5F4FB601C7011995609623
:1026F0000FB6F894DEBF0FBECDBFDF91CF911F9113
:102700000F91FF90EF90DF90CF900895EF92FF929E
:102710000F931F93CF93DF93EC018B011D821C82DB
:102720001A821B82E880F980E114F10409F464C084
:102730008091201090912110892B09F45DC0672BA6
:1027400009F48701F80180858F708630D1F46BE041
:1027500079E0C8010E94565A009719F0FC01818562
:102760008A8366EA75E0C8010E94565A009719F0FC
:10277000FC01818505C0F801808191810E9443CDD3
:102780008B8360E675E0C7010E94565A009789F571
:102790001A810B8168EA79E089EF9EE00E9422B6F7
:1027A0004AE050E0602F89EF9EE00E94B1B666EAF1
:1027B00079E089EF9EE00E9422B64AE050E0612F66
:1027C00089EF9EE00E94B1B689EF9EE00E9449B772
:1027D00020E030E0A90160E675E0888199810E94DF
:1027E000D99F60E675E0888199810E94565A0097CA
:1027F00019F009969D838C83DF91CF911F910F91E2
:10280000FF90EF9008954F925F926F927F92AF92F8
:10281000BF92CF92DF92EF92FF920F931F93CF93CD
:10282000DF938091440A9091450AC4E0D0E021E012
:1028300030E0AC0142235323452B29F0A9014095F8
:10284000509584239523220F331F219791F790935E
:10285000450A8093440A4090400A5090410A609093
:10286000420A7090430A411451046104710409F44E
:1028700071C00E9407AC9B01AC01AA24AA94BA2C97
:1028800065011CE2E12EFF24F39400E010E0C30197
:10289000B2010E948248882309F45CC01092400A69
:1028A0001092410A1092420A1092430AE12CF12C34
:1028B000E091C80FF091C90FEC0FFD1F038110E0EC
:1028C000228130E0418150E0608170E0C7010E94C8
:1028D000D3108FEFE81AF80A249684E0E816F10482
:1028E00039F7C1E0D0E080912E0290912F028C1731
:1028F0009D0728F480912E0290912F0201C0CE01F5
:102900002091471030914810F901E80FF91F4AE073
:1029100050E060818CE59EE00E94B1B663E675E010
:102920008CE59EE00E945FB72196C131D105D9F6B2
:102930008CE59EE0DF91CF911F910F91FF90EF907A
:10294000DF90CF90BF90AF907F906F905F904F904F
:102950000C9449B7DF91CF911F910F91FF90EF90A9
:10296000DF90CF90BF90AF907F906F905F904F902F
:102970000895FC016115710519F48481958108950C
:1029800086819781681779072CF084819581860F5D
:10299000971F0895828193810C945769EF92FF925B
:1029A0000F931F93CF93DF93DC011296ED91FC916F
:1029B0001397309709F17A018B01EC0165E675E018
:1029C000808191810E94565A0097B1F0FC012085C8
:1029D0002F70243089F461857285E881F98102883D
:1029E000F389E02D9701A801CE01DF91CF911F91CE
:1029F0000F91FF90EF90199480E090E0DF91CF91DC
:102A00001F910F91FF90EF900895EF92FF920F9317
:102A10001F93CF93DF93CDB7DEB760970FB6F894CF
:102A2000DEBF0FBECDBF8C01CB01BA017901AE0173
:102A30004F5F5F4F0E94D249A701BE016F5F7F4F7A
:102A4000C8010E94CE1460960FB6F894DEBF0FBE88
:102A5000CDBFDF91CF911F910F91FF90EF9008951F
:102A60002F923F924F925F926F927F928F929F929E
:102A7000AF92BF92CF92DF92EF92FF920F931F938C
:102A8000CF93DF93CDB7DEB7C357D1090FB6F89414
:102A9000DEBF0FBECDBFDC0114962D913C91159782
:102AA000232B09F4EAC13B014C01A5969FAF8EAFE1
:102AB000A5978EE294E0A3969FAF8EAFA397A996B9
:102AC000BFAFAEAFA99786E194E0A7969FAF8EAF58
:102AD000A7976130710509F460C10CF4CBC1643073
:102AE00071050CF0C7C1D40112968C91803451F15C
:102AF00028F0823439F108F4BDC18058843008F0E0
:102B0000B9C1A3016FEFC4010E942B6DF4011281C2
:102B10001695117003818AEC800F803108F0B0C1E6
:102B20006AE675E0808191810E94565A5C010097A7
:102B300009F4A6C1DC0118968C918F70853009F0DC
:102B40009FC142C16AE675E0D4018D919C910E94BB
:102B5000565A8C01F401838190910E0F981309C08D
:102B600090910F0F903429F48091100F9091110FD4
:102B70000BC080930E0F90E490930F0F0E9489ABCF
:102B80009093110F8093100F5C010115110509F44A
:102B9000F0C0D80118962C912F70253009F0E9C0AB
:102BA000C8010E949C9FAA968FAFAA97843008F410
:102BB00079C063E0C8010E941B9FFC01818592855A
:102BC0004AE0742E789E1001799E300C112462E048
:102BD000C8010E941B9FDC0119968D919C911A9748
:102BE000789E6001799ED00C1124E496DFAECEAEC3
:102BF000E4972601DD0C6608770861E0C8010E94B1
:102C00001B9F7C0160E0C8010E941B9FDC0119969C
:102C10002D913D914D915C911C97AE962CAF3DAF9F
:102C20004EAF5FAFAE9795010B2C000C440B550BCC
:102C3000AE968CAD9DADAEADBFADAE97281B390B3A
:102C40004A0B5B0BC101032C000CAA0BBB0BBC0194
:102C5000CD0164197509860997090E94DFD5D7014E
:102C600019962D913D914D915C911C97AE96CCACEF
:102C7000DDACEEACFFACAE972C193D094E095F09F7
:102C8000AE962CAF3DAF4EAF5FAFAE970E9411D660
:102C9000420E531E641E751EAA962FADAA972530AC
:102CA00091F414C08AE08A9D20018B9D500C112460
:102CB000052C000C66087708E4961FAE1EAEE4975C
:102CC000212C38E2332E81E090E009C064E0C80195
:102CD0000E941B9FDC0119968D919C911A97A1016E
:102CE000032C000C660B770B44155505660577051C
:102CF00034F42A013B01AA24AA9423E0B22EE496DC
:102D0000CEACDFACE497A601DD0C660B770B441666
:102D100055066606770624F42A013B01A12CB12C46
:102D2000AA962FADAA97223009F020C32501BB0C2B
:102D30006608770860E0C8010E941B9FFC0181853E
:102D40009285A385B485481659066A067B060CF45D
:102D5000E8C261E0C8010E941B9FFC018185928549
:102D6000A385B48584159505A605B7050CF4DDC2C9
:102D700081C02AE0289F2001299F500C1124052C96
:102D8000000C66087708E4961FAE1EAEE497212C6F
:102D900098E2392E81E090E0E9C2F4018281853029
:102DA00059F0863009F066C061E070E0CE018B59C1
:102DB0009F4F0E9498915EC061E070E0CE018F59F4
:102DC0009F4F0E94386656C080910E0F801388C2B4
:102DD00080910F0F803409F083C28091100F909181
:102DE000110F6C01990FEE08FF0860E0C5010E9409
:102DF0001B9FFC0181859285A385B485C816D906E1
:102E0000EA06FB060CF46AC061E0C5010E941B9F44
:102E100055245394FC0181859285A385B4858C1536
:102E20009D05AE05BF050CF459C0D4011496ED9173
:102E3000FC9115978181E82FEF708E2F90E0FC01B7
:102E40003197EC30F10508F44BC0F4010481158191
:102E5000D8018C9183FB992790F9951509F43BC211
:102E6000982F907E09F4CEC1982F907E90528F714A
:102E7000892B8C9380E090E0B8C38FEF9FEFB5C3B0
:102E8000202F30E0F901EA54F14E8491F901E65720
:102E9000FF4E0491F901E053FF4EF490FF20A1F0A2
:102EA00081110E94FFA9EF2DF0E0EE0FFF1FE35507
:102EB000F64FA591B491EC910E2331E020E009F496
:102EC00030E0832F922F02C080E090E0212F30E08D
:102ED000552453942817390709F4A7CF512CA5CFAF
:102EE0008827EE58FF4F8F4F0C9466D60E9407AC90
:102EF0009B01AC0144275527D4011496ED91FC9118
:102F0000159782819381BC0180E090E0AA24AA9465
:102F1000BA2CC12CD12C18EEE12E13E0F12E00E0DA
:102F200010E00E948248882309F48FCFF4010081C9
:102F300011816EE675E0C8010E94565A892B09F08E
:102F4000DCC163E775E0C8010E94565A892B09F07D
:102F5000D4C1E4C00E9407AC9B01AC0144275527B3
:102F6000D4011496ED91FC91159782819381BC0157
:102F700080E090E0AA24AA94BA2CC12CD12C1CE2A7
:102F8000E12EFF24F39400E010E01AC00E9407AC89
:102F90009B01AC0144275527D4011496ED91FC9177
:102FA000159782819381BC0180E090E0AA24AA94C5
:102FB000BA2CC12CD12C16E9E12EF12C00E010E046
:102FC0000E948248882309F440CFA30164E0E6C050
:102FD0000E9407AC9B01AC0144275527D4011496ED
:102FE000ED91FC91159782819381BC0180E090E086
:102FF000AA24AA94BA2CC12CD12C18EEE12E13E0ED
:10300000F12E00E010E00E948248882309F41DCFD1
:10301000F4010081118169E775E0C8010E94565AE8
:10302000892B09F06DC16FE775E0C8010E94565AFF
:10303000892B09F065C172C00E9407AC9B01AC01ED
:1030400044275527D4011496ED91FC911597828160
:103050009381BC0180E090E0AA24AA94BA2CC12CF0
:10306000D12C1CE2E12EFF24F39400E010E01AC002
:103070000E9407AC9B01AC0144275527D40114964C
:10308000ED91FC91159782819381BC0180E090E0E5
:10309000AA24AA94BA2CC12CD12C16E9E12EF12C29
:1030A00000E010E00E948248882309F4CECEA301FC
:1030B00069E074C00E9407AC9B01AC01442755270E
:1030C000D4011496ED91FC91159782819381BC01F6
:1030D00080E090E0AA24AA94BA2CC12CD12C18EE3E
:1030E000E12E13E0F12E00E010E00E9482488823D8
:1030F00009F4ABCEF4010081118166E875E0C801E6
:103100000E94565A892B09F009C16CE875E0C80184
:103110000E94565A892B09F001C1F5C0A3016DE048
:103120006DC00E9407AC9B01AC0144275527D40118
:103130001496ED91FC91159782819381BC0180E0FA
:1031400090E0AA24AA94BA2CC12CD12C1CE2E12E26
:10315000FF24F39400E010E01AC00E9407AC9B012A
:10316000AC0144275527D4011496ED91FC91159795
:1031700082819381BC0180E090E0AA24AA94BA2CB9
:10318000C12CD12C16E9E12EF12C00E010E00E94B8
:103190008248882309F459CEA3016CE0C4010E943F
:1031A0002B6DF401048115810E9407ACD8011396A0
:1031B0007C936E93129749CE0E9407AC9B01AC01A1
:1031C00044275527D4011496ED91FC9115978281DF
:1031D0009381BC0180E090E0AA24AA94BA2CC12C6F
:1031E000D12C18E5E12E12E0F12E00E010E00E9453
:1031F0008248882309F429CEA30160E0C4010E941B
:103200002B6D23CE0E9407ACF80173836283D40137
:1032100012968C91129780FF15C0552009F42ACE82
:103220001496ED91FC9115978081886080831496A7
:10323000ED91FC9115976081617070E0C4010E946E
:10324000EA6B18CE652D70E0C4010E94EA6BD401D0
:103250001496ED91FC9115978181552099F08F700E
:10326000823069F028F481112DC0A30161E024C0EF
:10327000853029F0873031F5A3016AE01DC0A30134
:1032800066E01AC0E82FEF708E2F90E0FC013197B6
:10329000ED30F105B8F48827E258FF4F8F4F0C94BA
:1032A00066D6A30162E008C0A30165E005C0A301E2
:1032B00067E002C0A30160E0C4010E942B6D882377
:1032C00009F4D8CDD4011496ED91FC911597808125
:1032D00050FA83F903C08F718066F8018083CACDEC
:1032E00000930E0F80E480930F0F802F0E9489AB14
:1032F0009093110F8093100F74CDA30163E07ECFE4
:10330000A30168E07BCF6CE975E0C8010E94565AC2
:10331000892B09F003CFA30166E070CFA3016BE016
:103320006DCF412C512C320104C0412C512C320163
:103330004394D4011496ED91FC9115978281938169
:10334000092E000CAA0BBB0B84159505A605B70525
:1033500009F490CDB201C4010E94EA6BD401149625
:10336000ED91FC9115975382428284CDD40114963D
:10337000ED91FC911597228133816501C21AD30A20
:103380009601D7FE03C03195219531098217930725
:103390001CF480818F7112C04081842F82958695A4
:1033A0008770282F30E0263031054CF48F5F982F3E
:1033B0009295990F907E842F8F71892B8083D401F1
:1033C0001496ED91FC911597808182958695877072
:1033D00090E00597BCF0E4962EAD3FADE49769010F
:1033E000330FEE08FF084C145D046E047F0451F0A7
:1033F000C101330CAA0BBB0B481659066A067B06A3
:1034000009F038CD828193818A159B0509F432CD6C
:103410006D961CAE1DAE1EAE1FAE6D976C968FAD39
:103420006C978F7080666C968FAF6C976D968CAD35
:103430009DADAEADBFAD6D9765968CAF9DAFAEAF98
:10344000BFAF659769964CAE5DAE6EAE7FAE6997C5
:10345000D40113961C9169EC79E089EF9EE00E94FB
:1034600022B64AE050E0612F89EF9EE00E94B1B69B
:1034700067EC79E089EF9EE00E9422B6CE018F5A78
:103480009F4F0E94449963E975E0F4018081918126
:103490000E94565A6296EFAC62976396FFAC6397B0
:1034A00064960FAD649765961FAD659766962FADD0
:1034B000669767963FAD679768964FAD6897699630
:1034C0005FAD69976FEF0E94C34AD4010D911C91C3
:1034D00067E975E0C8010E94565A6C0165E675E01F
:1034E000C8010E94565A8C010097B9F1FC018085F1
:1034F0008F70843091F56185728540E450E0CE0193
:1035000001960E9417DA6FE270E0CE0101960E94E8
:10351000DED9892B61F4D80119962D913C911A9727
:1035200043E050E060E4CE0101960E94384900E09B
:1035300020E032E040E150E0BE016F5B7F4FCE0102
:103540008F5A9F4F0E9488970E94DD9D882329F003
:103550008091DC0A882309F440C0C114D104A9F188
:10356000F60180858F70843081F561857285CE018A
:1035700001960E94436ACE0101960E9490688823BA
:1035800001F1CC24C394E12CF12C62960FAD62972B
:1035900063961FAD639764962FAD649765963FADB4
:1035A000659766964FAD669767965FAD6797689625
:1035B0006FAD689769967FAD6997CE0101960E94BD
:1035C0002F25CE0101960E9418A0D4011496ED91EA
:1035D000FC911597B382A2824DCCBE016F5B7F4FE9
:1035E000CE0101960E94FF9EB8CFCD58DF4F0FB697
:1035F000F894DEBF0FBECDBFDF91CF911F910F9129
:10360000FF90EF90DF90CF90BF90AF909F908F9002
:103610007F906F905F904F903F902F9008954F92C2
:103620005F926F927F928F929F92AF92BF92CF9252
:10363000DF92EF92FF920F931F93CF93DF93CDB75B
:10364000DEB7C25AD1400FB6F894DEBF0FBECDBF71
:103650002091941030919510F9013B96EA31F105D3
:1036600008F0D8C38827E557FF4F8F4F0C9466D6D4
:103670000AEE13E0CE56DE4F19830883C259D140BB
:10368000CC56DE4F188219821A821B82C459D1404F
:10369000CE57DE4F19830883C258D140CC57DE4F36
:1036A000188219821A821B82C458D140CE59DE4F2B
:1036B00019830883C256D140CC59DE4F1882198233
:1036C0001A821B82C456D140CE5BDE4F1983088319
:1036D000C254D140CC5BDE4F188219821A821B8201
:1036E000C454D14062E87AE08CE49EE00E9422B6A5
:1036F0008CE49EE00E9449B7BE016E567E4F86E084
:1037000090E00E941258892B09F467C16CE67AE0B8
:103710008CE49EE00E9422B61A830983CC56DE4FC9
:1037200088819981AA81BB81C459D1408B839C83B4
:10373000AD83BE83CE0101960E947AB1BE016E5761
:103740007E4F8AE090E00E941258892B09F42EC126
:1037500066E67AE08CE49EE00E9422B61A83098332
:10376000CC57DE4F88819981AA81BB81C458D14052
:103770008B839C83AD83BE83CE0101960E947AB178
:10378000BE016E597E4F8EE090E00E941258892B48
:1037900009F4DFC061E67AE08CE49EE00E9422B684
:1037A0001A830983CC59DE4F88819981AA81BB8114
:1037B000C456D1408B839C83AD83BE83CE010196DA
:1037C0000E947AB1BE016E5B7E4F82E190E00E9462
:1037D0001258892B09F477C06AE57AE08CE49EE000
:1037E0000E9422B61A830983CC5BDE4F88819981BF
:1037F000AA81BB81C454D1408B839C83AD83BE839B
:10380000CE0101960E947AB11A830983CC5BDE4F08
:1038100088819981AA81BB81C454D1408B839C83C8
:10382000AD83BE83CF57DF4F19830883C158D04083
:10383000CC59DE4F88819981AA81BB81C456D14081
:10384000CD57DF4F88839983AA83BB83C358D04069
:10385000CE53DF4F19830883C25CD040CC57DE4F74
:1038600088819981AA81BB81C458D140CC53DF4F54
:1038700088839983AA83BB83C45CD040CE5FDE4F2C
:1038800019830883C250D140CC56DE4F888199817C
:10389000AA81BB81C459D140CC5FDE4F8883998314
:1038A000AA83BB83C450D1409E012F5F3F4FAE011E
:1038B0004F575F4FBE016E537F4FCE018E5F9E4FBD
:1038C0000E94F25685C01A830983CC59DE4F888145
:1038D0009981AA81BB81C456D1408B839C83AD83DF
:1038E000BE83CF57DF4F19830883C158D040CC57D0
:1038F000DE4F88819981AA81BB81C458D140CD57C0
:10390000DF4F88839983AA83BB83C358D040CE53AB
:10391000DF4F19830883C25CD040CC56DE4F8881CC
:103920009981AA81BB81C459D140CC53DF4F888390
:103930009983AA83BB83C45CD040AE014F5F5F4FC5
:10394000BE016F577F4FCE018E539F4F0E943E574F
:103950003FC01A830983CC57DE4F88819981AA81A1
:10396000BB81C458D1408B839C83AD83BE83CF572A
:10397000DF4F19830883C158D040CC56DE4F888171
:103980009981AA81BB81C459D140CD57DF4F88832B
:103990009983AA83BB83C358D040BE016F5F7F4F1A
:1039A000CE018F579F4F0E94905712C01A830983F0
:1039B000CC56DE4F88819981AA81BB81C459D14000
:1039C0008B839C83AD83BE83CE0101960E94DB571F
:1039D0008CE49EE00E9449B7F5C06EE47AE08CE486
:1039E0009EE00E9422B60FB6F894A89580916000E0
:1039F000886180936000109260000FBE8091A50ADC
:103A0000811107C08AE89AE00E94298181E08093B1
:103A1000A50A87E49AE09093DF0C8093DE0C0E9465
:103A20005456CE0101960E9488C589819A810E94D0
:103A30002C7546E050E060E97BE089E090E00E9470
:103A400052BC8AEE93E09A8389831B821C821D827A
:103A50001E82CE0103960E9416750E942B758091DE
:103A6000DE0C9091DF0CDC0192961D921D921D924E
:103A70001C929597FC0116A217A210A611A69A9661
:103A80001D921D921D921C929D9740EE5EE260E099
:103A900070E046AB57AB60AF71AF40EA5FE060E00B
:103AA00070E0DA964D935D936D937C93DD973E962F
:103AB00024E1DF011D922A95E9F726E0E0E9FBE029
:103AC000DC01189601900D922A95E1F7FC01EE5B5E
:103AD000FF4F10820E9472548C01019709F04AC076
:103AE000CE0101960E9488C589819A810E942C7519
:103AF0006091DE0C7091DF0C625F7F4FCE0101960A
:103B00000E9461B7CE0103960E9416756091DE0C8B
:103B10007091DF0C6A5E7F4FCE0101960E9461B703
:103B2000CE0103960E9424756091DE0C7091DF0C2B
:103B30006E5E7F4FCE0101960E9461B7CE01039663
:103B40000E941D750E942B756091DE0C7091DF0C38
:103B5000625E7F4FCE0101960E9461B78B819C818E
:103B6000AD81BE818093DA0C9093DB0CA093DC0CCA
:103B7000B093DD0C99E288E10FB6F894A895809394
:103B800060000FBE90936000A895012B69F46CE073
:103B90007AE084E59EE00E9422B66DED79E084E54E
:103BA0009EE00E9422B630C16DEC79E08CE49EE08C
:103BB0000E9422B6CE0101960E94D0B1CE0101969C
:103BC0000E947AB182E090E021C18091B10A811116
:103BD00003C081E08093B10A83E090E017C1809137
:103BE000DD0A811123C78091460A81110BC060E074
:103BF00070E080E090E00E940B7E08C10E94DD9D95
:103C0000811108C184E090E001C1A895CE55DE4F36
:103C10001882C25AD140FE01EE56FE4F1192119207
:103C20008EE0DF011D928A95E9F70E94DD9D8823D1
:103C300019F085E090E0EAC00091CD0F1091CE0F11
:103C40000115110509F444C2C8010E949C9FE82E89
:103C5000F12CB2E0EB16F1040CF03DC239C20E9427
:103C600007AC9B01AC016091AD0A7091AE0A8091E6
:103C7000AF0A9091B00AAA24AA94BA2C650118E858
:103C8000E12E13E1F12E00E010E00E94824888232B
:103C900009F4C0C020E030E043E050E061E4CE0130
:103CA00001960E94384962EA75E0CE0101960E94B1
:103CB000D3D900910C0D10910D0DB801CE010196D4
:103CC0000E94B4CD09960817190790F10E94DD9D56
:103CD000882371F18091120D9091130D019611F4CA
:103CE00081E090E09093130D8093120DE0910A0D06
:103CF000F0910B0D8091130D8583E0910A0DF091E9
:103D00000B0D8091120D868360910A0D70910B0D41
:103D100047E050E0CE0101960E94149EAC01455050
:103D2000510960910A0D70910B0D82EA0E94349E38
:103D300086E090E090939510809394106CE57CE081
:103D40008CE49EE00E9422B665C00E9407AC60939E
:103D5000AD0A7093AE0A8093AF0A9093B00A85EFD4
:103D60009FEF54C00E9407AC9B01AC016091AD0A6B
:103D70007091AE0A8091AF0A9091B00AAA24AA94D9
:103D8000BA2C650118E8E12E13E1F12E00E010E0F5
:103D90000E948248882309F43DC010929510109229
:103DA000941038C00E94DD9D81110E94FDB10E94D7
:103DB00007AC6093AD0A7093AE0A8093AF0A9093FC
:103DC000B00A8DE090E022C00E9407AC9B01AC01DC
:103DD0006091AD0A7091AE0A8091AF0A9091B00ADD
:103DE000AA24AA94BA2C650110E1E12E17E2F12E63
:103DF00000E010E00E948248811104CF0BC00E94B5
:103E0000A27D892B09F0FECE86EF9FEF909395104F
:103E1000809394100FB6F894A89580916000886103
:103E200080936000109260000FBE8091941090917A
:103E3000951002970CF43DC10091DE0C1091DF0C3F
:103E40000115110509F435C10E9407AC4B015C0155
:103E50007801FEE3EF0EF11CF70180819181A281D0
:103E6000B381A5019401281B390B4A0B5B0BCA01D6
:103E7000B901683E33E073078105910508F446C037
:103E800028EE33E040E050E00E94EFD5861A970A12
:103E9000A80AB90AD7018D929D92AD92BC92139750
:103EA000F80186A597A5A0A9B1A969017A01CC0C52
:103EB000DD1CEE1CFF1C8C159D05AE05BF0528F40E
:103EC00016A617A610AA11AA09C0821B930BA40B51
:103ED000B50BF80186A797A7A0ABB1ABF80182A9F3
:103EE00093A9A4A9B5A98C159D05AE05BF0528F415
:103EF00012AA13AA14AA15AA09C0821B930BA40B19
:103F0000B50BF80182AB93ABA4ABB5ABF80186A5BA
:103F100097A5A0A9B1A9892B8A2B8B2B69F4EE5BFD
:103F2000FF4F8081833041F484E08083C8010E9488
:103F3000725401967C0102C0E12CF12CF80182A997
:103F400093A9A4A9B5A9892B8A2B8B2BA1F4EE5B8D
:103F5000FF4F8081833011F081110DC01082F80174
:103F60003E9684E1DF011D928A95E9F7C8010E941F
:103F7000725403967C01B2E0EB16F10429F0E4E000
:103F8000EE16F10409F04AC0CE0101960E9488C5E0
:103F900089819A810E942C756091DE0C7091DF0CF2
:103FA000625F7F4FCE0101960E9461B7CE010396FA
:103FB0000E9416756091DE0C7091DF0C6A5E7F4F77
:103FC000CE0101960E9461B7CE0103960E9424752E
:103FD0006091DE0C7091DF0C6E5E7F4FCE0101961A
:103FE0000E9461B7CE0103960E941D750E942B7539
:103FF0006091DE0C7091DF0C625E7F4FCE01019606
:104000000E9461B78B819C81AD81BE818093DA0C67
:104010009093DB0CA093DC0CB093DD0CF3E0EF1677
:10402000F10461F15CF431E0E316F104D1F042E017
:10403000E416F104F1F562E27CE02FC054E0E516ED
:10404000F10449F185E0E816F10499F563E57CE0B7
:1040500084E59EE00E9422B684E59EE00E9449B776
:1040600006C06FE37CE084E59EE00E9422B686EF06
:104070009FEF90939510809394101BC06FE07CE0AD
:1040800084E59EE00E9422B60E94DD9D882379F39C
:104090000E94FDB1ECCF63EF7BE08CE49EE00E94D8
:1040A00022B6CE0101960E94D0B1CE0101960E94A7
:1040B0007AB199E288E10FB6F894A89580936000F0
:1040C0000FBE909360002091941030919510AEC473
:1040D0008EE090E09BCE60E070E0C8010E941F97E8
:1040E0008C019093D90A8093D80A66EE7BE08CE429
:1040F0009EE00E9422B6B8018CE49EE00E945FB769
:104100008CE49EE00E9449B763EE7BE089EF9EE07D
:104110000E9422B64AE050E0B70189EF9EE00E947B
:1041200042B789EF9EE00E9449B70091CD0F1091F0
:10413000CE0F61E070E0C8010E941F975C0192E021
:10414000E916F10491F062E0C8010E941B9FFC0196
:10415000C184D284F3E0EF16F10459F063E070E01B
:10416000C8010E941F978C0107C08BE5C82E87E00D
:10417000D82E8E010E551E4F40E150E0BE016E5606
:104180007E4F86E390E00E945E7D892B51F425E00E
:10419000E216F1040CF05FC3AE014E565E4F7A0199
:1041A00004C0CE018E569E4F7C01B092260DA09287
:1041B000250DD092280DC092270D8AE09CE990939E
:1041C0001E0D80931D0D40E150E066EB7BE0CE01BB
:1041D0008E579E4F0E94A1CD20E030E041E050E09C
:1041E00060E2CE018E599E4F0E94384940E250E075
:1041F0006FEA7BE0CE018E599E4F0E9483CD6FE81F
:104200007BE08CE49EE00E9422B6B5018CE49EE047
:104210000E945FB76DE87BE08CE49EE00E9422B6CE
:104220004AE050E0B6018CE49EE00E9442B766E8A6
:104230007BE08CE49EE00E9422B6B8018CE49EE014
:104240000E945FB761E87BE08CE49EE00E9422B6AA
:10425000D8018C91811104C0E12CF12C00E010E018
:10426000A090D80AB090D90A0E94DD9D81117DC12D
:104270008091080D9091090DDC01ED91FC9106886B
:10428000F789E02D19958823A1F081E090E09093C3
:10429000130D8093120D87E0EAE3F2E0DE01119640
:1042A00001900D928A95E1F7FE01319685E090E04C
:1042B00037C06091250D7091260D8091080D909169
:1042C000090D4091270D5091280DDC01ED91FC91D5
:1042D0006115710521F00088F189E02D16C0068472
:1042E000F785E02D2AEE33E03A8329834090210DB3
:1042F0005090220D6090230D7090240D4B825C82B3
:104300006D827E82BE016F5F7F4F1995019709F420
:10431000BCCF8EEF9FEF90932C0D80932B0DAFC2EF
:104320002191A0910A0DB0910B0DA80FB91F2C93EC
:1043300001968C309105A1F70115110529F0E114C2
:10434000F10421F086EF03C086E301C086EBC09044
:104350000A0DD0900B0DF601848780910F0D858793
:1043600080910E0D868780900C0D90900D0DB401FC
:10437000C5010E94B4CD41968816990608F4E9C09B
:104380004FE050E0B601C5010E94149E6C01A09060
:104390000C0DB0900D0DB501CE018E599E4F0E94AF
:1043A000B4CD8C0D9D1D0296A816B90608F4D1C097
:1043B00060910A0D70910B0DA601CE018E599E4F92
:1043C0000E94149E6C01A0900C0DB0900D0DB501D3
:1043D000CE018E579E4F0E94B4CD8C0D9D1D02962E
:1043E000A816B90608F4B5C060910A0D70910B0DBE
:1043F000A601CE018E579E4F0E94149E6C0101159E
:104400001105B9F1A0900C0DB0900D0DB501C801CA
:104410000E94B4CD96012E5F3F4F820F931FA816C6
:10442000B90608F496C060910A0D70910B0DA601B3
:10443000C8010E94149E6C01E114F104D1F00091B6
:104440000C0D10910D0DB801C7010E94B4CD96015D
:104450002E5F3F4F820F931F0817190708F479C08A
:1044600060910A0D70910B0DA601C7010E94149E68
:104470006C01A6014550510960910A0D70910B0D18
:1044800080E10E94349E0E9407AC6093140D7093EB
:10449000150D8093160D9093170D6093180D709362
:1044A000190D80931A0D90931B0D8091080D90911A
:1044B000090DDC01ED91FC910084F185E02D199549
:1044C000892B01F50E9407AC2091100D3091110D40
:1044D000C090180DD090190DE0901A0DF0901B0DA2
:1044E0004B015C018C189D08AE08BF08A8EEB3E034
:1044F0000E9443D686169706A806B906B0F28CEF3E
:104500009FEF23C0CE018F579F4F0E9493AE643020
:10451000710581059105E9F4E0910A0DF0910B0D0B
:104520008381811111C00E9407AC6093180D7093B4
:10453000190D80931A0D90931B0D10921C0D109263
:104540002C0D10922B0D11C090E090932C0D8093A8
:104550002B0D8091080D9091090DDC01ED91FC91DE
:104560000488F589E02D19958AC10091D80A109127
:10457000D90A63E77BE08CE49EE00E9422B6B80192
:104580008CE49EE00E945FB78CE49EE00E9449B7F5
:1045900081E08093460A20E030E043E050E061E4AF
:1045A000CE018F579F4F0E94384962EA75E0CE01D5
:1045B0008F579F4F0E94D3D9CE018F579F4F0E9494
:1045C000FF5520E030E042E050E061E4CE018F573B
:1045D0009F4F0E94384966EA75E0CE018F579F4F82
:1045E0000E94D3D9BE016F577F4F8CE59EE00E9499
:1045F0007B71CE018F579F4F0E94FF5520E030E026
:1046000041E050E061E4CE018F579F4F0E9438494E
:1046100066EA75E0CE018F579F4F0E94D3D9BE0145
:104620006F577F4F8CE59EE00E947B71CE018F57C4
:104630009F4F0E94FF55FE01EE5FFE4F11921192B7
:104640001EE3DF01812E1D928A94E9F71A821982F6
:10465000FE0133968EE7DF011D928A95E9F720E08F
:1046600030E041E050E060E4CE018E5F9E4F0E945A
:10467000384940E450E06FEA7BE0CE018E5F9E4F08
:104680000E9483CD40E850E06CE27BE0CE010196D1
:104690000E94A1CDBE016F5F7F4FCE018E5F9E4F06
:1046A0000E94FF9E20E030E041E050E060E4CE0157
:1046B0008E5F9E4F0E94384940E450E066E27BE006
:1046C000CE018E5F9E4F0E9483CD40E850E06CE1AA
:1046D0007BE0CE0101960E94A1CD40E850E069E068
:1046E0007BE0CE0101960E9483CDBE016F5F7F4FBC
:1046F000CE018E5F9E4F0E94FF9E20E030E041E0A1
:1047000050E060E4CE018E5F9E4F0E94384940E445
:1047100050E069E67DE1CE018E5F9E4F0E9483CD21
:1047200040E850E069EF7AE0CE0101960E94A1CD09
:10473000BE016F5F7F4FCE018E5F9E4F0E94FF9E36
:1047400020E030E041E050E060E4CE018E5F9E4F1B
:104750000E94384940E450E062EF7AE0CE018E5F7B
:104760009E4F0E9483CD40E850E06CEE7AE0CE018F
:1047700001960E94A1CDBE016F5F7F4FCE018E5F7B
:104780009E4F0E94FF9E8091DD0A8F5F8093DD0A1D
:10479000A0919610B0919710109709F444C08091A1
:1047A000410290914202AE014E5B5E4FFA0181934D
:1047B00091932EE111922A95E9F79E012E533F4FD6
:1047C000F9018193919311921A95E9F716960D913B
:1047D0001C911797E0909610F0909710E114F10457
:1047E00079F00115110561F0D80118968C918F7040
:1047F0008530A1F7C8010E949C9F882379F367C088
:1048000020E030E041E050E060E4CE018E5F9E4F5A
:104810000E94384940E450E06FE87AE0CE018E5FB4
:104820009E4F0E9483CD8091DD0A81508093DD0AE6
:1048300085E090E090939510809394100E9407ACCF
:104840006093AD0A7093AE0A8093AF0A9093B00A5A
:1048500066E57BE075CA64E070E08091CD0F9091D1
:10486000CE0F0E941F977C0163EC7BE08CE49EE0FE
:104870000E9422B68CE49EE00E9449B796CC00913B
:104880002B0D10912C0D6AE47BE084E59EE00E94E4
:1048900022B64AE050E0B80184E59EE00E9442B7AB
:1048A00062E37BE084E59EE00E9422B684E59EE020
:1048B0000E9449B70E9407AC6093AD0A7093AE0A9C
:1048C0008093AF0A9093B00A8CE090E09FCA60E0BA
:1048D000C8010E941B9FFC0181859285A385B48538
:1048E0008A30910508F463C020E030E041E050E0F8
:1048F00060E4CE018E5F9E4F0E943849F8016081CE
:10490000718140E450E0CE018E5F9E4F0E94F9D944
:1049100068EA75E0CE018E5F9E4F0E94D3D940E4D5
:1049200050E06EE97AE0CE018E5F9E4F0E9483CD0B
:10493000BE016E5B7E4FCE018E5F9E4F0E94FF9E3A
:10494000CE53DF4F8881C25CD040882361F120E0E4
:1049500030E041E050E060E4CE018E5F9E4F0E9467
:104960003849D8016D917C9140E450E0CE018E5FD2
:104970009E4F0E94F9D968EA75E0CE018E5F9E4F86
:104980000E94D3D940E450E066E97AE0CE018E5F20
:104990009E4F0E9483CDBE016E537F4FCE018E5F2E
:1049A0009E4F0E94FF9EF8010281138113CFFC01EC
:1049B00040E250E08827EB55FF4F8F4F0C9466D6AE
:1049C00066EE7AE0CE018E5B9E4F0E94A1CDCE5363
:1049D000DF4F1882C25CD04087CF61EE7AE0CE0113
:1049E0008E5B9E4F0E94A1CD40E450E060EC7AE0E7
:1049F00017C06AEB7AE0CE018E5B9E4F0E94A1CD7C
:104A000040E450E066EB7AE00BC06EEA7AE0CE015B
:104A10008E5B9E4F0E94A1CD40E450E068EA7AE0B0
:104A2000CE018E539F4F0E94A1CD5ECFC901CE55BE
:104A3000DE4F0FB6F894DEBF0FBECDBFDF91CF9132
:104A40001F910F91FF90EF90DF90CF90BF90AF90AC
:104A50009F908F907F906F905F904F9008952F92CE
:104A60003F924F925F926F927F928F929F92AF92FE
:104A7000BF92CF92DF92EF92FF920F931F93CF934B
:104A8000DF93CDB7DEB7C75BD1090FB6F894DEBFB1
:104A90000FBECDBF5C01C755DF4F0883C95AD04058
:104AA000C655DF4F1883CA5AD040822FC555DF4FF5
:104AB0002883CB5AD040C455DF4F3883CC5AD040DE
:104AC000C355DF4F4883CD5AD040C255DF4F58837E
:104AD000CE5AD040C155DF4F6883CF5AD040C05521
:104AE000DF4F7883C05BD040CF54DF4FF982E8823C
:104AF000C15BD040C954DF4FC882C75BD0408F70C4
:104B0000682E712C4091941050919510CD54DF4F28
:104B100059834883C35BD040EE2DFF2D309719F0A9
:104B20008081811121C0D5011B968C91882341F091
:104B3000C5010B96CF54DF4F99838883C15BD0406A
:104B40006114710409F055C0CF54DF4FE881F98139
:104B5000C15BD040309761F4F501658876886114B7
:104B6000710409F446C010C06114710409F041C019
:104B70008081882389F3CE018F549F4F0E945A6809
:104B80003C01892B49F335C0C555DF4F8881CB5A8D
:104B9000D0408F7071F5662DCE0187559F4F0E94D2
:104BA000859AC756DF4F2883C959D040C656DF4F74
:104BB0003883CA59D040C556DF4F4883CB59D040BF
:104BC000C456DF4F5883CC59D040C356DF4F68835B
:104BD000CD59D040C256DF4F7883CE59D040C15610
:104BE000DF4F8883CF59D040C056DF4F9883C05ADB
:104BF000D0400E94294A1B012C018B01CF54DF4F6A
:104C0000E880F980C15BD040D501ED91FC91C08076
:104C1000D18063E77DE089EF9EE00E9422B64AE002
:104C200050E0B10189EF9EE00E9442B76CE67DE062
:104C300089EF9EE00E9422B6B60189EF9EE00E94B5
:104C40005FB766E67DE089EF9EE00E9422B6B7017D
:104C500089EF9EE00E945FB760E67DE089EF9EE00D
:104C60000E9422B66DE57DE089EF9EE00E9422B6AB
:104C7000083C11054CF46FE47DE084E59EE00E9461
:104C800022B684E59EE0A5C0CE0187559F4F0E94C5
:104C90004499F50180819181892B11F40C94002FA6
:104CA000C5010E947E514C01CC24C39418161906EC
:104CB0000CF0C12C89EF9EE00E9449B7D5011896EF
:104CC0008C91873009F489C0CF54DF4F0881198156
:104CD000C15BD0400115110509F45AC067EF7FE0B0
:104CE000C8010E946ACD892BD9F163EF7FE0C8012A
:104CF0000E946ACD892BB9F164E87CE0C8010E946A
:104D00006ACD892B99F160E87CE0C8010E946ACDE8
:104D1000892B79F16CEB7FE0C8010E946ACD892B69
:104D200059F167EB7FE0C8010E946ACD892B39F108
:104D300061EC7FE0C8010E946ACD892B19F167E719
:104D40007CE0C8010E946ACD892BF9F063E77CE022
:104D5000C8010E946ACD892BD9F40EE010E01AC078
:104D600001E010E017C002E010E014C005E010E020
:104D700011C006E010E00EC00AE010E00BC00BE02E
:104D800010E008C00CE010E005C00DE010E002C02B
:104D900000E010E0C5010E94366AE82EF12CE11413
:104DA000F10411F4EC2CF12C01151105B1F0E01611
:104DB000F10699F069E37DE089EF9EE00E9422B65A
:104DC0004AE050E0B70189EF9EE00E9442B789EFC8
:104DD0009EE00E9449B70C94002FCF55DF4F1882F8
:104DE00019821A821B82C15AD040CB55DF4F1882DC
:104DF00019821A821B82C55AD040CD55DF4F888157
:104E0000C35AD0408F70CD55DF4F8883C35AD040EE
:104E1000CF55DF4F1882C15AD04040E0B501CE01D6
:104E20008F559F4F0E94EE99811182C06CE17DE009
:104E300089EF9EE00E9422B6F50181859285009758
:104E400041F0DC01ED91FC91028CF38DE02D199580
:104E500003C0F501808590E08D30910528F4FC01B8
:104E6000E456FB4F808101C080E08F70282F22958F
:104E7000207FCD55DF4F9881C35AD0409F70922B31
:104E8000CD55DF4F9883C35AD040843028F4823008
:104E9000C8F4813069F133C0883039F0893079F550
:104EA00080E090E0A6E9B2E404C080E090E0A0EAEF
:104EB000B1E4CB55DF4F88839983AA83BB83C55A5E
:104EC000D04025C084E6C955DF4F8883C75AD040FB
:104ED000C855DF4F8881C85AD0408E7FC855DF4FF4
:104EE0008883C85AD040CA55DF4F1882C65AD0406E
:104EF0008FEFCB55DF4F8883C55AD04008C0CB55C4
:104F0000DF4F188219821A821B82C55AD04040E0B6
:104F1000B501CE018F559F4F0E949699CE018F55B6
:104F20009F4F0E94449960E07AE0C5010E942A4F99
:104F3000C755DF4F6881C95AD040643089F038F4D2
:104F4000662309F4CEC2633009F49DC049C46730BA
:104F500009F4FEC008F444C46A3008F448C140C4EF
:104F6000181419047CF562E0CE018F559F4F0E9402
:104F7000AD9ACF56DF4F2883C159D040CE56DF4F70
:104F80003883C259D040CD56DF4F4883C359D040F3
:104F9000CC56DF4F5883C459D040CB56DF4F68837F
:104FA000C559D040CA56DF4F7883C659D040C9563C
:104FB000DF4F8883C759D040C856DF4F9883C85900
:104FC000D0402EC061E0CE018F559F4F0E94AD9A18
:104FD000C757DF4F2883C958D040C657DF4F3883A3
:104FE000CA58D040C557DF4F4883CB58D040C4572C
:104FF000DF4F5883CC58D040C357DF4F6883CD581C
:10500000D040C257DF4F7883CE58D040C157DF4FD2
:105010008883CF58D040C057DF4F9883C059D040C5
:10502000CF55DF4F6881C15AD040CE0187559F4F81
:105030000E94AD9ACF57DF4F2883C158D040CE573A
:10504000DF4F3883C258D040CD57DF4F4883C35815
:10505000D040CC57DF4F5883C458D040CB57DF4F98
:105060006883C558D040CA57DF4F7883C658D040B0
:10507000C957DF4F8883C758D040C857DF4F988340
:10508000C858D040C8C3D50118968C91873009F410
:10509000C4C3C5010E94366A082F10E0853009F0AC
:1050A000B1C66DE07DE089EF9EE00E9422B64AE045
:1050B00050E0B80189EF9EE00E9442B789EF9EE080
:1050C0000E9449B7F5018085853019F56CE0CE0165
:1050D0008F559F4F0E94AD9AEA962FAFEA97EB96B5
:1050E0003FAFEB97EC964FAFEC97ED965FAFED9738
:1050F000EE966FAFEE97EF967FAFEF97C158DF4F09
:105100008883CF57D040C058DF4F9883C058D040D5
:1051100082C361E0CE018F559F4F0E94AD9AE29607
:105120002FAFE297E3963FAFE397E4964FAFE49754
:10513000E5965FAFE597E6966FAFE697E7967FAFA8
:10514000E797E8968FAFE897E9969FAFE99763C333
:10515000D50118968C91873009F45FC3C5010E9470
:10516000366A082F10E0863081F56CEF7CE089EF1D
:105170009EE00E9422B64AE050E0B80189EF9EE02E
:105180000E9442B789EF9EE00E9449B762E0CE01DB
:105190008F559F4F0E94AD9AAA962FAFAA97AB96B4
:1051A0003FAFAB97AC964FAFAC97AD965FAFAD97B7
:1051B000AE966FAFAE97AF967FAFAF97E0968FAFDB
:1051C000E097E1969FAFE19726C364EE7CE089EF1C
:1051D0009EE00E9422B64AE050E0B80189EF9EE0CE
:1051E0000E9442B789EF9EE00E9449B70BC660E07B
:1051F000CE018F559F4F0E94AD9AA2962FAFA297D6
:10520000A3963FAFA397A4964FAFA497A5965FAF81
:10521000A597A6966FAFA697A7967FAFA797A896D4
:105220008FAFA897A9969FAFA997C555DF4F8881E3
:10523000CB5AD040807F41F0CE0187559F4F0E94CE
:10524000D29B8B01672B11F405E010E0C755DF4FAF
:105250008881C95AD040893019F4119501951109F6
:10526000B2E06B16710499F03CF46114710409F01A
:10527000D4C2CC24C3940BC0F9E06F16710409F4B6
:105280009EC02AE06216710409F4ECC0C6C2CD5576
:10529000DF4F8881C35AD040E82FE295EF708E2F00
:1052A00090E0FC013197EB30F10508F0B6C2882799
:1052B000E155FF4F8F4F0C9466D6CB55DF4F888159
:1052C000C55AD040080F111D0F3F110509F02CF4ED
:1052D00017FF05C000E010E002C00FEF10E0CB5553
:1052E000DF4F0883C55AD0406EC2CB55DF4F68816F
:1052F0007981C55AD040060F171F053611052CF4C9
:1053000017FF05C000E010E002C004E610E0012E27
:10531000000C220B330BCB55DF4F088319832A83F4
:105320003B83C55AD0404FC2CB55DF4F688179814E
:105330008A819B81C55AD0400E9477D7600F711F28
:10534000653671052CF477FF05C060E070E002C09F
:1053500064E670E0072E000C880B990B0E94ACD419
:10536000CB55DF4F688379838A839B83C55AD040AE
:105370002AC2CB55DF4F88819981C55AD0404AE077
:10538000409F9001419F300D1124820F931F893E51
:1053900043E094072CF497FF05C080E090E002C042
:1053A00088EE93E0092E000CAA0BBB0BCB55DF4F08
:1053B00088839983AA83BB83C55AD04004C2CD5544
:1053C000DF4F8881C35AD04082958F70823009F0B8
:1053D00024C2C955DF4F6881C75AD040C855DF4F36
:1053E0008881C85AD040782F7170060F171F0E366B
:1053F00051E015072CF417FF05C00DE611E002C0BF
:1054000000E010E0C955DF4F0883C75AD040C855A7
:10541000DF4F8881C85AD04010FB80F9C855DF4F54
:105420008883C85AD04062E0CE018F559F4F0E94BA
:10543000859A6A962FAF6A976B963FAF6B976C967B
:105440004FAF6C976D965FAF6D976E966FAF6E971F
:105450006F967FAF6F97A0968FAFA097A1969FAFE3
:10546000A197B1C1CD55DF4F8881C35AD0408295F5
:105470008F70823009F0D1C1CA55DF4F8881C65A7A
:10548000D040080F111D053611052CF417FF05C07B
:1054900000E010E002C004E610E0CA55DF4F0883C8
:1054A000C65AD04062E0CE018F559F4F0E94859A28
:1054B00062962FAF629763963FAF639764964FAF44
:1054C000649765965FAF659766966FAF66976796C8
:1054D0007FAF679768968FAF689769969FAF699718
:1054E00072C1C555DF4F8881CB5AD040807F09F407
:1054F00094C189E06816710409F438C154F4611448
:105500007104F9F0A2E06A16710409F086C1D12C89
:1055100060C0BBE06B16710409F44AC10CF4F3C01F
:10552000FCE06F16710409F078C188E0FE01E755D0
:10553000FF4FDE01AF55BF4F01900D928A95E1F705
:105540006CC1181419043CF5CE0187559F4F0E9479
:10555000D29B672B682B692B59F562E0CE018F55E2
:105560009F4F0E94AD9A2A962FAF2A972B963FAF56
:105570002B972C964FAF2C972D965FAF2D972E968D
:105580006FAF2E972F967FAF2F9760968FAF609754
:1055900061969FAF61971814190454F0CE01875596
:1055A0009F4F0E94D29B672B682B692B09F030C458
:1055B000CF55DF4F6881C15AD040C5010E940B6AA8
:1055C00060E079E0C5010E942A4FDD24D394CC2409
:1055D000C394CD55DF4F8881C35AD040982F929500
:1055E0009F70945F9F70923050F4C555DF4F988143
:1055F000CB5AD04092959F70923009F428C4D501BF
:1056000018962C91273061F4C555DF4F8881CB5A0D
:10561000D040807E803209F422C4803409F41FC453
:10562000F50181859285009741F0DC01ED91FC91B7
:10563000028CF38DE02D199502C0822F90E07C0141
:10564000C755DF4F0881C95AD040C655DF4F188172
:10565000CA5AD040C555DF4F2881CB5AD040C455D7
:10566000DF4F3881CC5AD040C355DF4F4881CD5AE7
:10567000D040C255DF4F5881CE5AD040C155DF4F80
:105680006881CF5AD040C055DF4F7881C05BD04091
:10569000CE018F559F4F0E94AC8629AF3AAF4BAFDA
:1056A0005CAF6DAF7EAF8FAF21969FAF2197DD20AE
:1056B00009F489C0CD55DF4F8881C35AD040829507
:1056C0008F708150823008F07EC0CB55DF4F28812B
:1056D000C55AD04030E0AFEFB0E00E9443D661152C
:1056E000B4E67B07810591053CF424E630E040E018
:1056F00050E00E9411D601C02FEFCB55DF4F288319
:10570000C55AD04060C0C255DF4F9881CE5AD040B4
:10571000CD55DF4F8881C35AD040282F22952F7056
:1057200019F0223041F079C08F708062CD55DF4F83
:105730008883C35AD040892F90E08536910514F0B4
:1057400084E690E0CA55DF4F8883C65AD04062E0B5
:10575000CE018F559F4F0E94859A29AB3AAB4BAB38
:105760005CAB6DAB7EAB8FAB98AF2DC0C155DF4F3F
:105770006881CF5AD040C055DF4F7881C05BD040A0
:105780007170CE018F559F4F0E94B76E882309F428
:1057900044C062E0CE018F559F4F0E94859A29A791
:1057A0003AA74BA75CA76DA77EA78FA798AB0BC0A6
:1057B000CE0187559F4F0E947A85BC01CE018F553F
:1057C0009F4F0E949C8540E0B501CE018F559F4FB1
:1057D0000E94969960E07AE0C5010E942A4F1DC0A0
:1057E000CE018F559F4F0E94AD9A29A33AA34BA398
:1057F0005CA36DA37EA38FA398A7662DCE018F55C2
:105800009F4F0E94859A298F3A8F4B8F5C8F6D8FA7
:105810007E8F8F8F98A3CC24C394F501418452844A
:105820004114510409F433C1C755DF4F8881C95A67
:10583000D04090E08A30910508F0D3C0FC01882761
:10584000E654FF4F8F4F0C9466D61814190454F188
:1058500067ED7CE089EF9EE00E9422B6D5011996A3
:10586000ED91FC911A970190F081E02D8488958844
:10587000CF54DF4FE880F980C15BD04061E0CE01BA
:105880008F559F4F0E94AD9ACC24C39489019A01F1
:10589000AB01BC01F50181859285F40119958C015C
:1058A00066E053C067EC7CE05BC0181419043CF55B
:1058B000D201ED91FC9184889588CF54DF4FE88028
:1058C000F980C15BD04062E0CE018F559F4F0E94AE
:1058D000AD9ACC24C39489019A01AB01BC01F501B6
:1058E00081859285F40119958C0165E0C5010E94BE
:1058F0000B6A60E071E0C5010E942A4FC6C065EBEB
:105900007CE02EC0C5010E94366A853039F1D20193
:10591000ED91FC9184889588CF54DF4FE880F98021
:10592000C15BD04062E0CE018F559F4F0E94AD9A7F
:10593000CC24C39489019A01AB01BC01F501818596
:105940009285F40119958C0162E0C5010E940B6AF1
:1059500060E071E0C5010E942A4F86C065EA7CE0E4
:1059600089EF9EE00E9422B64DC2CF54DF4FE880FF
:10597000F980C15BD040D201ED91FC910488F5899A
:10598000E02DCF55DF4F0881C15AD040CE55DF4FB3
:105990001881C25AD040CD55DF4F2881C35AD0401C
:1059A000CC55DF4F3881C45AD040CB55DF4F4881AA
:1059B000C55AD040CA55DF4F5881C65AD040C95544
:1059C000DF4F6881C75AD040C855DF4F7881C85A29
:1059D000D040C20119958C0147C0181419040CF469
:1059E00041C0CF54DF4FE880F980C15BD040D20185
:1059F000ED91FC910488F589E02DCC24C394CF551A
:105A0000DF4F0881C15AD040CE55DF4F1881C25AAE
:105A1000D040CD55DF4F2881C35AD040CC55DF4F01
:105A20003881C45AD040CB55DF4F4881C55AD04049
:105A3000CA55DF4F5881C65AD040C955DF4F6881DB
:105A4000C75AD040C855DF4F7881C85AD040C201EC
:105A500019958C01CF55DF4F6881C15AD04066231C
:105A600019F073CF0FEF1FEF69E97CE089EF9EE03B
:105A70000E9422B64AE050E0B80189EF9EE00E9401
:105A800042B789EF9EE00E9449B7C801F5C1F50110
:105A900080858630C9F138F4843009F40BC1853033
:105AA00009F49AC092C1883009F462C120F08930AB
:105AB00009F42FC18AC1C954DF4FF881C75BD040B8
:105AC000FF2309F482C1D5011296ED91FC91139741
:105AD00090859F70953009F078C1CD54DF4F488193
:105AE0005981C35BD0404530510509F46EC1CF5494
:105AF000DF4F48815981C15BD040BE0167557F4F60
:105B0000CF010E94E46A61C160E070E0C5010E94BB
:105B100057698C01009709F458C197FF07C0119588
:105B20000195110966246394712C02C0612C712CBB
:105B3000C80101978634910508F047C1CF55DF4F62
:105B4000E880C15AD040F12CD02E61E0802F0E9415
:105B500084AA672869F051E0E516F10429F061E0B4
:105B600086E0E816F10409F460E0E62EF12C12C09C
:105B700091E0E916F10451F091E080E0A6E0EA1628
:105B8000F10409F090E0E92EF82E03C0EE24E3942E
:105B9000F12C6E2D8D2D0E9455AA64E97CE089EFD1
:105BA0009EE00E9422B64AE050E0B80189EF9EE0F4
:105BB0000E9442B762E97CE089EF9EE00E9422B633
:105BC0004AE050E0B70189EF9EE00E9442B789EFBA
:105BD0009EE00E9449B7F9C0B2E06B16710409F467
:105BE00061C0ECE06E16710409F0EFC0C5010E94BF
:105BF0003C696B017C01EF2849F4D501ED91FC91E2
:105C0000608171818AEA95E00E949B6ECE018F557A
:105C10009F4F0E94949B20E030E048EC52E40E94A9
:105C20000BD50E9477D7CD54DF4F688379838A8361
:105C30009B83C35BD040CD54DF4FC880D980C35B0A
:105C4000D04088E00E946C482B013C017B016EE84B
:105C50007CE089EF9EE00E9422B64AE050E0CD54FD
:105C6000DF4F68817981C35BD04089EF9EE00E945D
:105C700042B769E87CE089EF9EE00E9422B6B3015A
:105C8000A201662777272AE089EF9EE00E945BB693
:105C900089EF9EE00E9449B7B701A601C5010E94A5
:105CA000DE6893C040E0B501CE018F559F4F0E9442
:105CB00096998BC0CC2009F488C0CF55DF4F08815E
:105CC000C15AD040CE55DF4F1881C25AD040CD5571
:105CD000DF4F2881C35AD040CC55DF4F3881C45A9A
:105CE000D040CB55DF4F4881C55AD040CA55DF4F11
:105CF0005881C65AD040C955DF4F6881C75AD04035
:105D0000C855DF4F7881C85AD040C5010E945C4E0B
:105D10005CC0CC2009F459C0CF55DF4F0881C15A6F
:105D2000D040CE55DF4F1881C25AD040CD55DF4FFD
:105D30002881C35AD040CC55DF4F3881C45AD04057
:105D4000CB55DF4F4881C55AD040CA55DF4F5881E7
:105D5000C65AD040C955DF4F6881C75AD040C85590
:105D6000DF4F7881C85AD040C5010E947F4D2DC0B9
:105D7000CC2059F1CF55DF4F0881C15AD040CE55C4
:105D8000DF4F1881C25AD040CD55DF4F2881C35A0A
:105D9000D040CC55DF4F3881C45AD040CB55DF4F6F
:105DA0004881C55AD040CA55DF4F5881C65AD040A5
:105DB000C955DF4F6881C75AD040C855DF4F788139
:105DC000C85AD040C5010E945752CF55DF4F688155
:105DD000C15AD0406623C9F0C755DF4F8881C95AE0
:105DE000D040853021F4181419047CF465E0C50115
:105DF0000E940B6A60E071E0C5010E942A4F05C055
:105E00008FEF01C08DEF9FEF37C081E090E034C08D
:105E100061E0CE018F559F4F0E94AD9A22962FAF21
:105E2000229723963FAF239724964FAF249725962A
:105E30005FAF259726966FAF269727967FAF279758
:105E400028968FAF289729969FAF2997B1CB8F704F
:105E50008062CD55DF4F8883C35AD040D0CBCD551B
:105E6000DF4F9881C35AD0409F709062CD55DF4F6D
:105E70009883C35AD040D4CBC954DF4F0FB6F8949F
:105E8000DEBF0FBECDBFDF91CF911F910F91FF906D
:105E9000EF90DF90CF90BF90AF909F908F907F90CA
:105EA0006F905F904F903F902F900895089583E0FA
:105EB00090E008958091B20A9091B30A08952F92CC
:105EC0003F924F925F926F927F928F929F92AF928A
:105ED000BF92CF92DF92EF92FF920F931F93CF93D7
:105EE000DF93CDB7DEB72E970FB6F894DEBF0FBEA7
:105EF000CDBF1C010E947712D10114968D919C9107
:105F00001597892B79F484E190E00E9473CABC0153
:105F1000F101828193810E949C68D10115969C9326
:105F20008E931497F1010480F581E02DFA87E987BB
:105F3000EF2B59F463E17EE084E59EE00E9422B6F7
:105F400084E59EE00E9449B7EAC2A985BA851D9200
:105F50001C92F1010280F381E02DFE87ED87028122
:105F60001381EF2B09F462C20115110509F45EC219
:105F7000D80118968C918F70853009F057C2C801EE
:105F80000E949C9F882309F451C260E0C8010E94CE
:105F90001B9F8C01FC0180858F70853039F06AEB86
:105FA0007DE084E59EE00E9422B6A2C2C8010E9464
:105FB0009C9F823031F148F4813009F06BC0C12CD4
:105FC000D12C7601460157013BC0863008F062C0F3
:105FD00062E0C8010E941B9FFC0190859F70933076
:105FE00029F4C184D284E384F4840EC0923049F44D
:105FF00061857285838594850E94ACD46B017C0198
:1060000003C0C12CD12C760161E0C8010E941B9F06
:10601000FC0190859F70933029F481849284A3843D
:10602000B4840EC0923049F461857285838594856D
:106030000E94ACD44B015C0103C0812C912C540113
:1060400060E0C8010E941B9FFC0190859F70933007
:1060500029F441845284638474840AC0923021F507
:1060600061857285838594850E94ACD42B013C01A7
:1060700020E030E0A901C301B2010E94A5D487FF4E
:1060800019C077FA709477F87094E1E0F0E0FC873B
:10609000EB8712C01C861B86C12CD12C76014601D1
:1060A00057012601370108C01C861B86412C512C44
:1060B000320102C01C861B86AD85BE851496ED910B
:1060C000FC91159780858295807F8595859585952E
:1060D0008595823039F0833091F481859285A3854E
:1060E000B48511C061857285838594850E94ACD486
:1060F000E985FA8562877387848795870AC080E07F
:1061000090E0A0EAB1E4E985FA8582879387A487C5
:10611000B5878CE390E00E9473CA8C0189859A85CB
:106120000296D8015F969C938E935E9789859A8597
:1061300006965D969C938E935C9789859A850A96C0
:1061400091969C938E939097DA961C92F80112AADE
:1061500013AA14AA15AA80E090E0AFE7B3E486ABD7
:1061600097ABA0AFB1AF84E690E0A0E0B0E086A727
:1061700097A7A0ABB1AB8B859C85918F808F20E0DA
:1061800030E0A901C301B2010E94A5D487FD7DC002
:1061900020E030E0A901C501B4010E94A5D487FD2B
:1061A00074C020E030E0A901C701B6010E94A5D467
:1061B00087FD6BC081E090E0D8015B969C938E9345
:1061C0005A97DB968C93DB97F8014082518262826A
:1061D000738214968D929D92AD92BC921797C08651
:1061E000D186E286F3861C964D925D926D927C92EA
:1061F0001F972DEC3CEC4CEC5DE3C501B4010E9413
:106200000BD54B015C01F801608B718B828B938BFA
:106210002DEC3CEC4CEC5DE3C701B6010E9405D7C8
:106220006B017C01D80154966D937D938D939C9363
:106230005797EB85FC85319741F5A301920160E00A
:1062400070E0CB010E9498D6D8011C966D937D9387
:106250008D939C931F97A501940160E070E0CB01A2
:106260000E9498D6F801608B718B828B938BA7016B
:10627000960160E070E0CB010E9498D6D801549658
:106280006D937D938D939C9357970E9407ACF80173
:1062900086A497A4A0A8B1A8DC01CB01881999090C
:1062A000AA09BB0982A393A3A4A3B5A3D101149601
:1062B000ED91FC911597118300830115110509F4E7
:1062C0001BC1F80182AD81113BC0068CF78DE02D1A
:1062D000C080D180E280F380D8019696CD92DD9285
:1062E000ED92FC9299975C96ED91FC915D9780817F
:1062F0009181A281B381F80182A793A7A4A7B5A732
:1063000046A857A860AC71ACA3019201C701B601C1
:106310000E94ADD718166CF0F80142A853A864A8E3
:1063200075A8A3019201C701B6010E94A5D487FFF9
:1063300007C0D80196964D925D926D927C92999786
:1063400081E0F80182AFC501B4010E94AAD49B018B
:10635000AC0160E070E48CE995E40E9405D76B0124
:106360007C019B01AC01D80150966D917D918D917E
:106370009C9153970E940BD5F801608B718B828B97
:10638000938BA701960164897589868997890E94F4
:1063900005D7D80154966D937D938D939C93579711
:1063A00088E893E1A0E0B0E0F80186A797A7A0AB4A
:1063B000B1ABD1011296ED91FC9113970190F08150
:1063C000E02D008111816FEE7DE08CE49EE00E9463
:1063D00022B6B8018CE49EE00E945FB78CE49EE098
:1063E0000E9449B7F1018281938119821A821B822E
:1063F0001C821D821E821F8218862B812F70CC2446
:10640000C394E12CF12C01E01A813C8140E05E81D3
:106410006F8178850E942F25D1011496ED91FC9112
:10642000159781E090E0938B828B7BC0C8010E941E
:106430009C9FE82ED80118968C918F70FF24F394BE
:10644000853009F4F12C6BED7DE084E59EE00E943F
:1064500022B64AE050E061E070E084E59EE00E94F0
:1064600042B769ED7DE084E59EE00E9422B661E0DE
:1064700070E0ED85FE85EF2B11F460E070E04AE0FE
:1064800050E084E59EE00E9442B767ED7DE084E540
:106490009EE00E9422B661E070E0012B11F460E002
:1064A00070E04AE050E084E59EE00E9442B765ED6E
:1064B0007DE084E59EE00E9422B66F2D70E04AE008
:1064C00050E084E59EE00E9442B763ED7DE084E504
:1064D0009EE00E9422B661E070E0F1E0FE1510F44B
:1064E00060E070E04AE050E084E59EE00E9442B740
:1064F00084E59EE00E9449B762E07EE084E59EE08C
:106500000E9422B684E59EE00E9449B7D10114960C
:10651000ED91FC91159782E090E0938B828B80E067
:1065200090E02E960FB6F894DEBF0FBECDBFDF9180
:10653000CF911F910F91FF90EF90DF90CF90BF9080
:10654000AF909F908F907F906F905F904F903F9013
:106550002F9008950C940BCBCF92DF92EF92FF9285
:106560000F931F93CF93DF93CDB7DEB728970FB666
:10657000F894DEBF0FBECDBF6C01822F2B838F70CE
:10658000E82EF12C002331F0E114F10419F4EE248B
:10659000E394F12C60E070E1F601828193810E9426
:1065A000BC69F1E0EF16F10481F082E0E816F10435
:1065B00041F0EF2851F569EA7DE089EF9EE00E9405
:1065C00022B68B81807F59F10AC0602FF60182814B
:1065D00093810E940B6A013011F00230B1F4F60190
:1065E000828193810E943C69672B682B692B51F053
:1065F00080E00E946C48AB01BC01F601828193816E
:106600000E94DE6881E090E00CC06DE97DE089EFDA
:106610009EE00E9422B689EF9EE00E9449B780E08A
:1066200090E028960FB6F894DEBF0FBECDBFDF9185
:10663000CF911F910F91FF90EF90DF90CF90089531
:10664000CF93DF93EC0169EB75E08CE59EE00E944F
:106650007B716D858C810E9455AA6D858D810E940C
:1066600055AA40E050E0BA018A819B810E94DE6811
:106670001092B30A1092B20A81E090E0DF91CF91BC
:1066800008952F923F924F925F926F927F928F92D6
:106690009F92AF92BF92CF92DF92EF92FF920F93B1
:1066A0001F93CF93DF93CDB7DEB760970FB6F89403
:1066B000DEBF0FBECDBF4C01FC01E280F38060E085
:1066C00070E1C7010E94F469892B09F46EC260E091
:1066D00070E2C7010E94F469892B79F4809100026D
:1066E000882309F462C260E070E2C7010E94BC69BD
:1066F00080910002815080930002F401E280F380D7
:10670000C7010E943C692B013C0119821A821B823D
:106710001C821D821E821F8218868B818F708B8344
:10672000198240E0B701CE0101960E94EE9960E027
:10673000CE0101960E94D19A9A878987F4018281BD
:1067400093810E94366A823011F0853011F41A86E6
:106750001986F40186819AEC980F9031B0F5218565
:106760003285A90160E070E04D875E876F87788B86
:10677000C384D484E12CF12C0E9489AB9C878B8745
:10678000092E000CAA0BBB0B9C01AD012C193D0975
:106790004E095F09AFEFB0E00E9430D62D853E85EF
:1067A0004F8558892C193D094E095F090E9411D661
:1067B000190137FDF2C15FEF2516310409F00CF421
:1067C000EEC122242A94312CEAC1411451046104FF
:1067D000710409F4D5C16FEF7FEF7C876B872224AA
:1067E0002A94322CF401878190859C01990F440BE7
:1067F000550B2D873E874F87588B0E9407AC9B0116
:10680000AC01AA24AA94BA2C6501ED84FE840F85FC
:106810001889C301B2010E948248882309F4A7C1E4
:106820006FE87DE089EF9EE00E9422B689EF9EE04E
:106830000E9449B7E12CF12CF40116816BE87DE050
:1068400089EF9EE00E9422B6612F110F770B4AE07C
:1068500050E089EF9EE00E9442B765E87DE089EF55
:106860009EE00E9422B64AE050E06B857C8589EF6D
:106870009EE00E9442B763E87DE089EF9EE00E94BF
:1068800022B64AE050E0B10189EF9EE00E9442B793
:1068900060E87DE089EF9EE00E9422B64AE050E089
:1068A00069857A8589EF9EE00E9442B768E77DE0BE
:1068B00089EF9EE00E9422B64AE050E0B70189EFDE
:1068C0009EE00E9442B789EF9EE00E9449B7F6EF32
:1068D000EF16FFEFFF060CF080C0F401658585819F
:1068E0000E9455AAF401828193810E943C69672B22
:1068F000682B692B51F480E00E946C48AB01BC010D
:10690000F401828193810E94DE68F40114818EEF8C
:10691000810F65858C3020F084ED810F8330C8F4C1
:10692000AA27BB27AE19BF09662351F09D01A1E03C
:10693000BFEF0E9475D629E130E040E050E080C012
:106940002FEF30E00E947DD629E130E040E050E0BA
:106950008AC0F40185819EEF980F9C3020F08C5204
:10696000833008F0D2C081E06827812F0E9455AAA9
:10697000F4018585AA27BB27AE19BF09882359F0E2
:106980002FEF30E00E947DD629E130E040E050E07A
:106990000E9411D612C09D01A1E0BFEF0E9475D6E2
:1069A00029E130E040E050E00E9411D6DA01C9014F
:1069B00081509F4FAF4FBF4F9C012634310544F0AB
:1069C000B9012F3F310531F02CF06FEF70E002C0BC
:1069D00066E470E0F401858195C0FBE0EF16F104F8
:1069E0000CF499C0F401658584810E9455AAF401D4
:1069F000828193810E943C69672B682B692B51F43B
:106A000080E00E946C48AB01BC01F401828193815B
:106A10000E94DE68F40115818EEF810F65858C3050
:106A200020F084ED810F833078F5662399F097018B
:106A3000A1E0BFEF0E9475D623E330E040E050E0D4
:106A40000E9411D6DA01C90181509F4FAF4FBF4F4D
:106A50009C010BC02FEF30E0D7010E947DD623E3CD
:106A600030E040E050E00E9411D62634310544F079
:106A7000B9012F3F310531F02CF06FEF70E002C00B
:106A800066E470E0812F3EC0F40184819EEF980F90
:106A90009C3018F08C528330C0F581E06827812F3C
:106AA0000E9455AAF4018585882369F02FEF30E014
:106AB000D7010E947DD629E130E040E050E00E94FD
:106AC00011D6B90112C09701A1E0BFEF0E9475D69F
:106AD00029E130E040E050E00E9411D6DA01C9011E
:106AE00081509F4FAF4FBF4FBC016F3F710509F001
:106AF0002CF477FF05C060E070E002C06FEF70E03B
:106B0000F40184810E94C0AA50C081E06827812FCF
:106B10000E9455AA4AC067EC75E08CE59EE00E9491
:106B20007B71F401658584810E9455AAF401658515
:106B300085810E9455AA40E050E0BA01F4018281AB
:106B400093810E94DE6860E070E1F40182819381AC
:106B50000E94826960E070E2F401828193810E9468
:106B60008269809100028F5F809300021EC0FFEF58
:106B70002F163F0649F0E984FA84E218F3085CCE48
:106B80002FEF3FEF3C872B87E984FA843FE7E31A36
:106B9000F10822242A94322C4FCE212C312C41147E
:106BA00051046104710439F31DCE80E090E06096D9
:106BB0000FB6F894DEBF0FBECDBFDF91CF911F910E
:106BC0000F91FF90EF90DF90CF90BF90AF909F908C
:106BD0008F907F906F905F904F903F902F9008958F
:106BE0000895FC01838594859C0144E035952795A3
:106BF0004A95E1F756E0959587955A95E1F728175C
:106C0000390719F081E090E0089582E090E008955E
:106C100080E090E008958091BC0A9091BD0A0895AB
:106C20000C940BCB2F923F924F925F926F927F9278
:106C30008F929F92AF92BF92CF92DF92EF92FF928C
:106C40000F931F93CF93DF93CDB7DEB7AF970FB6F8
:106C5000F894DEBF0FBECDBF5C010E8F1F8F28A33F
:106C600039A34AA35BA36CA37DA3CFA61C8A1B8A6E
:106C7000DC0118968D919C91199701979E8B8D8BB5
:106C8000E114F104D1F0CE0145969F938F930297C2
:106C90009F938F938EEC95E09F938F93FF92EF924B
:106CA0000E949DDA0FB6F894DEBF0FBECDBF0197EC
:106CB00021F48B899C899E8B8D8BFE8DF8A70D8985
:106CC0001E896B897C894AE050E089EF9EE00E9432
:106CD00042B761E37EE089EF9EE00E9422B64AE07F
:106CE00050E0B80189EF9EE00E9442B76BE27EE07F
:106CF00089EF9EE00E9422B64AE050E068A589EF45
:106D00009EE00E94B1B689EF9EE00E9449B71986C5
:106D10001A861B861C861D861E861F86188A8B85F2
:106D20008F7080648B871986D50118968D919C9100
:106D300019972D893E89281739071CF001979E8BDA
:106D40008D8B8B899C8997FF02C01C8A1B8ACB88FC
:106D5000DC88F601EE0FFF1FEE0FFF1FFAA7E9A771
:106D6000C601880F991F8C010C0D1D1D1CA70BA7B8
:106D70008D899E898C159D050CF474C118A5113060
:106D800021F0123009F41BC12AC12090BE0A3090B4
:106D9000BF0AD10112968D919C911397C816D906FE
:106DA00008F050C11E968C911E971B96AC901B97B5
:106DB00019960D911C911A9718964C9018971C963D
:106DC000BC91BEA3E82EF12CF101F585FFA38A1139
:106DD00064C02BA53CA5020F131F442009F443C037
:106DE000512C612C712CF801EB0FF11D608170E0CA
:106DF000762F6627072E000C880B990BA3019201B2
:106E00000E94EFD58824922EA32EB42EF801EE0D09
:106E1000FF1D608170E0762F6627072E000C880B1F
:106E2000990BA30192010E94EFD5D90199278827D8
:106E3000882A992AAA2ABB2AF8018FA1E80FF11DF6
:106E4000608170E0762F6627072E000C880B990B67
:106E5000A30192010E94EFD5D501C401822B932B8F
:106E6000A42BB52BA0C0F8019EA1E90FF11D8081D4
:106E7000F801EE0DFF1D2081422F50E060E070E030
:106E8000BA0155274427582BF801AFA1EA0FF11D8D
:106E900080818A019B01082B84C029A53AA5020F95
:106EA000131F8A2D90E09EA78DA7442009F45AC095
:106EB000512C612C712CF801EE0DFF1D608170E0EA
:106EC000762F6627072E000C880B990BA3019201E1
:106ED0000E94EFD5B22EAA2499248824EDA5FEA500
:106EE000E00FF11F608170E0762F6627072E000CFF
:106EF000880B990BA30192010E94EFD5D901992724
:106F00008827882A992AAA2ABB2AF8019FA1E90F73
:106F1000F11D608170E0762F6627072E000C880B2C
:106F2000990BA30192010E94EFD5822A932AA42AE9
:106F3000B52AF801AEA1EA0FF11D608170E0762F4D
:106F40006627072E000C880B990BA30192010E9463
:106F5000EFD5B42FA32F922F882788299929AA2902
:106F6000BB2921C0F801EE0DFF1D8081EDA5FEA516
:106F7000E00FF11F2081422F50E060E070E0BA0185
:106F800055274427782BF801BFA1EB0FF11D808115
:106F9000482BF8012EA1E20FF11D80818A019B018F
:106FA000182BD901C801892B8A2B8B2B09F04AC0D9
:106FB0002FEF3FEF4FEF50E0B601C10141C080918C
:106FC000BE0A9091BF0ADC0112962D913C91139755
:106FD000C216D306B8F520E030E0A90130C0EE2497
:106FE000EA94FE2C0E8D1F8D28A139A14AA15BA128
:106FF0006CA17DA1CE0109960E94AC8629833A83BB
:107000004B835C836D837E838F8398878091BE0AD8
:107010009091BF0AFC0122813381C216D30690F4FD
:107020006F852E85022F10E020E030E0322F212FD7
:10703000102F0027262B6D85A9019801262BB6015C
:107040000E9400A5FFEFCF1ADF0A09A51AA50C5F61
:107050001F4F1AA709A72BA53CA52D5F3F4F3CA7A3
:107060002BA786CE3FA5332309F4CEC00091BE0ADC
:107070001091BF0AD80119968D919C911A97892B6E
:1070800009F4B8C0F801C784D088E188F2880E946A
:10709000A8AB6C157D058E059F0548F40E94A8AB32
:1070A000D8011F966D937D938D939C9352970E9468
:1070B000A8ABF801C784D088E188F288DC01CB0155
:1070C0008C199D09AE09BF098C329140A105B1050B
:1070D000C8F2F894D80114968D919C9115979A8BCB
:1070E000898B1996ED91FC911A977F01BFEFEB1AEE
:1070F000FB0A80818D8FF80190810388F489E02D4F
:10710000D80155968C91992309F430C09081982B21
:107110009C8F9081809589238B8F8B8D888F88E0C1
:107120008F8B5C8D6B8D4D8D3F89288D89899A89D8
:10713000D701508347FD252F3A952083262F39F01C
:10714000441F00C000006083000000C0F2CF38E0A0
:107150004D9160830000019761F7D8015496FC932C
:10716000EE9353974D8F3F8B288F3AC09081982B89
:107170009C8F9081809589238B8F8B8D8A8F88E05F
:10718000898F5C8D6B8D4D8D398D2A8D89899A897A
:10719000D701508347FD252F00C000C0208300C0C9
:1071A00000C000C000C000C060830000262F3A95D8
:1071B00041F0441F000000C000C000C000C000C07B
:1071C000E8CF38E04D9100C0608300C0019709F717
:1071D000D8015496FC93EE9353974D8F398F2A8F95
:1071E0009A8B898B78940E94A8ABF8016787708B83
:1071F000818B928B66E27EE089EF9EE00E9422B650
:1072000089EF9EE00E9449B781E090E0AF960FB60B
:10721000F894DEBF0FBECDBFDF91CF911F910F91CC
:10722000FF90EF90DF90CF90BF90AF909F908F90A6
:107230007F906F905F904F903F902F900895CF93E5
:10724000DF9364ED75E08CE59EE00E947B71C09158
:10725000BE0AD091BF0A4C815D8160E070E08985F3
:107260009A850E94EBD3209771F089859A850E94B8
:107270000BCB8E819F8197FD03C060E00E9484AAA2
:10728000CE010E940BCB1092BD0A1092BC0A81E085
:1072900090E0DF91CF9108952F923F924F925F92AD
:1072A0006F927F928F929F92AF92BF92CF92DF9216
:1072B000EF92FF920F931F93CF93DF93CDB7DEB77B
:1072C00061970FB6F894DEBF0FBECDBF0E9407AC2A
:1072D0009B01AC016091C40A7091C50A8091C60AF5
:1072E0009091C70AAA24AA94BA2C650118E8E12E45
:1072F00013E1F12E00E010E00E948248882309F497
:107300006DC3E0909210F0909310D70112968C917B
:10731000823089F466E67EE089EF9EE00E9422B624
:1073200089EF9EE00E9449B780919210909193104E
:107330000E945378E8C18091C20A9091C30A892BB8
:1073400009F067C083E190E00E9473CA8C018CE36E
:1073500090E8F801928B818BF682E582148210828C
:1073600089E0818381E0828383831093C30A009341
:10737000C20A0E9407AC4B015C01F0E18F0EF7E2FC
:107380009F1EA11CB11CD8011596ED91FC9116977A
:107390008FEF83871486DF0113963B961D92EA17C1
:1073A000FB07E1F7F8011482DD24D394BE01665F88
:1073B0007F4FD80115968D919C9116970E94287940
:1073C000181644F40E9407AC681579058A059B05D8
:1073D00008F4A4C100E010E0E12CF12C2091BA0ADD
:1073E0003091BB0A8091C20A9091C30AE216F3065B
:1073F00074F46091B80A7091B90A600F711F0E940D
:10740000A9C4BFEFEB1AFB0A085F1F4FE7CFFC01CF
:1074100012828091C00A9091C10A2091BA0A3091DB
:10742000BB0A821793070CF46AC00E9407AC1B01C9
:107430002C016CE57EE08CE59EE00E944DB7E0916A
:107440009210F0919310309751F08FEF838714864C
:10745000DF0113963B961D92AE17BF07E1F7E0914F
:10746000B40AF091B50A80E090E02091BA0A309118
:10747000BB0A821793073CF4208131812E7F219330
:1074800031930196F2CF66246394712C809192100F
:1074900090919310009709F482C26091BA0A70919A
:1074A000BB0A23E0660F771F2A95E1F72091B80AFF
:1074B0003091B90A620F731F0E94287918160CF0D8
:1074C0006EC28090BA0A9090BB0AF4E18F169104C4
:1074D0000CF065C20E9407AC9B01AC01AA24AA94DF
:1074E000BA2C650118E8E12E13E1F12E00E010E05E
:1074F000C201B1010E948248811151C294C1009120
:10750000B80A1091B90A9C0143E0220F331F4A9533
:10751000E1F7020F131FF8012081283209F0EEC0B5
:10752000AE014F5F5F4FB8018091C20A9091C30ACC
:107530000E94E778882369F12A8130E0C901982FF9
:107540008827990F990F990F6981F8E06F9FB00113
:1075500011249C01262B372BD8018C918031E1F42A
:10756000688570E08F81FB01E81BF109CF019695DA
:10757000982F8827979587950E9452D66051710958
:10758000207F13E0220F331F1A95E1F7620F731F5C
:1075900004C060E874EE01C0B9016138F4EE7F0701
:1075A0007CF0072E000C880B990B0E94ACD420E0D5
:1075B00030E040E05CE30E940BD59B01AC0104C0CD
:1075C00020E030E04EEF52ECE091B60AF091B70ABD
:1075D000309789F08091C00A9091C10ABC01A3E064
:1075E000660F771FAA95E1F7A091B80AB091B90A82
:1075F0006A0F7B1F19950091C00A1091C10A43E0E0
:10760000000F111F4A95E1F78091B80A9091B90ACD
:10761000080F191FE090C20AF090C30AD8018C919C
:10762000803149F0B801C7010E94FA78D82E88232A
:1076300009F460C002C03CE0D32EF7018581968139
:107640000E945378882309F455C0B801D7011596D4
:107650008D919C9116970E940978F701408164E40E
:10766000858196810E94E777D70112968C918823B5
:1076700009F440C0E7EFED0DE33040F4F0E0EE0F29
:10768000FF1FEB5FFC4F4080518004C09EEE492EEF
:1076900092E0592E0115110539F1F70183818823F4
:1076A00019F18081811120C00E9407AC4B015C015F
:1076B000052C000C66087708AE014F5F5F4FB801DC
:1076C000C7010E9491788981811114C00E9407AC82
:1076D000DC01CB0184199509A609B709881599051C
:1076E000AA05BB0548F306C0B201550C880B990BDF
:1076F0000E94CDAB8091C00A9091C10A01969093EF
:10770000C10A8093C00A0E9407AC6093C40A7093B8
:10771000C50A8093C60A9093C70A60C167E0CE018C
:107720000A960E9496779989891373C064EE75E072
:107730008CE59EE00E945FB7F8018081811138C01E
:10774000858196810E945378BE01665F7F4FD80184
:1077500015968D919C9116970E94097840E064EBF4
:10776000F801858196810E94E777D8011596ED9002
:10777000FC901697C7010E94A377C7010E944D474E
:1077800067E880EE9CE00E94584460E880EE9CE050
:107790000E945844C7010E943F47C7010E94A37737
:1077A000F82EF801858196810E945378F5FE38C045
:1077B000AE014F5F5F4FBE01665F7F4FC8010E9401
:1077C0009178D8011196FC908A85803109F401C125
:1077D000BE01665F7F4FC8010E94FA788F1518F4CA
:1077E000F80181810BC08A85803111F48CE006C0DC
:1077F000BE01665F7F4FC8010E94FA78D8011196DA
:107800008C93119714968C9114978F5F14968C9388
:10781000CDCD66EE75E08CE59EE00E945FB7C6CDEB
:10782000D801DC92C5CFA090B80AB090B90A740113
:1078300083E0EE0CFF1C8A95E1F7EA0CFB1C67E085
:10784000C7010E949677F701978189131FCE00E048
:1078500010E008151905CCF548E050E0B701C50166
:107860000E94A1D928E0A20EB11C892B59F5000F66
:10787000111FE091B40AF091B50AE00FF11F808169
:10788000918181609183808365E57EE089EF9EE050
:107890000E9422B68091BA0A9091BB0AA3E0880F99
:1078A000991FAA95E1F72091B80A3091B90A820F81
:1078B000931F0E942BC56EE47EE089EF9EE00E943C
:1078C0004DB7E4CD0F5F1F4FC4CF8091C20A909196
:1078D000C30A892B09F4DACDE091BA0AF091BB0A08
:1078E000EE0FFF1F8091B40A9091B50AE80FF91FBF
:1078F000718260820091BA0A1091BB0A69E47EE04D
:1079000089EF9EE00E9422B64AE050E0B80189EF7C
:107910009EE00E9442B762E47EE089EF9EE00E9412
:1079200022B68091BA0A9091BB0A63E0880F991F32
:107930006A95E1F72091B80A3091B90A820F931F36
:107940000E942BC589EF9EE00E9449B76091BA0A58
:107950007091BB0AE3E0660F771FEA95E1F780912B
:10796000B80A9091B90A680F791FDB018C918832AF
:1079700061F48091C20A9091C30A0E94A9C48091C7
:107980009210909193100E9460488091BA0A909151
:10799000BB0A01969093BB0A8093BA0A77CD0091F7
:1079A000BA0A1091BB0A63E37EE089EF9EE00E9471
:1079B00022B64AE050E0B80189EF9EE00E9442B74B
:1079C00089EF9EE00E9449B71092C10A1092C00A46
:1079D0009ACEFCE0FF1508F403CF08CF61960FB6EE
:1079E000F894DEBF0FBECDBFDF91CF911F910F91F5
:1079F000FF90EF90DF90CF90BF90AF909F908F90CF
:107A00007F906F905F904F903F902F9008950F93CD
:107A10001F93CF93DF938C010E947712C8010E94BD
:107A200060C168EE75E08CE59EE00E947B718091FC
:107A3000BE0A9091BF0A892B09F586E190E00E9469
:107A400073CAEC01F801238534854285042E000CAD
:107A5000550B608571850E946FA5D093BF0AC093B6
:107A6000BE0A8E819F8197FD07C061E00E9484AAB3
:107A700060E08E810E9455AA81E0898381E090E0D8
:107A80009093BD0A8093BC0ADF91CF911F910F9113
:107A900008958F929F92AF92BF92CF92DF92EF9212
:107AA000FF920F931F93CF93DF9300D000D0CDB7F9
:107AB000DEB78090C80A9090C90A8114910409F435
:107AC000B5C08091DD0A8F5F8093DD0A0E9407AC0C
:107AD0009B01AC016091D00A7091D10A8091D20AC9
:107AE0009091D30AAA24AA94BA2C65011FE0E12E32
:107AF000F12C00E010E00E948248882309F44DC078
:107B0000F4010681178101151105C9F1F80180857D
:107B10008F70863081F563E975E0C8010E94565A7E
:107B20000097D9F0FC0120852F702530B1F4E68054
:107B3000F780E114F104F9F0FA82E982B801CE018C
:107B400001960E94861362E070E0CE0101960E94C9
:107B50003015F701E280F380ECCF1A83098360E0EF
:107B600070E0CE0101960E94861362E070E0CE01C3
:107B700001960E943015F80102811381C4CF0E9442
:107B800007AC6093D00A7093D10A8093D20A909385
:107B9000D30A10920E0F10920F0F0E9407AC9B0198
:107BA000AC016091CC0A7091CD0A8091CE0A90917F
:107BB000CF0AAA24AA94BA2C650118E8E12E13E191
:107BC000F12E00E010E00E948248882351F1E091FC
:107BD000C80AF091C90A0681178101151105B9F08B
:107BE000F80180858F70863071F41A83098360E014
:107BF00070E0CE0101960E94861361E070E0CE0134
:107C000001960E943015F80102811381E6CF0E948F
:107C100007AC6093CC0A7093CD0A8093CE0A909300
:107C2000CF0A8091DD0A81508093DD0A26960FB637
:107C3000F894DEBF0FBECDBFDF91CF911F910F91A2
:107C4000FF90EF90DF90CF90BF90AF909F908F907C
:107C500008952F923F924F925F926F927F929F92E0
:107C6000AF92BF92CF92DF92EF92FF920F931F934A
:107C7000CF93DF93CDB7DEB7CE55D1090FB6F894C9
:107C8000DEBF0FBECDBF8091DD0A8F5F8093DD0A1E
:107C9000E0919610F09197103097B9F00681178116
:107CA000E0909610F0909710E114F10471F0011536
:107CB000110559F0F80180858F708530A9F7C8014A
:107CC0000E949C9F823080F3E6C18091DD0A815042
:107CD0008093DD0A8091941090919510059709F496
:107CE0004CC50E9407AC9B01AC016091D40A709115
:107CF000D50A8091D60A9091D70AAA24AA94BA2CC0
:107D0000650118EEE12E13E0F12E00E010E00E9474
:107D10008248882309F431C510E0AA24A394B12C29
:107D200022242A94322C5FE0452E53E0552E609198
:107D3000CA0A7091CB0A6115710509F41EC51111AB
:107D40001CC5FB0180858F70853009F089C1CE018B
:107D5000C8960E94CE6A21968FAD2197883009F48B
:107D600033C1893009F440C0843009F068C1809182
:107D70002F1090913010892B09F021C160E074E040
:107D8000CE01C8960E94F469892B09F46AC0198251
:107D90001A821B821C821D821E821F8218868B8182
:107DA0008F708B83198241E0BE01685C7F4FCE01EA
:107DB00001960E94EE9965E77EE089EF9EE00E94C1
:107DC00022B660E074E0CE01C8960E948269098103
:107DD0001A812B813C814D815E816F817885CE0136
:107DE000C8960E945C4EEBC080912F10909130108D
:107DF000892B09F0E4C060E074E0CE01C8960E94CF
:107E0000F469892B09F4EFC119821A821B821C8242
:107E10001D821E821F8218868B818F708B83198230
:107E200041E0BE01685C7F4FCE0101960E94EE9951
:107E300067ED7EE089EF9EE00E9422B660E074E08C
:107E4000CE01C8960E94826909811A812B813C81EA
:107E50004D815E816F817885CE01C8960E947F4DED
:107E6000AEC0EAACFBACF70180858F70853009F0BD
:107E70002BC1C7010E949C9FC82ED12CF2E0CF16C7
:107E8000D1040CF421C1B0923010A0922F1060E008
:107E900070E0CE01C8960E9457693C0161E070E035
:107EA000CE01C8960E9457698C01F5E0CF16D10427
:107EB0000CF478C164E0C7010E941B9FFC01E184BF
:107EC000F28426E040E855E260E070E088E99BE05B
:107ED0000E94DEA260922F0D88E99BE090932E0D08
:107EE00080932D0D10923A0E10923C0E10923B0E84
:107EF000F1E0EF16F10409F408C10CF4ECC092E0D3
:107F0000E916F10409F0F3C01093310D0093300D20
:107F1000B092330DA092320D83E00E9427A0982EDC
:107F2000911024C1E090340DF090350DC7010F2C55
:107F3000000CAA0BBB0B89839A83AB83BC8380E1C3
:107F400090E09E838D83E8ADF9ADC080D18067EA73
:107F50007EE089EF9EE00E9422B6B60189EF9EE0A6
:107F60000E945FB760EA7EE089EF9EE00E9422B641
:107F7000BE016F5F7F4F89EF9EE00E94D86B0E9429
:107F800049B7B701CE01C8960E94B373E091CA0AFF
:107F9000F091CB0A62817381CE0101960E94CE6A74
:107FA0008091CA0A9091CB0A892B09F0BFC0CE01FB
:107FB00001960E9418A01092301010922F10CE013E
:107FC000C8960E946051CDC380912F1090913010BF
:107FD000892BA9F760E074E0CE01C8960E94F4698D
:107FE000892B69F319821A821B821C821D821E82D0
:107FF0001F8218868B818F708B83198241E0BE01AE
:10800000685C7F4FCE0101960E94EE996CE27FE0A2
:1080100089EF9EE00E9422B660E074E0CE01C8962F
:108020000E94826909811A812B813C814D815E8188
:108030006F817885CE01C8960E945752C0CFCE017D
:10804000C8960E94605161E070E0CE01C8960E941F
:10805000E572892B09F085C3CE01C8960E9418A04D
:10806000E091CA0AF091CB0A309709F486C3828165
:1080700093819093CB0A8093CA0A892B09F057CE3B
:10808000E0919610F0919710868197819093CB0A9A
:108090008093CA0A72C3B801CE0101960E94CE6ACB
:1080A000CE0101960E949068882331F062E070E072
:1080B000CE0101960E94E572F80102811381CE0182
:1080C00001960E9418A0ECCD64EC7EE089EF9EE062
:1080D0000E9422B674CFEF2811F51093310D009352
:1080E000300DB092330DA092320D81E016CFE3E057
:1080F000EE16F104A1F41093310D0093300DB092FF
:10810000330DA092320D84E008CF1093310D00930F
:10811000300DF092330DE092320D82E0FECE6CEA2B
:108120007EE089EF9EE00E9422B6FACECE01019653
:108130000E949068882309F43ACF8985843009F039
:1081400036CF60E070E0CE0101960E945769681654
:10815000790609F02CCF61E070E0CE0101960E9413
:1081600057690817190709F022CF20C0892D90E020
:10817000A0E0B0E089839A83AB83BC8380E190E088
:108180009E838D836AE87EE089EF9EE00E9422B69E
:10819000BE016F5F7F4F89EF9EE00E94D86B0E9407
:1081A00049B709CF82E0E82EF12C8BCEB701CE0182
:1081B00001960E94B373E091CA0AF091CB0A8281C2
:1081C00093819093CB0A8093CA0A892B09F0EFCE52
:1081D000E0919610F0919710868197819093CB0A49
:1081E0008093CA0AE4CEB0923010A0922F100E9461
:1081F0002ABB3C01892B29F0F3018085807F8660B2
:10820000808720E030E043E050E060E2CE0101965C
:108210000E943849E8ADF9AD608171814FE150E0CD
:10822000CE0101960E94F9D965EF75E0CE01019665
:108230000E94D3D926E040E855E260E070E088E98A
:108240009BE00E94DEA260E070E0CE01C8960E9432
:10825000576980932F0D88E99BE090932E0D8093B2
:108260002D0D10923A0E10923C0E10923B0E84E3AC
:1082700098E09093310D8093300DEAE0F0E0F093B8
:10828000330DE093320D83E00E9427A081110AC1D3
:1082900062E27FE089EF9EE00E9422B624E3E22EB4
:1082A0002DE0F22E00E110E0F701819191917F0124
:1082B000092E000CAA0BBB0B89A39AA3ABA3BCA3EA
:1082C0001EA30DA3BE016F5D7F4F89EF9EE00E944C
:1082D000D86B60E27FE00E9422B6F8E4EF16FDE082
:1082E000FF0611F789EF9EE00E9449B76091380DB3
:1082F0007091390D80E090E00E94ACD420E030E035
:1083000048EC52E40E9405D79B01AC0164EE75E095
:10831000C3010E947473C0903C0DD0903D0DE12CC0
:10832000F12CA70196016BEF75E0C3010E94D99F64
:1083300060913E0D70913F0D80E090E00E94ACD4C2
:1083400020E030E048EC52E40E9405D79B01AC01EC
:1083500066EE75E0C3010E9474736091400D7091E8
:10836000410D80E090E00E94ACD420E030E040E29B
:1083700051E40E9405D79B01AC016DEF75E0C3018C
:108380000E9474732091340D3091350D40E050E01F
:108390006FEF75E0C3010E94D99FCD28CE28CF286A
:1083A00009F49AC0EAADFBAD90859F70953009F055
:1083B00093C061E0CF010E941B9F009709F48CC01D
:1083C000FC0120852F70243009F086C061857285FC
:1083D000CE0181960E94436ACE0181960E949068E8
:1083E000882309F45AC063961CAE1DAE1EAE1FAEA4
:1083F000639767961CAE1DAE1EAE1FAE6797629662
:108400008FAD62978F70806162968FAF62978FEFAA
:1084100064968FAF649765965FAD659766963FAD3E
:10842000669767962FAD679760969FAD6097619648
:108430007FAD619762966FAD629763964FAD63971C
:10844000092F68969FAF689769967FAF69976A967C
:108450006FAF6A976B964FAF6B97482F6C968FAF45
:108460006C976D965FAF6D976E963FAF6E976F96F8
:108470002FAF6F97CC24C394E12CF12C172F262F0C
:108480006B963FAD6B976E966FAD6E976F967FADA7
:108490006F97CE0181960E942F25CE0181960E9472
:1084A00018A01AC090E0A0E0B0E089A39AA3ABA303
:1084B000BCA380E190E09EA38DA36AE07FE089EFFA
:1084C0009EE00E9422B6BE016F5D7F4F89EF9EE065
:1084D0000E94D86B0E9449B78091340D83FF2EC053
:1084E0008EE398E09093310D8093300DB092330D70
:1084F000A092320D83E00E9427A081110BC0209131
:10850000340D3091350D40E050E062E076E0C3017B
:108510000E94D99F1092301010922F10CE01C89651
:108520000E947E511816190624F4CE01C8960E94A6
:108530000E73B0923010A0922F1008C020E030E0EF
:10854000A90162E076E0C3010E94D99F62E370E076
:1085500080E090E00E94CDAB83E190E09093310DFC
:108560008093300DE4E0F0E0F093330DE093320DB2
:1085700083E00E9427A08111A0C060E07FE089EF26
:108580009EE00E9422B694E3E92E9DE0F92E0CE3D2
:108590001DE0F701619171917F014AE050E089EFA0
:1085A0009EE00E9442B76EEF7EE089EF9EE00E945F
:1085B00022B60E151F0569F789EF9EE00E9449B7A4
:1085C0000091340D1091350D01151105D1F0B80150
:1085D000012E000C880B990B0E94ACD42DEE3EE9C5
:1085E0004CE35EE30E940BD522E538EB42E152E416
:1085F0000E9498D69B01AC0164E876E0C3010E941A
:1086000074736091360D7091370D072E000C880B36
:10861000990B0E94ACD42DEE3EE94CE35EE30E9440
:108620000BD522E538EB42E152E40E9498D66B016B
:108630007C019B01AC0169EF75E0C3010E9474737A
:1086400060913A0D70913B0D16161706A4F4072E93
:10865000000C880B990B0E94ACD420E030E040E283
:1086600051E40E9405D79B01AC0166E076E0C301AE
:108670000E94747308C020E030E0A90166E076E053
:10868000C3010E94D99F20E030E040E252E4C701DC
:10869000B6010E94ADD7181644F5012B31F10E94A6
:1086A000DD9D882329F08091DC0A882309F44AC0E3
:1086B000CE01C8960E940E7318C090E0A0E0B0E012
:1086C00089A39AA3ABA3BCA380E190E09EA38DA352
:1086D00068EE7EE089EF9EE00E9422B6BE016F5DEB
:1086E0007F4F89EF9EE00E94D86B80E091E00E946E
:1086F00073CA8C010097B9F01CA21BA21EA21DA276
:1087000038A62FA25AA249A21AA619A69CA78BA7DF
:1087100080E091E098AB8FA71EA61DA6B301CE0105
:1087200081960E941EA80E94DD9D882321F08091E1
:10873000DC0A882381F0C8010E940BCBC3010E9490
:10874000427339CCE8ADF9AD608171818AE096E081
:108750000E949B6EADCFB801CE0101960E949B6E28
:10876000EACF0E9407AC6093D40A7093D50A809335
:10877000D60A9093D70A11E06FCCC25ADF4F0FB6DA
:10878000F894DEBF0FBECDBFDF91CF911F910F9147
:10879000FF90EF90DF90CF90BF90AF909F907F9031
:1087A0006F905F904F903F902F9008954091460BAF
:1087B000262F30E0240F311D21323105DCF42091C9
:1087C0006A0B2430C9F4FC0180E090E0861758F46D
:1087D0003091460B2191DC01AA5DB44FA30FB11D6E
:1087E0002C930196F3CF8091460B680F6093460B54
:1087F00080E0089581E0089582E008950895089545
:10880000E091171080911610E81730F4F0E0E05076
:10881000F54F808190E008958FEF9FEF089590913C
:10882000171080911610981750F4E92FF0E0E050DF
:10883000F54F208130E09F5F9093171002C02FEF1B
:108840003FEFC90108958091161090E02091171014
:10885000821B91090895CF92DF92EF92FF920F93BE
:108860001F93CF93DF937C01CB018A012091FF0AF4
:10887000222389F0EB016B01C40ED51ECC15DD055A
:1088800069F06991D701ED91FC910190F081E02DA3
:10889000C7011995F3CF642F0E94D643C801DF9119
:1088A000CF911F910F91FF90EF90DF90CF9008959F
:1088B000CF93DF931F92CDB7DEB769832091FF0A74
:1088C0002223D1F020911410203240F021E030E03A
:1088D000FC013383228380E090E015C08091151065
:1088E000E82FF0E0E152F54F998190838F5F8093FC
:1088F00015108093141005C061E0CE0101960E940E
:10890000D64381E090E00F90DF91CF910895DC0194
:1089100016968D919C911797009739F0DC01ED9197
:10892000FC910190F081E02D199481E090E0089590
:10893000DC0116968D919C911797009739F0DC0118
:10894000ED91FC910680F781E02D19940895109225
:108950006A0B81E080936C0B10926B0B61E084E1F9
:108960000E9455AA61E085E10E9455AAE9EBF0E07A
:1089700080818E7F808380818D7F808388E4809357
:10898000B80085E48093BC000895CF93DF9391E015
:108990009093250B8823B9F0C091B800D091BA000C
:1089A0008091BC008A7B8093BC0060E084E10E94DF
:1089B00055AA60E085E10E9455AA0E94A744D09381
:1089C000BA00C093B800DF91CF91089585ED8093F0
:1089D000BC008091210B9091220BA091230BB091B0
:1089E000240B0796A11DB11D23E0B695A795979579
:1089F00087952A95D1F72091BC0024FF1CC0409197
:108A0000210B5091220B6091230B7091240B452B6D
:108A1000462B472B81F30097A105B10541F025E3D3
:108A20002A95F1F700000197A109B109E4CF8091DF
:108A3000200B0C94C54410926A0B08951F920F925C
:108A40000FB60F9211240BB60F922F933F934F93B3
:108A50005F936F937F938F939F93AF93BF93EF93A6
:108A6000FF938091B900887F803609F49CC068F537
:108A7000883209F45BC090F4803109F454C038F4B2
:108A8000882309F4F6C0883009F44DC0F6C0883157
:108A900009F44CC0803209F45DC0EFC0803409F4A1
:108AA00068C048F4803309F455C0883309F0E5C044
:108AB0008093690BD8C0803509F44FC0883509F41C
:108AC0005DC0883409F0D9C0D6C0883909F4C7C060
:108AD000A8F4883709F467C038F4883609F463C00D
:108AE000803709F460C0C9C0883809F4B8C080393B
:108AF00009F45FC0803809F0C0C05BC0803B09F456
:108B000086C038F4803A09F466C0883A09F47FC018
:108B1000B4C0803C09F4A7C0883C09F4A4C0883BD9
:108B200009F48AC0AAC080918F0B10C090918E0B5F
:108B300080918D0B981770F5E0918E0B81E08E0F70
:108B400080938E0BF0E0E359F44F80818093BB005B
:108B500085EC86C08093690B8EC0E0918E0B81E01E
:108B60008E0F80938E0B8091BB00F0E0E359F44FA1
:108B7000808390918E0B80918D0B6EC0E0918E0B57
:108B800081E08E0F80938E0B8091BB00F0E0E35963
:108B9000F44F808380916C0B81116DC081E08093D4
:108BA0006B0B84EA61C083E080936A0B1092680BC0
:108BB000CFCF8091680B803208F051C0E091680BF4
:108BC00081E08E0F8093680B8091BB00F0E0E85B42
:108BD000F44F8083BDCF85EC8093BC0010926A0B6C
:108BE0008091680B803230F4E091680BF0E0E85B34
:108BF000F44F10826091680B70E0E0911010F091DA
:108C0000111088E49BE019951092680B36C084E03F
:108C100080936A0B1092470B1092460BE091121052
:108C2000F091131019958091460B811105C081E0D8
:108C30008093460B1092260BE091470B81E08E0F3C
:108C40008093470BF0E0EA5DF44F80818093BB0096
:108C50009091470B8091460B981708F479CF85E8DF
:108C60008093BC000AC085EC8093BC0010926A0B14
:108C700004C01092690B0E94E644FF91EF91BF91EE
:108C8000AF919F918F917F916F915F914F913F91A4
:108C90002F910F900BBE0F900FBE0F901F90189545
:108CA0008F929F92AF92BF92CF92DF92EF92FF92FC
:108CB0000F931F93CF93DF9310911410113208F08C
:108CC000C2C0062FD091DE0A0E94A8AB6B017C01C6
:108CD000C0916A0BCC2311F18091210B9091220B52
:108CE000A091230BB091240B892B8A2B8B2B81F322
:108CF0000E94A8AB8090210B9090220BA090230B98
:108D0000B090240BDC01CB018C199D09AE09BF0981
:108D100088169906AA06BB06D8F681C082E0809321
:108D20006A0B00936C0B8FEF8093690B10928E0B84
:108D300010938D0BAFEDBAE0EDE6FBE080E0181785
:108D400021F09D9191938F5FFACF10928F0B9091AC
:108D50008F0B8D2F880F892B80938F0B80916B0B3E
:108D6000813089F510926B0B0E94A8AB6B017C01DE
:108D700080918F0B8093BB008091210B9091220BEF
:108D8000A091230BB091240B892B8A2B8B2BA9F05C
:108D90000E94A8AB0091210B1091220B2091230B74
:108DA0003091240BDC01CB018C199D09AE09BF0960
:108DB000081719072A073B0790F18091BC0083FD33
:108DC000D7CF85EC01C085EE8093BC000E94A8AB94
:108DD0006B017C0180916A0B823039F58091210B07
:108DE0009091220BA091230BB091240B892B8A2BFD
:108DF0008B2B81F30E94A8AB0091210B1091220BC9
:108E00002091230B3091240BDC01CB018C199D099F
:108E1000AE09BF09081719072A073B07D8F6809142
:108E2000200B0E94C544C5E013C08091690B8F3FA1
:108E300079F08091690B803241F08091690B803329
:108E400031F0C4E005C0C1E003C0C2E001C0C3E02E
:108E500010921510109214101092FF0A8C2FDF91AF
:108E6000CF911F910F91FF90EF90DF90CF90BF9027
:108E7000AF909F908F90089561E00C94504680EEE3
:108E80009CE00C943C4781E08093FF0A6093DE0AEB
:108E900010921510109214100895FC01618180EE5B
:108EA0009CE00C9443471F93CF93DF93EC01162F64
:108EB0000E944D4761EE80EE9CE00E945844612F75
:108EC00080EE9CE00E945844CE01DF91CF911F912B
:108ED0000C943F478F929F92AF92BF92CF92DF92B6
:108EE000EF92FF920F931F93CF93DF93F62ED42F21
:108EF0000E94A8AB4B015C01C0916A0BCC2339F1F5
:108F00008091210B9091220BA091230BB091240B07
:108F1000892B8A2B8B2B81F30E94A8AB0091210B0C
:108F20001091220B2091230B3091240BDC01CB01FB
:108F300088199909AA09BB09081719072A073B07C5
:108F4000D8F68091200B0E94C544C0E090C0D13279
:108F500008F0D0E281E080936A0B80936C0B9FEF66
:108F60009093690B10928E0B9D0F90938D0B8093B5
:108F70008F0B80918F0B6F2D660F682B60938F0B7B
:108F800080916B0B813089F510926B0B0E94A8AB1E
:108F90006B017C0180918F0B8093BB008091210B32
:108FA0009091220BA091230BB091240B892B8A2B3B
:108FB0008B2BA9F00E94A8AB8090210B9090220BE4
:108FC000A090230BB090240BDC01CB018C199D09E0
:108FD000AE09BF0988169906AA06BB0690F18091D2
:108FE000BC0083FDD7CF85EC01C085EE8093BC002B
:108FF0000E94A8AB6B017C0180916A0B813031F536
:109000008091210B9091220BA091230BB091240B06
:10901000892B8A2B8B2B81F30E94A8AB8090210B8C
:109020009090220BA090230BB090240BDC01CB017D
:109030008C199D09AE09BF0988169906AA06BB06B8
:10904000D8F68091200B0E94C54411C080918E0BF0
:109050008D1710F4D0918E0BEDE6FBE0A0E0BBE0A5
:10906000C0E0CD1721F081918D93CF5FFACF1092A0
:109070001710C09316108C2FDF91CF911F910F9175
:10908000FF90EF90DF90CF90BF90AF909F908F9028
:10909000089541E0FC01618180EE9CE00E946A47F6
:1090A00080EE9CE00E940F440895CF93DF93EC0183
:1090B00063EC0E945347CE01DF91CF910C94494855
:1090C000CF93DF93EC010E945548682F6460CE0176
:1090D000DF91CF910C942878CF93C82F0E9407ACD2
:1090E00004C09695879577956795CA95D2F76115CF
:1090F00071058105910521F461E070E080E090E068
:10910000CF9108954F925F926F927F92AF92BF92EC
:10911000CF92DF92EF92FF920F931F93CF93DF9343
:1091200000D01F92CDB7DEB72B013C0129833A83D3
:109130004B835C83A60195016E0D7F1D801F911FDF
:109140000E94EFD529813A814B815C8162177307B8
:109150008407950770F4241535054605570510F466
:1091600021E017C021E0461657066806790688F008
:109170000FC0461657066806790650F421E089812B
:109180009A81AB81BC8184159505A605B70508F0C9
:1091900020E0822F0F900F900F900F90DF91CF91D2
:1091A0001F910F91FF90EF90DF90CF90BF90AF9005
:1091B0007F906F905F904F9008958F929F92AF92A3
:1091C000BF92CF92DF92EF92FF920F931F93CF93B4
:1091D000DF93CDB7DEB72B970FB6F894DEBF0FBE87
:1091E000CDBF8C01CE0101967C016C018AE0882EF6
:1091F000912CA12CB12CC6018E199F094115510546
:109200006105710581F0CB01BA01A50194010E94AD
:10921000EFD5942F852F605DF60161936F01A90151
:10922000692F782FE8CFFC013197EE0DFF1DD80193
:109230009E012150310940814D933197E217F30788
:10924000D1F7F801E80FF91F10822B960FB6F894AA
:10925000DEBF0FBECDBFDF91CF911F910F91FF9069
:10926000EF90DF90CF90BF90AF909F908F90089538
:109270008F929F92AF92BF92CF92DF92EF92FF9226
:109280000F931F93CF93DF938C014A015901E09014
:10929000DA0AF090DB0AC62F660FDD0BE114F10449
:1092A00071F1F70180858F70863049F567E176E0CE
:1092B000C7010E94565A6C01F2E08F16910439F0F2
:1092C00083E08816910451F467E378E002C06CE112
:1092D00076E0C7010E94565A7C0102C0E12CF12CB5
:1092E000C114D10471F0F60180858F70843049F487
:1092F00061857285AE01C8010E9417DA08C0E12CB1
:10930000F12CAE016BE47FE0C8010E94A1CDAE015B
:1093100068EA75E0C8010E94F9D9E114F10441F04E
:10932000F70180858F70843019F4618572850FC0D4
:10933000F2E08F169104A1F083E08816910461F0A9
:109340008A94892899F46091D80A7091D90AAE015B
:10935000C8010E94F9D90AC0AE0165E47FE003C0EC
:10936000AE0162E47FE0C8010E9483CDAE0168EAED
:1093700075E0C8010E94F9D9A114B10429F0AE0129
:10938000B501C8010E94F9D9C801DF91CF911F91A1
:109390000F91FF90EF90DF90CF90BF90AF909F9094
:1093A0008F900895CF92DF92EF92FF920F931F93C9
:1093B000CF93DF936B017C01EA010E9477D78B0189
:1093C0001F936F9383EB99E09F938F93DF93CF93DA
:1093D0000E946EDA0F900F900F900F900F900F90E9
:1093E00020E030E0A901C701B6010E94ADD71816F0
:1093F00024F0F7FAF094F7F8F09409900020E9F7D8
:1094000021978EE28883B80117FF03C0719561959B
:109410007109072E000C880B990B0E94ACD49B019C
:10942000AC01C701B6010E9498D620E030E040E2CE
:1094300051E40E940BD50E9477D7605D69831A8240
:10944000DF91CF911F910F91FF90EF90DF90CF9020
:109450000895CF93DF931F921F92CDB7DEB780910F
:10946000B0119091B111009711F48CEB91E1BE0114
:109470006F5F7F4F681B790B072E000C880B990BD1
:109480000F900F90DF91CF910895EF92FF920F937D
:109490001F93CF93DF93FC01892B81F1A081B181D0
:1094A000109761F18C91882349F1E080F180D70118
:1094B0008C91882359F08D3249F080538A3030F0F6
:1094C000BFEFEB1AFB0AF182E082EFCF8F01C701F9
:1094D0000E9443CDD82FC92F6CE270E0C7010E94D3
:1094E000DED9009721F4F8011182108204C00196A0
:1094F000D8018D939C938D2F9C2F02C080E090E02B
:10950000DF91CF911F910F91FF90EF9008959FE908
:10951000980F963010F4875508959FEB980F96306A
:1095200010F48753089580538A3008F080E008953E
:10953000CF93DF93DA01382FEC018C2F831B861732
:10954000C8F4CE01E991F0E024E0F595E7952A957D
:10955000E1F7E95CFC4F20812C93FC018081E82F2E
:10956000EF70F0E0E95CFC4F808111968C931197CD
:109570001296E3CFFA01E60FF11DE60FF11D1082FE
:10958000DF91CF9108958F929F92AF92BF92CF9229
:10959000DF92EF92FF920F931F93CF93DF93CDB79C
:1095A000DEB7C855D1090FB6F894DEBF0FBECDBFE8
:1095B0006296EFAE62976396FFAE639764960FAFC5
:1095C000649765961FAF659766962FAF6697679607
:1095D0003FAF679768964FAF689769965FAF699797
:1095E000009709F484C1D62E8C01FC0180858295F8
:1095F000807F8595859585958595853019F0863090
:1096000091F175C18091DD0A8F5F8093DD0AF801C9
:10961000A680B780A114B10401F16296EFAC629705
:109620006396FFAC639764960FAD649765961FAD24
:10963000659766962FAD669767963FAD6797689674
:109640004FAD689769965FAD69976D2DC5010E9412
:10965000C34AF501A280B380DDCF8091DD0A81503D
:109660008093DD0A44C163E975E0C8010E94565A3F
:109670000097E1F06296EFAC62976396FFAC639758
:1096800064960FAD649765961FAD659766962FAD8E
:10969000669767963FAD679768964FAD68976996EE
:1096A0005FAD69976D2D0E94C34A2DC167E975E0D2
:1096B000C8010E94565A4C0165E675E0C8010E9437
:1096C000565A5C01DD2021F0F1E0DF1641F03FC089
:1096D00061E276E0C8010E94565A7C011AC06BE232
:1096E00076E0C8010E94565A7C0160E376E0C8012A
:1096F0000E94565A6C01E114F10409F000C161E2C4
:1097000076E0C8010E94565A7C01C114D10409F0C8
:10971000F0C066E276E0C8010E94565A6C01E1147E
:10972000F10441F0F70180858F70843019F4E184F1
:10973000F28402C0E12CF12CC114D10451F0F601E5
:1097400080858F70843029F40185128510C0E12C4A
:10975000F12C00E020E033E040E150E0BE016F5B1F
:109760007F4FCE018F5A9F4F0E9488978C018114A2
:10977000910489F1F4016185728589EF9EE0E1141D
:10978000F10491F00E945FB76CE57FE089EF9EE005
:109790000E9422B6B70189EF9EE00E945FB789EF71
:1097A0009EE00E9449B708C00E945FB767E57FE06E
:1097B00089EF9EE00E9422B6CE018F5A9F4F0E94F1
:1097C0004499A114B10459F4F40180858F70843058
:1097D00009F08BC04EC0A114B10409F486C0F50194
:1097E0006185728589EF9EE00E945FB762E57FE048
:1097F00089EF9EE00E9422B6B80189EF9EE00E94A8
:109800005FB789EF9EE00E9449B70115110561F12C
:10981000F50180858F70843039F56185728540E46B
:1098200050E0CE0101960E9417DA0E94DD9D882348
:10983000D9F08091DC0A811117C06FE270E0CE018F
:1098400001960E94DED9892B51F4F50121853285DC
:1098500043E050E060E4CE0101960E943849B8012F
:10986000CE0101960E94FF9E8114910409F0ACCFB5
:109870003CC0F40161857285CE0101960E94436A65
:10988000CE0101960E949068882359F1E114F104F9
:1098900041F040E050E0B701CE0101960E94D86E41
:1098A00020C0CC24C394E12CF12C62960FAD6297BA
:1098B00063961FAD639764962FAD649765963FAD31
:1098C000659766964FAD669767965FAD67976896A2
:1098D0006FAD689769967FAD6997CE0101960E943A
:1098E0002F25CE0101960E9418A081E00CC080E0D7
:1098F0000AC0892B09F016CFE12CF12C20CF892B3F
:1099000009F010CF06CFC85ADF4F0FB6F894DEBF6C
:109910000FBECDBFDF91CF911F910F91FF90EF90C0
:10992000DF90CF90BF90AF909F908F900895882345
:1099300019F06CE67FE002C061E67FE089EF9EE00F
:109940000C9422B6FF920F931F93CF93DF93EC01F9
:10995000888199810E949C9F082F10E00430110596
:10996000ACF40E942ABBFC01892B41F08085807FEA
:10997000826080871186128613861486BF018881D3
:1099800099810E94BC9F0F5F1F4FE8CF088119810A
:1099900060E0C8010E941B9FDC011996FC90F886CC
:1099A00061E0C8010E941B9F9B838A8362E0C8011B
:1099B0000E941B9F9D838C8364E0C8010E941B9FB3
:1099C0008C019F838E838F2D90E08F30910508F05E
:1099D00080C0FC018827EC53FF4F8F4F0C9466D654
:1099E0008AE090E00E9473CA8C01BE010E94A26BC3
:1099F00080E495E0F801918380833EC088E090E0A8
:109A00000E9473CA8C01BE010E94A26B8FEC94E08D
:109A1000D8018D939C9330C08DE090E00E9473CA72
:109A20008C01BE010E94A26B85EE92E0F801918349
:109A30008083C8010E9460C11FC084E090E00E9442
:109A400073CADC011396DC93CE9312972DEA34E0AF
:109A50002D933C939A8789873CC08EE090E00E94CA
:109A600073CA8C01FC01D383C28385E692E09183A3
:109A70008083C8010E9499901A8709872AC086E0CE
:109A800090E00E9473CAFC01D383C28383EF94E009
:109A900009C086E090E00E9473CAFC01D383C283B0
:109AA0008EE195E0918380830115110571F0D80155
:109AB00018968C9118978F70823029F416960D9114
:109AC0001C91179702C000E010E015830483FA8709
:109AD000E987DF91CF911F910F91FF900895CF9368
:109AE000DF93EC016AEF7FE089EF9EE00E9422B6EF
:109AF00060E074E0CE01DF91CF910C94BC69BF921D
:109B0000CF92DF92EF92FF920F931F93CF93DF9349
:109B1000CDB7DEB728970FB6F894DEBF0FBECDBF26
:109B20007C0109831A832B833C834D835E836F837F
:109B30007887CE0101960E94289F6C01023011F0B7
:109B4000053011F4C12CD12C60E070E0C7010E94F7
:109B50005769B82E192F64E170E189EF9EE00E94E9
:109B600022B64AE050E06B2D712F89EF9EE00E94F3
:109B700042B762E170E189EF9EE00E9422B64AE0BE
:109B800050E0B60189EF9EE00E9442B789EF9EE067
:109B90000E9449B700912F10109130100115110546
:109BA00061F041E0B701CE0101960E949699C7018C
:109BB0000E946F4D00E010E06EC081E090E0909355
:109BC000301080932F1026E040E855E260E070E00E
:109BD00088E99BE00E94DEA2B0922F0D88E99BE00D
:109BE00090932E0D80932D0D10923A0E10923C0EF4
:109BF00010923B0E80ED97E09093B50D8093B40DDD
:109C00001092B70D1092B60DC114D10439F085E051
:109C100090E09093B90D8093B80D04C01092B90DE7
:109C20001092B80D86E00E9427A0B82E64E670E07E
:109C300080E090E00E94CDABB1100AC06CE070E112
:109C400089EF9EE00E9422B689EF9EE00E9449B70C
:109C500082ED97E09093B50D8093B40D1092B70DFF
:109C60001092B60D24E62C9DC0012D9D900D11245F
:109C70009093B90D8093B80D86E00E9427A01092B2
:109C8000301010922F10882321F0C7010E946F4DD1
:109C900002C001E010E0C80128960FB6F894DEBFBC
:109CA0000FBECDBFDF91CF911F910F91FF90EF902D
:109CB000DF90CF90BF9008952F923F924F925F9286
:109CC0006F927F928F929F92AF92BF92CF92DF92CC
:109CD000EF92FF920F931F93CF93DF93CDB7DEB731
:109CE0002E970FB6F894DEBF0FBECDBF5C0109837F
:109CF0001A832B833C834D835E836F837887CE01E9
:109D000001960E94289F4C01023011F0053011F499
:109D1000812C912CF50102811381F80180858F70CF
:109D2000853009F051C0C8010E949C9FE82EF12C9B
:109D3000F2E0EF16F1040CF447C060E0C8010E94A5
:109D40001B9FFC01818592859C878B8761E0C80100
:109D50000E941B9FFC01418452846384748480911F
:109D60002F10909130109E878D8792E0E916F104B4
:109D700009F44CC062E0C8010E941B9FFC01818570
:109D800092859A878987F3E0EF16F10409F442C0BF
:109D900063E0C8010E941B9FFC0121843284F4E02F
:109DA000EF16F104A1F064E0C8010E941B9FFC01C2
:109DB000C184D28421143104D1F08D859E85892BF4
:109DC00051F0C5010E946F4D80E090E02AC022E072
:109DD000C22ED12CEFCF9101D4010E9475D624E67A
:109DE00030E040E050E00E9411D6790105C0ED85D9
:109DF000FE85EF2B31F7740109851A859601A201C2
:109E00006B857C85C5010E94D4850BC0EFEFFFEF09
:109E1000FA87E9878FE3282E312C92E0C92ED12CC6
:109E2000CCCF2E960FB6F894DEBF0FBECDBFDF911C
:109E3000CF911F910F91FF90EF90DF90CF90BF9047
:109E4000AF909F908F907F906F905F904F903F90DA
:109E50002F900895AF92BF92CF92DF92EF92FF9230
:109E60000F93CF93DF93CDB7DEB7CC55D1090FB6A3
:109E7000F894DEBF0FBECDBF6C017B015B01AA244D
:109E800088E0B82273FD0DC00E94294A6639710529
:109E90008105910530F0809194109091951005976F
:109EA00081F4B70166277370C6010E94BC6969E935
:109EB0007FE089EF9EE00E9422B6AA24AA94BA2CE1
:109EC000EDC169961CAE1DAE1EAE1FAE69976D96B4
:109ED0001CAE1DAE1EAE1FAE6D9768968FAD689717
:109EE0008F7068968FAF689766961FAE669741E051
:109EF000B601CE018B5A9F4F0E94EE9960E073E04D
:109F0000C6010E94F469E82AF92A1AAA19AAFE01D0
:109F1000F39682E1DF011D928A95E9F77A96119214
:109F2000119286E0DF011D928A95E9F7F0FE21C0CB
:109F300066968FAD669790E08831910590F4FC01AC
:109F40008827ED52FF4F8F4F0C9466D667EF7FE066
:109F500002C063EF7FE0CE01835B9F4F0E9473CD11
:109F600008C065EE7FE089EF9EE00E9422B6E8948B
:109F7000F0F868968FAD689782958F70813008F4FD
:109F80005EC0833018F0883009F059C00E94DD9D12
:109F9000882309F47FC18091DC0A81117BC120E014
:109FA00030E043E050E060E3CE0101960E94384982
:109FB000D601ED91FC91608171814FE250E0CE01BC
:109FC00001960E94F9D901E020E032E044E150E03E
:109FD000BE016F5C7F4FCE018B5A9F4F0E948897C6
:109FE000F1FE06C066968FAD6697823009F02DC1EE
:109FF000F0FE25C0BE01635B7F4FCE0101960E943B
:10A00000FF9E66ED7FE089EF9EE00E9422B6BE01D2
:10A010006F5F7F4F89EF9EE00E945FB763ED7FE047
:10A0200089EF9EE00E9422B6BE01635B7F4F89EFFD
:10A030009EE00E945FB789EF9EE00E9449B7F1FE63
:10A040008CC020E030E043E050E060E3CE010196B8
:10A050000E943849D601ED91FC91608171814FE2F7
:10A0600050E0CE0101960E94F9D968EA75E0CE0170
:10A0700001960E94D3D968968FAD689782958F70AC
:10A080008450823010F567E1CE018B5A9F4F0E94B9
:10A09000AD9A26962FAF269727963FAF27972896FB
:10A0A0004FAF289729965FAF29972A966FAF2A97C7
:10A0B0002B967FAF2B972C968FAF2C972D969FAF1B
:10A0C0002D9700E020E033E003C000E020E032E024
:10A0D00044E150E0BE016F5C7F4FCE018B5A9F4F31
:10A0E0000E94889740E350E06FEC7FE0CE0101963C
:10A0F0000E9483CD69EC7FE089EF9EE00E9422B64A
:10A10000BE016F5F7F4F89EF9EE00E945FB766ECF4
:10A110007FE089EF9EE00E9422B6BE016F5C7F4F18
:10A1200089EF9EE00E945FB789EF9EE00E9449B7E9
:10A130000E94DD9D882309F4ADC08091DC0A811165
:10A14000A9C0BE016F5C7F4FCE0101960E94FF9EA9
:10A1500060E072E0C6010E948269F0FE97C06696D8
:10A160008FAD66978A3059F028F4813071F08630CF
:10A1700061F016C08B3031F08C3059F011C06CEBAF
:10A180007FE009C067EB7FE006C0F601808585307F
:10A1900039F461EC7FE0CE01835B9F4F0E9473CD69
:10A1A00020E030E043E050E060E3CE0101960E9401
:10A1B0003849D601ED91FC91608171814FE250E008
:10A1C000CE0101960E94F9D968EA75E0CE010196A8
:10A1D0000E94D3D940E350E063EB7FE0CE010196CB
:10A1E0000E9483CD6DEA7FE089EF9EE00E9422B657
:10A1F000BE016F5F7F4F89EF9EE00E945FB76AEA02
:10A200007FE089EF9EE00E9422B6BE01635B7F4F34
:10A2100089EF9EE00E945FB789EF9EE00E9449B7F8
:10A220000E94DD9D8823B1F18091DC0A811132C04A
:10A23000BE01635B7F4FCE0101960E94FF9E60E0EE
:10A2400071E0C6010E94826921C0853009F4D0CE38
:10A25000BE016F5C7F4FCE0101960E94FF9E6FEDA5
:10A260007FE089EF9EE00E9422B6BE016F5F7F4FC4
:10A2700089EF9EE00E945FB76CED7FE089EF9EE082
:10A280000E9422B6BE016F5C7F4FD1CEAA24A39458
:10A29000B12C04C0B701C6010E94BC69C501C45AF3
:10A2A000DF4F0FB6F894DEBF0FBECDBFDF91CF9169
:10A2B0000F91FF90EF90DF90CF90BF90AF900895F7
:10A2C000CF93DF93EC0160E073E00E94F4690097A4
:10A2D00091F020919410309195102630310559F469
:10A2E000BC01CE010E942A4F60E073E0CE01DF91F5
:10A2F000CF910C948269DF91CF9108950F931F93B2
:10A30000CF93DF93CDB7DEB728970FB6F894DEBFB3
:10A310000FBECDBF8C0119821A821B821C821D8246
:10A320001E821F8218868B818F708B831982D801C1
:10A33000ED91FC916081718189EF9EE00E945FB791
:10A34000C8010E94906881110DC060E97FE089EF2B
:10A350009EE00E9422B689EF9EE00E9449B78FEFEF
:10A360009FEF9AC0C8010E94366AF8019085973025
:10A37000D1F08530A1F028F4813041F0823079F0BD
:10A3800012C0863019F08A50833068F46CE67FE0A2
:10A3900089EF9EE00E9422B681E090E07DC080E0DF
:10A3A0000E94974C5CC0D80119968D919C911A9788
:10A3B000009789F0DC01ED91FC910688F789E02D8A
:10A3C000199511E0892B09F410E0812F0E94974C18
:10A3D000812F90E061C040E0B801CE0101960E945B
:10A3E000EE99F8018085873059F028F4833059F1CF
:10A3F000843011F12EC0883031F18930E9F029C064
:10A400000280F381E02D80858F70853059F56AE8F0
:10A410007FE089EF9EE00E9422B640E050E060E0DD
:10A4200070E0F801828193810E94E46A082F10E0B5
:10A430000E94974CC80130C060E0CE0101960E9496
:10A44000D19A8C0111C0CE0101960E94D29B8B0142
:10A450000BC060E87FE089EF9EE00E9422B680E0BA
:10A4600090E01AC000E010E065E77FE089EF9EE031
:10A470000E9422B64AE050E0B80189EF9EE00E94B7
:10A4800042B789EF9EE00E9449B731E020E0012BFE
:10A4900009F430E0832F922F28960FB6F894DEBF90
:10A4A0000FBECDBFDF91CF911F910F9108958F9275
:10A4B0009F92AF92BF92CF92DF92EF92FF920F9353
:10A4C0001F93CF93DF93CDB7DEB76F970FB6F89496
:10A4D000DEBF0FBECDBF7C01088F198F2A8F3B8F47
:10A4E0004C8F5D8F6E8F7F8FCE0148960E94949B1C
:10A4F0004B015C01D7011296ED91FC911397808579
:10A500008F70843009F0C4C0D02E61857285CE0171
:10A5100001960E94436ACE0101960E9490688823AA
:10A5200009F448C08985893009F044C060E070E0D2
:10A53000CE0101960E945769C82E192F60E270E182
:10A5400089EF9EE00E9422B64AE050E06C2D712F08
:10A5500089EF9EE00E9442B76EE170E189EF9EE0D4
:10A560000E9422B6B501A40189EF9EE00E9443A398
:10A5700068E170E189EF9EE00E9422B6602F70E0F2
:10A580004AE050E089EF9EE00E9442B789EF9EE0EA
:10A590000E9449B700912F1010913010011511053C
:10A5A00061F041E0B701CE0148960E949699C7013B
:10A5B0000E946F4D00E010E066C081E090E0909353
:10A5C000301080932F1026E040E855E260E070E004
:10A5D00088E99BE00E94DEA2C0922F0D88E99BE0F3
:10A5E00090932E0D80932D0D10923A0E10923C0EEA
:10A5F00010923B0EB2E0DB1609F452C085E0D8168B
:10A6000009F44EC022E538EB42E152E4C501B40141
:10A610000E9499D620E030E040E251E40E940BD540
:10A620002DEE3EE94CE35EE30E9405D74B015C0151
:10A6300020E030E0A9010E94ADD720E030E040E00A
:10A640005FE387FD28C0C501B4010E9499D60E942E
:10A6500077D783ED97E09093B50D8093B40D10926A
:10A66000B70D1092B60D7093B90D6093B80D86E0DA
:10A670000E9427A01092301010922F10882399F07A
:10A68000C7010E946F4DCE0101960E9418A00EC016
:10A6900000E010E00BC0C501B4010E9498D6D7CFEE
:10A6A00060E070E0D6CF01E010E0EDCFC8016F961A
:10A6B0000FB6F894DEBF0FBECDBFDF91CF911F91D3
:10A6C0000F91FF90EF90DF90CF90BF90AF909F9051
:10A6D0008F9008957F928F929F92AF92BF92CF9268
:10A6E000DF92EF92FF920F931F93CF93DF93CDB73B
:10A6F000DEB7A6970FB6F894DEBF0FBECDBF8C01B4
:10A70000762E942E852E20E2B22ECE0101967C016B
:10A71000FC012B2D11922A95E9F78AEE93E09AA37A
:10A7200089A38FEF8BA38CA38DA38EA3680183E4F1
:10A73000C80ED11C43E450E0BE016F5D7F4FC601DF
:10A740000E943385019609F4B9C081E089838A8328
:10A7500086E0A82EAB821C82F80164817581868117
:10A7600097810E946ED66D837E838F8398878986BA
:10A770009A8680E890E09C878B874CE150E0B70197
:10A78000C6010E948880F7012B2D11922A95E9F7C6
:10A79000480188E0880E911CF401D70101900D92C8
:10A7A000AA94E1F740E150E0B701C6010E94888019
:10A7B000F7011192BA94E9F796E0A92EB12C40E284
:10A7C00050E0B701C6010E948880F1E0AF1AB108DD
:10A7D000B1F783E6898392E89A8393E59B838C8320
:10A7E00085E38D8381E08E837F829DE3988797E068
:10A7F00099878A8786E0F401DE011B9601900D920D
:10A800008A95E1F78CE0898B8A8B65E376E0CE014F
:10A8100043960E94F2D9F8016385CE0149960E94C1
:10A8200001B3F8016485CE014B960E9401B3F80193
:10A830006585CE014D960E9401B34EE150E0B7010F
:10A84000C6010E948880F3E07F121EC082E38983E4
:10A8500084E08A83F80196859B8397859C83908901
:10A860009D8391899E8396E39F838887828D8987C4
:10A87000838D8A87848D8B87858D8C874CE050E013
:10A88000B701C6010E94888087E3898386E08A83B6
:10A8900091E09B8393E09C838D838FE08E838AE39A
:10A8A0008F838BE388878FEF898749E050E0B7017A
:10A8B000C6010E948880C6010E946084A6960FB6D9
:10A8C000F894DEBF0FBECDBFDF91CF911F910F91E6
:10A8D000FF90EF90DF90CF90BF90AF909F908F90C0
:10A8E0007F9008952F923F924F925F926F927F9246
:10A8F0008F929F92AF92BF92CF92DF92EF92FF9290
:10A900000F931F93CF93DF9300D000D0CDB7DEB766
:10A910008C010E94DFCB2FEC37E040E050E00E943A
:10A9200011D6DC01CB010196A11DB11DF801848374
:10A930009583A683B78380839183A283B3835801D1
:10A94000F3E4AF0EB11CC5010E94278264E470E0FD
:10A95000C5010E943384882309F436C10E9407ACE4
:10A960002B013C01812C912CC8018E5B9F4F9E8353
:10A970008D8348EEC42E43E0D42EE12CF12C52E01E
:10A98000252EAD81BE818C91833009F404C18111E3
:10A9900020C0F80184819581A681B7810196A11D0F
:10A9A000B11D84839583A683B7830E9407AC641985
:10A9B000750986099709A70196010E94EFD5A9019B
:10A9C00061E0C8010E946A5381E0AD81BE818C9331
:10A9D000CAC08430F9F4F80184819581A681B781D9
:10A9E0000196A11DB11D84839583A683B7830E9420
:10A9F00007AC6419750986099709A70196010E9499
:10AA0000EFD5A90163E0C8010E946A53AD81BE8100
:10AA10002C92A9C0813059F5F80142AD53AD64AD17
:10AA200075AD9E012F5F3F4FC8010E9416B3382EAF
:10AA3000F2E08F1392C089819A81AB81BC81F801C9
:10AA400084839583A683B7830E9407AC6419750934
:10AA500086099709A70196010E94EFD5A90163E035
:10AA6000C8010E946A53AD81BE813C927CC0823095
:10AA700009F079C0F80142AD53AD64AD75AD9E01EA
:10AA80002F5F3F4FC8010E9416B3382EF5E08F1399
:10AA90005DC0E3E0AD81BE81EC93F80182A193A19A
:10AAA000A4A1B5A1892B8A2B8B2B41F484E893E0D8
:10AAB000A0E0B0E082A393A3A4A3B5A3F80186A16C
:10AAC00097A1A0A5B1A5892B8A2B8B2B61F482A11C
:10AAD00093A1A4A1B5A1B695A7959795879586A3AF
:10AAE00097A3A0A7B1A7F80182A593A5A4A5B5A592
:10AAF000892B8A2B8B2BA9F482A193A1A4A1B5A1A8
:10AB0000AC01BD0123E076956795579547952A9549
:10AB1000D1F7841B950BA60BB70B82A793A7A4A70D
:10AB2000B5A7F80186A197A1A0A5B1A586A797A76B
:10AB3000A0ABB1AB82A593A5A4A5B5A582AB93AB01
:10AB4000A4ABB5AB88248394912C0DC0F6E08F1391
:10AB500004C0AD81BE811C9206C0BFEF3B1203C092
:10AB6000ED81FE811082F1E08F16910409F409CF86
:10AB70000E9407ACDC01CB0184199509A609B7092D
:10AB8000F80126A937A940AD51AD281739074A0762
:10AB90005B0708F0F6CEC5010E942782F801848188
:10ABA0009581A681B7810196A11DB11D84839583EE
:10ABB000A683B7830E9407ACF801FE966083718379
:10ABC00082839383C40102C080E090E026960FB692
:10ABD000F894DEBF0FBECDBFDF91CF911F910F91D3
:10ABE000FF90EF90DF90CF90BF90AF909F908F90AD
:10ABF0007F906F905F904F903F902F9008950F93AC
:10AC00001F93CF93DF93EC0100910C0D10910D0D6C
:10AC1000B8010E94B4CD209709F440C009960817E6
:10AC20001907E0F10E94DD9D8823C1F18091120D8A
:10AC30009091130D019611F481E090E09093130D23
:10AC40008093120DE0910A0DF0910B0D8091130D80
:10AC50008583E0910A0DF0910B0D8091120D868392
:10AC600060910A0D70910B0D47E050E0CE010E94FB
:10AC7000149EE0910A0DF0910B0DE80FF91F108260
:10AC8000AC014450510960910A0D70910B0D82E89E
:10AC9000DF91CF911F910F910C94349E80E0DF9152
:10ACA000CF911F910F9108951F93CF93DF931F9220
:10ACB0001F92CDB7DEB76CE271E080E090E00E94B9
:10ACC000CDAB1FB7F8948091960B811127C0E5E0BA
:10ACD000F1E18491EFEBF0E19491E82FF0E0EE0FD9
:10ACE000FF1FE059FF4EA591B491EC91E92321F4A7
:10ACF00061E085E30E9455AA61E085E30E9484AA91
:10AD00008CB580618CBD8CB580648CBD61E084E3C2
:10AD10000E9484AA61E083E30E9484AA8091960B3A
:10AD20008F5F8093960B1FBF809104018860809392
:10AD300004018091040184608093040180910501E5
:10AD4000847080930501CE0101960E9488C5898197
:10AD50009A810E942C7567E080E090E00E9481BC9F
:10AD600065E58BE190E00E9481BC65E58AE190E0B9
:10AD70000E9481BC0E942B7580E090E490939F110B
:10AD800080939E1180E090E69093A7118093A61186
:10AD900080E098E49093A1118093A01180E098E660
:10ADA0009093A9118093A81180E090E59093A3114E
:10ADB0008093A21180E090E79093AB118093AA1149
:10ADC00080E098E59093A5118093A41180E098E726
:10ADD0009093AD118093AC110F900F90DF91CF91B4
:10ADE0001F910895AF92BF92CF92DF92EF92FF92A0
:10ADF0000F931F93CF93DF931F921F92CDB7DEB7B0
:10AE00005C018B016A0179010E945456CE010196C2
:10AE10000E9488C589819A810E942C7546E050E085
:10AE200060E97BE089E090E00E9452BCC501029697
:10AE30000E941675C60102960E942475C7010296EB
:10AE40000E941D750E942B75F80182819381A48157
:10AE5000B5818093DA0C9093DB0CA093DC0CB0935B
:10AE6000DD0C0F900F90DF91CF911F910F91FF900C
:10AE7000EF90DF90CF90BF90AF900895CF92DF9288
:10AE8000EF92FF92CF93DF93CDB7DEB768970FB6FF
:10AE9000F894DEBF0FBECDBFFA012AEE33E03A834D
:10AEA00029835FEF5B835C835D831E8238872F83FA
:10AEB000C280D380E480F580C986DA86EB86FC8682
:10AEC0003E872D87FB0142815381648175814F87C5
:10AED000588B698B7A8B3C8B2B8BFC018281938105
:10AEE000A481B5818D8B9E8BAF8BB88F9E012F5F18
:10AEF0003F4FAE01495F5F4FBE01635F7F4FCE01A1
:10AF000043960E94F25668960FB6F894DEBF0FBEC5
:10AF1000CDBFDF91CF91FF90EF90DF90CF9008955C
:10AF20000F931F93CF93DF93CDB7DEB768970FB61C
:10AF3000F894DEBF0FBECDBFFB01DC0112964D9130
:10AF40005D916D917C9115974D8B5E8B6F8B788F9A
:10AF50008AEE93E09A83898321E0288F0D891E89E8
:10AF60002F89388D0B831C832D833E8398878F8395
:10AF7000028113812481358109871A872B873C87B9
:10AF80009E878D874F87588B698B7A8BAE014F5F79
:10AF90005F4FBE01695F7F4FCE010D960E943E5705
:10AFA00068960FB6F894DEBF0FBECDBFDF91CF918C
:10AFB0001F910F910895CF93DF93CDB7DEB76297BE
:10AFC0000FB6F894DEBF0FBECDBFFC018281938126
:10AFD000A481B5818F87988BA98BBA8B2AEE33E039
:10AFE0003A83298341E04A8B4F85588969897A8958
:10AFF0004B835C836D837E8338872F8389879A8711
:10B00000AB87BC87BE016F5F7F4FCE0107960E9462
:10B01000905762960FB6F894DEBF0FBECDBFDF919A
:10B02000CF910895CF92DF92EF92FF920F931F93EB
:10B03000CF93DF936C01EB017B0182E0E80EF11C02
:10B0400000E010E0C601800F911F0E94C9D5F701F2
:10B0500081937F010F5F1F4F0430110599F78A819B
:10B06000882361F08F3F61F48B818F3F49F48C819D
:10B070008F3F31F481E09D819F3F19F480E001C052
:10B0800081E090E0DF91CF911F910F91FF90EF90C1
:10B09000DF90CF900895EF92FF920F931F93CF937D
:10B0A000DF937C018B010E5F1F4FC0E0D0E0F80101
:10B0B00061918F01C7018C0F9D1F0E94D1D52196F0
:10B0C000C430D105A1F7DF91CF911F910F91FF906F
:10B0D000EF900895FC01DC018D918111FDCF40E0DE
:10B0E00050E020E030E08AE09191992301F1243092
:10B0F00031055CF59E3271F44F3F510509F02CF596
:10B10000DB01A20FB31F12964C932F5F3F4F40E01D
:10B1100050E0EACF849FD001859FB00D1124492FC4
:10B12000990F550B405351094A0F5B1FDDCF4F3F1D
:10B13000510509F054F4243031053CF4FB01E20FD1
:10B14000F31F428381E090E0089580E090E008954D
:10B150004F925F926F927F928F929F92AF92BF9227
:10B16000CF92DF92EF92FF920F931F93CF93DF93D3
:10B17000CDB7DEB768970FB6F894DEBF0FBECDBF70
:10B180006C018A015901DC0114968D919C911597EF
:10B19000DC011F968D919C915097DC011696ED90E5
:10B1A000FC9017972B01770F66087708E114F104DC
:10B1B00009F463C1B2E0AB16B10439F083E0A8161C
:10B1C000B10449F460E476E002C06CE376E0C701C4
:10B1D0000E94565AFC01309709F449C18185928535
:10B1E000A385B48584159505A605B70509F03FC16B
:10B1F00063E476E0C7010E94565A5C016AE675E096
:10B20000C7010E94565AD6011296ED91FC911397F0
:10B2100062E0828193810E941B9F6C01003448F49C
:10B22000F801FF27EE0FFF1FE35DF24F0781108546
:10B2300002C00FEF1FEF198A1A8A1B8A1C8A1D8A07
:10B240001E8A1F8A188E8B898F708B8B198AA11486
:10B25000B10409F43DC0F50180858F708430C1F5DB
:10B260008184928499E2A92E90E1B92E612C712CEF
:10B2700081149104D1F0B501C4010E946ACD892BDB
:10B2800051F485E0869DF001879DF00D1124E35D6A
:10B29000FF4E64910CC0FFEF6F1A7F0A85E0A80E85
:10B2A000B11CA9E06A16710419F761E070E0B62ECE
:10B2B000862F660F990BAA0BBB0BFC013197E93067
:10B2C000F10590F58827E551FF4F8F4F0C9466D616
:10B2D0008B898F70806A8B8B20E030E00D8B1E8B0A
:10B2E0002F8B388FBB24B3941FC08B898F70806ADB
:10B2F00014C08B898F70806B10C08B898F70806BAE
:10B300008B8B11270BC08B898F70806B8B8B102FD1
:10B31000002704C08B898F7080668B8B20E030E023
:10B320000D8B1E8B2F8B388FF7018080918000E072
:10B3300020E033E040E150E0BE016F5F7F4FCE017F
:10B3400041960E9488978C0168E670E189EF9EE043
:10B350000E9422B6B80189EF9EE00E945FB761E6C5
:10B3600070E189EF9EE00E9422B66B2DBB0C770B3B
:10B370004AE050E089EF9EE00E9442B76FE570E13D
:10B3800089EF9EE00E9422B6B40189EF9EE00E9400
:10B390005FB789EF9EE00E9449B7C114D10409F458
:10B3A00063C0D60118968C918F70863009F05CC00E
:10B3B000F701E080F180B701C6010E94565A6C0186
:10B3C000009709F451C060E675E00E94565A8C015E
:10B3D0000097E9F0DC0119968D909D90AD90BC909E
:10B3E0001C976989662321F070E080E090E004C03A
:10B3F000CE0141960E94D29B86169706A806B906F2
:10B4000099F1F801618772878387948721C066E587
:10B4100070E189EF9EE00E9422B6B70189EF9EE0BD
:10B420000E945FB789EF9EE00E9449B729892223D5
:10B4300021F030E040E050E006C0CE0141960E948D
:10B44000D29B9B01AC0160E675E0C6010E94D99FCA
:10B45000E988FA880B891C892D893E894F89588D86
:10B460006FEFC6010E94C34A81E090E008C0D70197
:10B470001296ED90FC90139799CE80E090E068963C
:10B480000FB6F894DEBF0FBECDBFDF91CF911F91F5
:10B490000F91FF90EF90DF90CF90BF90AF909F9073
:10B4A0008F907F906F905F904F9008950F931F93B0
:10B4B000CF93DF938B01FC01C681D781209759F090
:10B4C000B801888199810E94C0D9892B21F00A8016
:10B4D000DB81C02DF3CFCE01DF91CF911F910F9172
:10B4E00008950C94A27D64EC72E18CE49EE00E94CD
:10B4F00022B6E0E0F0E01994BF92CF92DF92EF9293
:10B50000FF920F931F93CF93DF93CDB7DEB7A8972A
:10B510000FB6F894DEBF0FBECDBF6B01122FB32E56
:10B520007A0194E0E2EFF3E0DE01119601900D92D2
:10B530009A95E1F7FE0135968CE1DF011D928A951F
:10B54000E9F7AE014F5F5F4F68E0C6010E94984A7D
:10B550001A8A8091201090912110892B09F46BC0D8
:10B5600089EF9EE00E9449B76AE171E189EF9EE0B0
:10B570000E9422B6412F5B2DB70189EF9EE00E9409
:10B5800043A368E171E189EF9EE00E9422B6BE010B
:10B590006F5F7F4F89EF9EE00E945FB766E171E1C8
:10B5A00089EF9EE00E9422B689EF9EE00E9449B793
:10B5B000BE016F5F7F4F80919810909199100E940B
:10B5C000565A6C0120E030E04EEF52EC612F7B2D9B
:10B5D000C7010E94A5D4882371F120E030E04AEA37
:10B5E00052E4612F7B2DC7010E94A5D4882319F155
:10B5F00020E030E0A901612F7B2DC7010E94A5D476
:10B600008823C9F019A21AA21BA21CA20BA10F70B9
:10B610000067212F812F9B2DD7018DA39EA3AFA360
:10B62000B8A7E9A0FAA01CA13EA14FA158A56FEFB1
:10B63000C6010E94C34AA8960FB6F894DEBF0FBE9B
:10B64000CDBFDF91CF911F910F91FF90EF90DF90D1
:10B65000CF90BF900895CF93C1E068EE73E080E093
:10B6600090E00E94CDAB4AE050E06C2F8CE49EE06D
:10B670000E94B1B6CF5FC43181F7CF9108950F9387
:10B680001F93CF93DF93CDB7DEB728970FB6F8940B
:10B69000DEBF0FBECDBF0E94A27C6DE171E18CE4E4
:10B6A0009EE00E9422B6CE0101960E94D0B1CE014A
:10B6B00001960E947AB10AEE13E01A8309831B8275
:10B6C0001C821D821E82CE0107960E9488C58F8132
:10B6D00098850E942C7544E050E0BE016D5F7F4F5D
:10B6E00081E090E00E9422BC0E942B75CE01019661
:10B6F0000E947AB11A8309831B821C821D821E82DA
:10B70000CE0107960E9488C58F8198850E942C756E
:10B7100044E050E0BE016D5F7F4F85E090E00E9405
:10B7200022BC0E942B75CE0101960E947AB163E47F
:10B7300071E18CE49EE00E9422B628960FB6F89440
:10B74000DEBF0FBECDBFDF91CF911F910F91089546
:10B750005F926F927F928F929F92AF92BF92CF92A1
:10B76000DF92EF92FF920F931F93CF93DF93CDB7AA
:10B77000DEB76D970FB6F894DEBF0FBECDBF009158
:10B780002010109121100115110509F43DC580917B
:10B79000DD0A8F5F8093DD0A68E476E0C8010E94CD
:10B7A000565A90939710809396106EE476E0C801F5
:10B7B0000E94565A9093DB0A8093DA0A6DE576E090
:10B7C000C8010E94565A9093C90A8093C80A65E539
:10B7D00076E0C8010E94565A9093CE0F8093CD0F09
:10B7E0006AE576E0C8010E94565A9093CC0F809388
:10B7F000CB0F009709F4A3C00E949C9F082F10E074
:10B800000115110509F49BC0000F111F000F111F36
:10B810008091C80F9091C90F892B09F07FC0C80192
:10B820000E9473CA9093C90F8093C80F109244105E
:10B83000109243101092D00F1092CF0F109242101E
:10B8400010924610109245107801013082E01807DE
:10B850001CF0E12CA2E0FA2EC70101960E9473CAE7
:10B86000909348108093471090934110809340101C
:10B870008E0D9F1D90933B1080933A100E9407AC51
:10B8800060933C1070933D1080933E1090933F1056
:10B8900080E090E0E0914710F0914810E80FF91F28
:10B8A00010820196E816F906ACF782E090E09093DA
:10B8B00044108093431080E98093C9001092C8001F
:10B8C0001092CD0083E08093CC008EE08093CA007C
:10B8D000F0922F02E0922E022091471030914810F2
:10B8E00080912E0290912F02820F931F90933B1014
:10B8F00080933A10232B09F45AC36DEE72E18CE564
:10B900009EE00E9422B66AE070E0C8010E94AA9FF1
:10B9100083E091E1909339108093381061E674E1EF
:10B920008CE49EE00E9422B64AE050E0B8018CE42C
:10B930009EE00E9442B78CE49EE00E9449B760E618
:10B9400076E080912010909121100E94565A8C012F
:10B95000009709F442C00E949C9F81112FC33DC0F3
:10B960000E94294A4B015C0169EF72E189EF9EE078
:10B970000E9422B62AE030E0B501A40189EF9EE0E2
:10B980000E94A4B689EF9EE00E9449B765E474E185
:10B990008CE49EE00E9422B64AE050E0B6018CE4BE
:10B9A0009EE00E9442B78CE49EE00E9449B70E944C
:10B9B000294A6B017C016FE374E189EF9EE00E94EC
:10B9C00022B62AE030E0B701A60189EF9EE00E948E
:10B9D000A4B689EF9EE00E9449B700912010109113
:10B9E000211064E676E0C8010E94565A90932E100A
:10B9F00080932D1061EE76E0C8010E94565A909314
:10BA0000991080939810009709F4B3C120919A106F
:10BA10002111AFC1DC011696ED90FC901797809133
:10BA2000921090919310892B09F0DDC06DE973E1BC
:10BA300089EF9EE00E9422B689EF9EE00E9449B7FE
:10BA40000E94294A4B015C0167E973E189EF9EE09E
:10BA50000E9422B62AE030E0B501A40189EF9EE001
:10BA60000E94A4B689EF9EE00E9449B781E190E070
:10BA70000E9473CA8C0188E1F801818312821082CE
:10BA8000108A17860E94CE72109393100093921022
:10BA9000012B39F465E873E184E59EE00E9422B64B
:10BAA0005AC080EA90E00E9473CA9093B90A8093CA
:10BAB000B80A0E94294A4B015C0169E773E189EFEA
:10BAC0009EE00E9422B62AE030E0B501A40189EF91
:10BAD0009EE00E94A4B689EF9EE00E9449B788E2EA
:10BAE00090E00E9473CA9093B50A8093B40A0E94B2
:10BAF000294A4B015C016CE673E189EF9EE00E94EC
:10BB000022B62AE030E0B501A40189EF9EE00E9450
:10BB1000A4B689EF9EE00E9449B78091B80A90913F
:10BB2000B90A892B31F08091B40A9091B50A892B1A
:10BB3000B9F40E94294A4B015C0164E573E184E594
:10BB40009EE00E9422B62AE030E0B501A40184E51F
:10BB50009EE00E94A4B684E59EE00E9449B74CC0D6
:10BB60008CE79AE59093B70A8093B60A0E94CE724A
:10BB700080919210909193100E944D4780EE9CE02E
:10BB80000E943C47811132C061E473E189EF9EE07D
:10BB90000E944DB70091921010919310C8010E941D
:10BBA0004D4740E060EFC8010E94E777C8010E945E
:10BBB0003F47E0919210F091931081E0808361E221
:10BBC00073E189EF9EE00E944DB7809192109091B1
:10BBD00093100E945378882331F065E173E189EF77
:10BBE0009EE00E944DB781E090E008C067E073E1FD
:10BBF00089EF9EE00E944DB780E090E0282F2170F1
:10BC000020939A10892B31F06FE274E18CE49EE06E
:10BC10000E9422B61092BB0A1092BA0ACC24C39496
:10BC2000D12CE114F10409F4A4C080919A10882366
:10BC300009F49FC0D70118968C9118978F708630A1
:10BC400009F093C00D911C91FE0131965F014801EE
:10BC5000F0E18F0E911C3501D8018C910E94874A2A
:10BC6000582EF80181810E94874A5294E0EF5E22AB
:10BC70008529D5018D935D010E5F1F4F80169106BA
:10BC800059F78091BA0A9091BB0A843191050CF062
:10BC90006CC0880F991FE091B40AF091B50AE80FC3
:10BCA000F91FD182C082A091BA0AB091BB0A53E0B9
:10BCB000AA0FBB1F5A95E1F78091B80A9091B90A73
:10BCC000A80FB91F88E0F30101900D928A95E1F762
:10BCD0000091BA0A1091BB0A65EC73E189EF9EE00E
:10BCE0000E9422B64AE050E0B80189EF9EE00E942F
:10BCF00042B76EEB73E189EF9EE00E9422B680911D
:10BD0000BA0A9091BB0A63E0880F991F6A95E1F720
:10BD10002091B80A3091B90A820F931F0E942BC557
:10BD200089EF9EE00E9449B7E091BA0AF091BB0A00
:10BD300073E0EE0FFF1F7A95E1F78091B80A9091BA
:10BD4000B90AE80FF91F8081883231F4809192108E
:10BD5000909193100E9460488091BA0A9091BB0A1A
:10BD600001969093BB0A8093BA0AF701E280F380B0
:10BD700058CF1092CB0A1092CA0AE0919610F09117
:10BD800097103097F9F0C680D780009196101091E7
:10BD900097100115110579F0C114D10461F0D60195
:10BDA00018968C918F708530A1F7C6010E949C9FD8
:10BDB000823078F335C1F801868197819093CB0A60
:10BDC0008093CA0A89EF9EE00E9449B7E091C80AB1
:10BDD000F091C90A309709F46BC08091DD0A8F5F3A
:10BDE0008093DD0A068117815E01F8E1AF0EB11C78
:10BDF00096E1692E94E0792E2EE2822E24E0922E96
:10BE00000115110509F44FC0D80118968C918F7057
:10BE1000863009F044C0198F088F60E070E0C501DA
:10BE20000E9486138C8D9D8D892BC9F180912010E5
:10BE300090912110892B99F1E88CF98CF70180857C
:10BE40008F708630B1F463E975E0C7010E94565ADD
:10BE5000009709F036C1FA82E98260E070E0CE0115
:10BE600001960E94861362E070E0CE0101960E9466
:10BE70003015EC8DFD8D10821182128213828A8D15
:10BE8000843008F03DC1823008F050C162E08B8DF3
:10BE90000E9484AAEC8DFD8D8181807F8183F801D1
:10BEA00002811381ADCF8091DD0A81508093DD0A3C
:10BEB0006AE074E18CE49EE00E9422B662E074E1E4
:10BEC0008CE49EE00E9422B681E020919610309191
:10BED0009710232B09F480E00E94977D69EF73E1AE
:10BEE0008CE49EE00E9422B681E02091C80A309145
:10BEF000C90A232B09F480E00E94977D6AEE73E162
:10BF00008CE49EE00E9422B66FED73E18CE49EE02B
:10BF10000E9422B681E020912D1030912E10232B0B
:10BF200009F480E00E94977D68ED73E18CE49EE067
:10BF30000E9422B681E02091CD0F3091CE0F232BAD
:10BF400009F480E00E94977D6FEC73E18CE49EE041
:10BF50000E9422B681E02091981030919910232BF5
:10BF600009F480E00E94977D8CE49EE00E9449B72E
:10BF70000E94294A6B017C016AEC73E18CE49EE02B
:10BF80000E9422B62AE030E0B701A6018CE49EE0D0
:10BF90000E94A4B68CE49EE00E9449B781E08093A1
:10BFA000CA0F8091DD0A81508093DD0A2DC166EDB4
:10BFB00072E18CE59EE00E944DB7AACC6FEF680F4E
:10BFC000C8010E941B9FDC011996CD90DD90ED9079
:10BFD000FC901C9790911810992359F08091700053
:10BFE0008E7F809370001092181010922A02109287
:10BFF000290282E18093280291110E940C77560158
:10C00000C6010E94347701E010E0A016B1060CF4DE
:10C01000A7CC60E0C8010E946A770F5F1F4FF5CF81
:10C02000B601CE0101960E94CE6ACE0101960E9411
:10C0300090688823E1F18A859B850097E1F0DC0117
:10C04000ED91FC910484F585E02D1995892B49F03B
:10C050008A859B85DC01ED91FC910284F385E02DBE
:10C0600019958A859B85DC01ED91FC910680F7810D
:10C07000E02D19951CC060E070E0CE0101960E9491
:10C0800057698C0197FFBDC0119501951109AA242C
:10C09000A394B12CCE0101960E94366AE82EF12CB1
:10C0A0008985853009F452C0863009F474C0D60100
:10C0B0001296CD90DC901397CE0101960E9418A0A5
:10C0C00064CEFC0120852F70253009F0C4CEC680D7
:10C0D000D780C114D10409F4CCCEDA82C982B70169
:10C0E000CE0101960E948613ED81FE81108211829D
:10C0F00012821382D6011296CD90DC901397E9CF6D
:10C100008630D9F060F4853009F0C9CEBC82AB82AC
:10C110009A828982CE0101960E940B94C0CE80340F
:10C1200039F0823409F0BBCE60E003C060E0AFCEEE
:10C1300062E08B8D0E9484AAB2CEBC82AB827A82EE
:10C140006982CE0101960E942293A9CEEF2829F49C
:10C1500062E0CE0101960E940B6A61E0802F0E948E
:10C1600084AA60E0802F0E9455AA67E274E189EFFB
:10C170009EE00E9422B64AE050E0B80189EF9EE0BE
:10C180000E9442B762E274E189EF9EE00E9422B60B
:10C1900060E274E131C0902E61E0802F0E9484AA99
:10C1A00061E0AB2821F0EA94EF2829F403C0EA9477
:10C1B000EF2809F060E0E62EF12C892D0E9455AAA7
:10C1C0006BE174E189EF9EE00E9422B64AE050E004
:10C1D000B80189EF9EE00E9442B769E174E189EFFE
:10C1E0009EE00E9422B64AE050E0B70189EF9EE04F
:10C1F0000E9442B767E174E189EF9EE00E9422B697
:10C2000056CFA12CB12C46CF6D960FB6F894DEBF59
:10C210000FBECDBFDF91CF911F910F91FF90EF9097
:10C22000DF90CF90BF90AF909F908F907F906F9056
:10C230005F9008958091E70F9091E80F81709927A2
:10C2400008958091D60F9091D70F08956BE676E010
:10C250008CE59EE00E947B711092D70F1092D60F52
:10C2600081E090E008950E94771266E776E08CE521
:10C270009EE00E947B7126E040E855E260E070E0BD
:10C2800085E39CE00E94DEA281E090E09093D70FCE
:10C290008093D60F0895EF92FF920F931F93CF9341
:10C2A000DF937C018B0101501109A801BC0185E3DA
:10C2B0009CE00E94DBB4F701329660E0CF018E195A
:10C2C0009F098017910718F48191680FF7CF85E3D4
:10C2D0009CE00E9462B585E39CE00E94AFB56EE7EA
:10C2E00076E08CE59EE00E945FB7E701CE018E19F3
:10C2F0009F0980179107A8F468816A3050F461E8BB
:10C3000076E08CE59EE00E945FB740E150E06881F6
:10C3100002C040E150E08CE59EE00E94B1B621965B
:10C32000E5CF8CE59EE0DF91CF911F910F91FF90BB
:10C33000EF900C9449B7CF92DF92EF92FF920F9358
:10C340001F93CF93DF93CDB7DEB762970FB6F89404
:10C35000DEBF0FBECDBF6C010B871C872D873E87CC
:10C360004F87588B698B7A8B6DEE74E1C7010E9401
:10C370006ACD892BD9F067EE74E1C7010E946ACDBE
:10C38000892BB9F061EE74E1C7010E946ACD892B57
:10C3900099F0ED851E2F1F706DED74E1C7010E94AD
:10C3A0006ACD892B61F0E12FF0E00BC0EDE0F0E009
:10C3B00008C0EFE0F0E005C0EEE0F0E002C0E0E130
:10C3C000F0E09B85992309F45CC13097B1F1319776
:10C3D000EF30F10508F041C18827EC50FF4F8F4F37
:10C3E0000C9466D6CE010B960E94D29B70930F10D0
:10C3F00060930E109B012A5031092531310508F058
:10C400002CC120EF260F20930C109B01770F440BBB
:10C41000550BD6011296ED91FC9113970190F08186
:10C42000E02D60817181ED91FC910684F785E02D0E
:10C4300003E816E0C601199510C11982892F90E012
:10C44000FC013197EE30F10508F085C08827ED5FDB
:10C45000FE4F8F4F0C9466D68091E70F81608093DA
:10C4600006106DE070E08BE192E00E944B61D60116
:10C470001296ED91FC9113970190F081E02D60816F
:10C480007181ED91FC910288F389E02D28E836E076
:10C490004DE856E01EC08091E70F8E7F8093061016
:10C4A0006DE070E08EE092E00E944B61D601129642
:10C4B000ED91FC9113970190F081E02D60817181E5
:10C4C000ED91FC910288F389E02D28E836E040E9FF
:10C4D00056E0C6011995D2C0109200108091E70F66
:10C4E00081608093061068ED74E131C081E0809333
:10C4F00000108091E70F81608093061063ED74E176
:10C5000026C082E0809300108091E70F81608093C5
:10C5100006106EEC74E11BC084E0809300108091E3
:10C52000E70F8160809306106AEC74E110C083E02D
:10C530008093001064E976E089EF9EE00E945FB787
:10C540008091E70F81608093061061EC74E1CE0169
:10C5500001960E9473CDD6011296ED91FC9113972E
:10C560000190F081E02D60817181ED91FC91028854
:10C57000F389E02D28E836E03CC01982903199F02B
:10C5800040F49C30F9F483E08093021068ED74E18C
:10C590000EC0913189F09231A9F482E080930210AB
:10C5A00061EB74E104C0109202106CEB74E1CE01F7
:10C5B00001960E9473CD0CC081E08093021065EB60
:10C5C00074E1F5CFCE010B960E94D29B60930210CE
:10C5D000D6011296ED91FC9113970190F081E02D18
:10C5E00060817181ED91FC910288F389E02D29E948
:10C5F00036E0AE014F5F5F4FC60119952EC0CE01E8
:10C600000B960E94D29B6093001027C0913019F0C6
:10C61000923061F022C080E506C0913019F092306E
:10C6200029F007C083E08093051017C01092051011
:10C6300014C0CE010B960E94D29B609304100DC0D3
:10C64000913031F0923049F480910610877F03C019
:10C65000809106108860809306101092FA0F81E096
:10C660008093F20F8DE48093F30F8FE58093F40FA6
:10C6700065E270E089EE9FE00E944B6181E090E00E
:10C680000EC0E031F10548F78827EF5EFE4F8F4F6F
:10C690000C9466D68FEF9FEF02C019825CCF629632
:10C6A0000FB6F894DEBF0FBECDBFDF91CF911F91C3
:10C6B0000F91FF90EF90DF90CF9008954F925F928F
:10C6C0006F927F928F929F92AF92BF92CF92DF92A2
:10C6D000EF92FF920F931F93CF93DF93CDB7DEB707
:10C6E0002A970FB6F894DEBF0FBECDBF613071053B
:10C6F00009F09CC24C010E9407AC9B01AC01609107
:10C70000E30F7091E40F8091E50F9091E60FAA245A
:10C71000AA94BA2C650118E8E12E13E1F12E00E08D
:10C7200010E00E9482488823B9F080E00E946C48A3
:10C730006093E30F7093E40F8093E50F9093E60FFF
:10C740006EE976E08CE59EE00E947B716DE070E022
:10C7500081E092E00E944B6164E670E080E090E04E
:10C760000E94CDAB85E39CE00E9436B518161906F1
:10C770000CF059C209EE1FE08EE0E82E80E1F82EA1
:10C780000E9407AC60933D0C70933E0C80933F0C6D
:10C790009093400C85E39CE00E9414B597FF49C23A
:10C7A0000E9407AC40903D0C50903E0C60903F0CB6
:10C7B0007090400CDC01CB0184199509A609B709DA
:10C7C0004090390C50903A0C60903B0C70903C0CAF
:10C7D00084159505A605B705E8F285E39CE00E945F
:10C7E00036B5892B59F062E070E080E090E00E945D
:10C7F000CDAB85E39CE00E9414B5EFCF80910D1086
:10C800009091E20F891709F40EC28093E20F809194
:10C810000C1090E0409690930F1080930E10809132
:10C82000F60F90E09093E10F8093E00F809100105D
:10C8300090E09093DF0F8093DE0F8091021090E0E4
:10C840009093DD0F8093DC0F8091041090E0909323
:10C85000DB0F8093DA0F8091061090E09093E80F41
:10C860008093E70F8091051090E09093D90F80930B
:10C87000D80F80910810F401A281B3812081318109
:10C880000D90BC91A02D6D917C91D9015296ED91A6
:10C89000FC91539726EA36E080FF03C04DE856E04E
:10C8A00002C040E956E0C40119958091D80F9091DB
:10C8B000D90F80389105A9F4D4011296ED91FC911D
:10C8C00013970190F081E02D60817181ED91FC91D1
:10C8D0000288F389E02D2DEA36E04DE856E0C401E8
:10C8E00019958091D80F9091D90F892BA9F4D40173
:10C8F0001296ED91FC9113970190F081E02D6081EB
:10C900007181ED91FC910288F389E02D2DEA36E0EA
:10C9100040E956E0C401199563EB76E08CE59EE0B2
:10C920000E945FB76AE070E08091E70F9091E80F96
:10C930000E94AA9F8091E70FF401A281B381208118
:10C9400031810D90BC91A02D6D917C91D9015296B1
:10C95000ED91FC9153972AEB36E083FF03C04DE83D
:10C9600056E002C040E956E0C40119958091E70FF6
:10C97000F401A281B381208131810D90BC91A02D61
:10C980006D917C91D9015296ED91FC91539721ECD8
:10C9900036E081FF03C04DE856E002C040E956E0B2
:10C9A000C40119952091DA0F3091DB0F032E000C92
:10C9B000440B550BD4011296ED91FC911397019005
:10C9C000F081E02D60817181ED91FC910684F78505
:10C9D000E02D0DEC16E0C40119958091DC0F9091CB
:10C9E000DD0F892BA9F4D4011296ED91FC911397D8
:10C9F0000190F081E02D60817181ED91FC910288C0
:10CA0000F389E02D29E936E044ED56E0C40119959B
:10CA10008091DC0F9091DD0F0197A9F4D40112965B
:10CA2000ED91FC9113970190F081E02D608171816F
:10CA3000ED91FC910288F389E02D29E936E049ED7A
:10CA400056E0C40119958091DC0F9091DD0F02979B
:10CA5000A9F4D4011296ED91FC9113970190F08105
:10CA6000E02D60817181ED91FC910288F389E02DC8
:10CA700029E936E040EE56E0C40119958091DC0FBB
:10CA80009091DD0F0397A9F4D4011296ED91FC91DA
:10CA900013970190F081E02D60817181ED91FC91FF
:10CAA0000288F389E02D29E936E044EE56E0C4011E
:10CAB00019958091DA0F9091DB0FF401A281B38177
:10CAC000208131810D90BC91A02D6D917C91D90177
:10CAD0005296ED91FC9153972DEC36E0892B19F489
:10CAE00040E956E002C04DE856E0C4011995209196
:10CAF0000E1030910F10032E000C440B550BD40177
:10CB00001296ED91FC9113970190F081E02D6081D8
:10CB10007181ED91FC910684F785E02D03E816E024
:10CB2000C40119952091E00F3091E10F2F3F31059D
:10CB3000B9F0032E000C440B550BD4011296ED9165
:10CB4000FC9113970190F081E02D60817181ED914E
:10CB5000FC910684F785E02D09EE16E0C4011995D5
:10CB600019828091DE0F9091DF0F009719F468ED24
:10CB700074E11DC08130910519F463ED74E117C0B3
:10CB80008230910519F46EEC74E111C08330910587
:10CB900019F461EC74E10BC08430910519F46AEC6E
:10CBA00074E105C08D36910531F46DEA74E1CE0172
:10CBB00001960E9473CD2091DE0F3091DF0F032E7E
:10CBC000000C440B550BD4011296ED91FC91139778
:10CBD0000190F081E02D60817181ED91FC910684DE
:10CBE000F785E02D0FEE16E0C40119958091E70F4F
:10CBF000F401A281B381208131810D90BC91A02DDF
:10CC00006D917C91D9015296ED91FC91539728E852
:10CC100036E080FF04C0AE014F5F5F4F02C040E9C5
:10CC200056E0C401199588EE93E00BC080E090E0D7
:10CC300008C0F80181938F01EE16FF0609F0A0CD20
:10CC4000CCCD2A960FB6F894DEBF0FBECDBFDF91D4
:10CC5000CF911F910F91FF90EF90DF90CF90BF90F9
:10CC6000AF909F908F907F906F905F904F900895BE
:10CC70002F923F924F925F926F927F928F929F92EC
:10CC8000AF92BF92CF92DF92EF92FF920F931F93DA
:10CC9000CF93DF93CDB7DEB762970FB6F894DEBFC0
:10CCA0000FBECDBF5C018091D10F811103C066E939
:10CCB00074E158C160E083E00E9455AA61E070E031
:10CCC00080E090E00E94CDABBE016F5F7F4F80E0BF
:10CCD0000E947972892B09F043C1898183FF40C189
:10CCE00044E0BE016F5F7F4F82E00E94FE710097BB
:10CCF00091F429813A813227232732273093FA0C85
:10CD00002093F90C2B813C81322723273227309343
:10CD1000F80C2093F70C0E94577265EF76E08CE5D3
:10CD20009EE00E945FB76091F90C7091FA0C80E070
:10CD300090E00E94AAD4D62E372E2C01462F572FD2
:10CD4000BC018CE59EE00E9443A36BEF76E08CE58E
:10CD50009EE00E945FB76091F70C7091F80C80E044
:10CD600090E00E94AAD4C62E272E898B9A8B462F3C
:10CD7000572FBC018CE59EE00E9443A363E077E05F
:10CD80008CE59EE00E945FB742E0BE016F5F7F4F7F
:10CD900081E10E94FE7149815A81892B21F4542737
:10CDA0004527542702C040E050E060E070E0409327
:10CDB000D20F5093D30F6093D40F7093D50F2AE006
:10CDC00030E08CE59EE00E94FAB620E030E44CE1D1
:10CDD00056E46D2D732DC2010E94A5D487FF6DC04E
:10CDE000D5011296ED91FC911397008111816FE0AE
:10CDF00077E0C8010E94565A3C0163E177E0C80120
:10CE00000E94565A4C0119821A821B821C820B8185
:10CE10000F7000670B832D2D8D2D932DD2018D83E7
:10CE20009E83AF83B887E980FA801C813E814F8161
:10CE300058856FEFC3010E94C34A19821A821B8270
:10CE40001C820B810F7000670B832C2D8C2D922D73
:10CE5000A989BA898D839E83AF83B887E980FA80D8
:10CE60001C813E814F8158856FEFC4010E94C34AE7
:10CE700028E137E04D2D532DB201C5010E94051563
:10CE80002DE137E04C2D522D69897A89C5010E9428
:10CE900005154091D20F5091D30F6091D40F70912E
:10CEA000D50FCE0101960E94DD4843E257E0BE0156
:10CEB0006F5F7F4FC5010E94CE1469E277E08CE579
:10CEC0009EE00E947B71BE016F5F7F4F80EE0E94EB
:10CED0007972892B19F419811F3F39F46BE277E0DD
:10CEE0008CE59EE00E947B7134C015FF06C06CE4A7
:10CEF00077E08CE59EE00E945FB714FF06C060E615
:10CF000077E08CE59EE00E945FB713FF06C063E701
:10CF100077E08CE59EE00E945FB712FF06C068E8EC
:10CF200077E08CE59EE00E945FB711FF06C06FE9D5
:10CF300077E08CE59EE00E945FB710FF06C065EBCE
:10CF400077E08CE59EE00E945FB78CE59EE00E9452
:10CF500049B761E083E00E9455AA81E090E00CC0EF
:10CF60006BE774E189EF9EE00E9422B689EF9EE0B4
:10CF70000E9449B780E090E062960FB6F894DEBF59
:10CF80000FBECDBFDF91CF911F910F91FF90EF901A
:10CF9000DF90CF90BF90AF909F908F907F906F90D9
:10CFA0005F904F903F902F900895089587E090E014
:10CFB00008958AE090E0089581E090E0089588E087
:10CFC00090E00895CF93DF93009709F46AC0FC01C5
:10CFD0002081222309F465C0EC016FEC7FE00E9400
:10CFE0006ACD892B09F442C063EB7FE0CE010E9439
:10CFF0006ACD892BF1F16BE375E1CE010E946ACD18
:10D00000892BD1F167E375E1CE010E946ACD892BAE
:10D01000B1F163E375E1CE010E946ACD892B91F1F4
:10D020006FE275E1CE010E946ACD892B71F16BE24E
:10D0300075E1CE010E946ACD892B51F167E275E15D
:10D04000CE010E946ACD892B31F162E275E1CE01F9
:10D050000E946ACD892B11F16EE175E1CE010E942B
:10D060006ACD892BF1F48CE090E01DC082E090E065
:10D070001AC081E090E017C088E090E014C085E01D
:10D0800090E011C086E090E00EC087E090E00BC019
:10D0900089E090E008C08AE090E005C08BE090E075
:10D0A00002C080E090E0DF91CF9108950C940BCB0B
:10D0B0000C940BCB0F931F93CF93DF938C01FC0148
:10D0C000C081D1816FE270E0CE010E9426DA009724
:10D0D000C1F0FC011192CF010E94E267EC0166E60B
:10D0E00075E189EF9EE00E9422B64AE050E0BE0161
:10D0F00089EF9EE00E9442B789EF9EE00E9449B707
:10D1000009C0CE010E94E267EC01892B19F0F801F9
:10D1100011821082CE01DF91CF911F910F9108955E
:10D12000DC01ED91FC91309729F090859F7081E0B2
:10D13000953009F080E00895EF92FF920F931F93CE
:10D14000CF93DF93EC017B018E819F81892B01F5C9
:10D15000888199810E949C9F082F10E0053011055D
:10D16000BCF40E942ABBFC01892B41F08085807FA2
:10D17000826080871186128613861486FF83EE8371
:10D18000BF01888199810E94BC9F0F5F1F4FE6CF2E
:10D19000EE81FF81309751F080858F70823021F4CD
:10D1A000E682F782F70102C0E0E0F0E0CF01DF9114
:10D1B000CF911F910F91FF90EF900895CF92DF9242
:10D1C000EF92FF920F931F93CF93DF93EC016A01CD
:10D1D0007B018E819F81892B01F5888199810E9435
:10D1E0009C9F082F10E005301105BCF40E942ABB5B
:10D1F000FC01892B41F08085807F826080871186C9
:10D20000128613861486FF83EE83BF01888199817D
:10D210000E94BC9F0F5F1F4FE6CFEE81FF813097CA
:10D2200011F180858F708230F1F4C186D286E38659
:10D23000F4866AE575E189EF9EE00E9422B62AE055
:10D2400030E0B701A60189EF9EE00E94FAB689EFAF
:10D250009EE0DF91CF911F910F91FF90EF90DF90B3
:10D26000CF900C9449B7DF91CF911F910F91FF9010
:10D27000EF90DF90CF900895FC0186819781009711
:10D2800091F0FC0120852F70223041F0253059F4B7
:10D2900060E00E941B9F009731F0FC016185728560
:10D2A00083859485089560E070E0CB0108950F9325
:10D2B0001F93CF93DF93FC01C281D381209799F014
:10D2C00088858F70823029F4672B69F489859A8567
:10D2D00014C0853041F48B01CE010E949C9F90E0E8
:10D2E000081719071CF080E090E007C0602FCE01FE
:10D2F0000E941B9FFC0181859285DF91CF911F9138
:10D300000F9108950F931F93CF93DF93EB0163E089
:10D31000FC01808191810E941B9F009741F1AE0129
:10D32000409550954F6F60E070E0FC0101851285DB
:10D3300023853485402351236223732341875287F9
:10D340006387748761E575E189EF9EE00E9422B6EC
:10D350004AE050E0BE0189EF9EE00E9442B789EFAB
:10D360009EE0DF91CF911F910F910C9449B7DF910F
:10D37000CF911F910F9108950F931F93CF93DF9338
:10D38000EB0163E0FC01808191810E941B9F00976B
:10D3900031F1AE01442760E070E0FC0101851285A7
:10D3A00023853485402B512B622B732B4187528769
:10D3B0006387748768E475E189EF9EE00E9422B676
:10D3C0004AE050E0BE0189EF9EE00E9442B789EF3B
:10D3D0009EE0DF91CF911F910F910C9449B7DF919F
:10D3E000CF911F910F910895CF93DF93EB0163E0ED
:10D3F000FC01808191810E941B9F009739F0FC0104
:10D400008185928588278C239D2302C080E090E04F
:10D41000DF91CF910895CF93C62F63E0FC01808107
:10D4200091810E941B9F0097F9F0FC014185528574
:10D43000638574854427662777274C2B418752875D
:10D440006387748760E475E189EF9EE00E9422B6ED
:10D450004AE050E06C2F89EF9EE00E94B1B689EF60
:10D460009EE0CF910C9449B7CF91089563E0FC0101
:10D47000808191810E941B9F009719F0FC0181859A
:10D4800008958FEF08958F929F92AF92BF92CF929F
:10D49000DF92EF92FF920F931F93CF93DF93CDB75D
:10D4A000DEB767970FB6F894DEBF0FBECDBF8C0115
:10D4B0007B014C018BE0880E911C9F8A8E8AF801BB
:10D4C000128611861386168A158A672B09F448C0BE
:10D4D000A0909610B0909710A114B10409F440C028
:10D4E0006FE270E0C7010E94DED96C01892B81F1E7
:10D4F000F701DE01119680E090E0BD012191222329
:10D5000041F02F3231F08431910519F02D930196BD
:10D51000F5CFFB01E80FF91F1082C5010E94565A92
:10D52000F80191838083B6016F5F7F4F4AE050E03E
:10D53000C4010E9417DACE0146960E945A68F8018B
:10D54000968B858B8E899F89892B69F413860BC0F6
:10D55000B701C5010E94565AF8019183808303C028
:10D56000F80111821082C8010E949068882319F086
:10D57000C8010E94A24C67960FB6F894DEBF0FBE9A
:10D58000CDBFDF91CF911F910F91FF90EF90DF9072
:10D59000CF90BF90AF909F908F900895CF93DF93DF
:10D5A000EC01798368831A8619861B861E8A1D8A78
:10D5B0000E949068882329F0CE01DF91CF910C94CE
:10D5C000A24CDF91CF9108954F925F926F927F921C
:10D5D0008F929F92AF92BF92CF92EF92FF920F9352
:10D5E0001F93CF93DF93CDB7DEB767970FB6F8944D
:10D5F000DEBF0FBECDBF009709F47CC0FC012085C3
:10D600002F70253009F076C02A015B018680978053
:10D610008091DD0A8F5F8093DD0A8114910409F403
:10D6200064C0F40180858F70843009F05AC0618530
:10D63000728580919610909197100E94565A3C01E5
:10D64000009709F44EC0FC0180858F70853009F089
:10D6500048C0B301CE0101960E94CE6AA114B10464
:10D6600031F0CE0101960E949068811145C060E0C2
:10D67000C3010E941B9F0097D9F0FC0120852F70E9
:10D680002230B1F481859285A385B4850797A105E1
:10D69000B10571F461E0C3010E941B9FA201B501B5
:10D6A0000E94E46AA114B104C1F48823B1F00FC050
:10D6B000A114B10491F4CE0101960E9490688823D0
:10D6C00061F0CE0101960E947E51892B31F0CE018E
:10D6D00001960E9418A081E01FC0CE0101960E9411
:10D6E00018A0F4018280938098CF8091DD0A815048
:10D6F0008093DD0A80E010C0C12C7201F501008129
:10D700001181228133814481558166817781CE01E7
:10D7100001960E942F25ABCF67960FB6F894DEBF17
:10D720000FBECDBFDF91CF911F910F91FF90EF9072
:10D73000CF90BF90AF909F908F907F906F905F90B1
:10D740004F9008950F931F93CF93DF93EC018B01BC
:10D750007B836A8381EC92E09983888360E070E048
:10D76000C8010E94576997FF03C09195819591095F
:10D770009D838C83D8011296ED91FC91139730977D
:10D7800071F090859F70923039F0953041F4CF015F
:10D790000E949C9F90E005C081E090E002C080E084
:10D7A00090E09F838E83DF91CF911F910F91089519
:10D7B000CF93DF93EC01FB012481358140815181BE
:10D7C000628173810E94FAB6CE01DF91CF910895F4
:10D7D000089508956F927F928F929F92AF92BF9219
:10D7E000CF92DF92EF92FF920F931F93CF93DF932D
:10D7F000CDB7DEB7C854D1090FB6F894DEBF0FBE5F
:10D80000CDBF3C014B01FC01E080F18067E975E090
:10D81000C7010E94565A5C0165E675E0C7010E9487
:10D82000565A6C01A114B10419F4892B09F4FDC0F6
:10D8300067EC77E0C7010E94565A8C016CEC77E0E8
:10D84000C7010E94565A7C01F301738063E175E1C0
:10D8500089EF9EE00E9422B64AE050E0672D89EFF2
:10D860009EE00E94B1B661E175E189EF9EE00E9401
:10D8700022B64AE050E0B40189EF9EE00E9442B730
:10D8800089EF9EE00E9449B7C114D104E1F1F6018D
:10D8900080858F708430B9F56185728540E450E0F1
:10D8A000CE0101960E9417DA0E94DD9D882359F16E
:10D8B0008091DC0A811127C06FE270E0CE010196F1
:10D8C0000E94DED9892B51F4F6012185328543E08F
:10D8D00050E060E4CE0101960E9438498114910421
:10D8E00009F491C00115110509F48AC0F801808579
:10D8F0008F70843009F084C0F80161857285FB0166
:10D90000808181118DC0A114B10409F48EC0F5018C
:10D9100080858F70843009F088C061857285CE0162
:10D9200001960E94436ACE0101960E949068882366
:10D9300009F461C0892801F10115110529F0F801E8
:10D9400080858F708430B1F025961CAE1DAE1EAE62
:10D950001FAE259729961CAE1DAE1EAE1FAE299791
:10D9600024962FAD24972F70CC24C394E12CF12C56
:10D9700001E01FC0F80133C0E114F10429F0F70100
:10D9800080858F70843051F125961CAE1DAE1EAE81
:10D990001FAE259729961CAE1DAE1EAE1FAE299751
:10D9A00024962FAD24972F70CC24C394E12CF12C16
:10D9B00002E023961FAD239725963FAD259740E0C3
:10D9C00027965FAD279728966FAD289729967FAD4C
:10D9D0002997CE0101960E942F250DC0F701618580
:10D9E0007285FB018081882331F040E050E0CE0158
:10D9F00001960E94D86ECE0101960E9418A015C013
:10DA00006DE876E00DC0E114F10429F0F70180859E
:10DA10008F70843019F060E976E002C0F7016DCFB5
:10DA2000CE0101960E94FF9E6ECFC85BDF4F0FB6FE
:10DA3000F894DEBF0FBECDBFDF91CF911F910F9144
:10DA4000FF90EF90DF90CF90BF90AF909F908F901E
:10DA50007F906F900895AF92BF92CF92DF92EF9236
:10DA6000FF920F931F93CF93DF93CDB7DEB7289725
:10DA70000FB6F894DEBF0FBECDBF6C01162F5A0152
:10DA8000DC018D919C911197892B09F442C1149668
:10DA9000ED91FC911597309709F43BC180816F3F60
:10DAA000B9F484FF34C14330510509F430C1118108
:10DAB00012951F7069EF74E189EF9EE00E9422B613
:10DAC0004AE050E0612F89EF9EE00E94B1B602C0AB
:10DAD00084FD1FC1D6011496ED91FC91159701812B
:10DAE0000F70101769F11396FC9067EF74E189EFDE
:10DAF0009EE00E9422B64AE050E06F2D89EF9EE042
:10DB00000E94B1B665EF74E189EF9EE00E9422B6F3
:10DB10004AE050E0602F89EF9EE00E94B1B662EFCC
:10DB200074E189EF9EE00E9422B64AE050E0612F46
:10DB300089EF9EE00E94B1B689EF9EE00E9449B74E
:10DB4000812F90E08D30910508F09CC0FC01D6013A
:10DB50001496ED90FC9015978827EF5DFE4F8F4F40
:10DB60000C9466D6F7019181292F2F70253009F486
:10DB700089C0D6018D919C91263048F42230A9F4B9
:10DB800062ED77E00E94565AF701608159C0273054
:10DB900049F02A3051F468ED77E00E94565AF701B7
:10DBA00060816BC061ED77E055C06CEC77E038C008
:10DBB00067EC77E0D6018D919C910E94565AF7014F
:10DBC0002081622F6170322F309530FB20F921C007
:10DBD0006FED77E0D6018D919C910E94565AF70126
:10DBE000208121FB662760F931E0362730FB21F9DF
:10DBF00010C06CE975E0D6018D919C910E94565A37
:10DC0000F701208122FB662760F931E0362730FBDF
:10DC100022F9208335C06CEC77E0D6018D919C9180
:10DC20000E94565A60E02CC06EE675E002C063E7C1
:10DC300075E0F601808191810E94565AD7016C915E
:10DC400061701EC069E775E002C06FE775E0F6011C
:10DC5000808191810E94565AD7016C9166956170BE
:10DC60000FC066E875E002C06CE875E0F6018081DF
:10DC700091810E94565AD7016C9162FB662760F928
:10DC8000009759F4D6011496ED91FC9115971F70E9
:10DC90008181807F182B11833AC0D6011496ED91B3
:10DCA000FC911597B3E0AB16B10411F11F702181FF
:10DCB000207F122B118319821A821B821C821D82E3
:10DCC0001E821F8218860B810F700B831982E12C34
:10DCD000FA801C8120E03E814F8158850E94C34A12
:10DCE000D6011496ED91FC91159780818F7E0EC020
:10DCF00081818F70982F9295907F892B8183D60197
:10DD00001496ED91FC91159780818061808381E06C
:10DD100001C080E028960FB6F894DEBF0FBECDBFDD
:10DD2000DF91CF911F910F91FF90EF90DF90CF90F7
:10DD3000BF90AF9008950F931F93CF93DF938C0103
:10DD4000EB01209741F060910C0D70910D0DCE010B
:10DD50000E94B4CD02C080E090E020E0AC01BE01A2
:10DD6000C801DF91CF911F910F910C949D9EFC01F2
:10DD70009281892F82958F7019F0823021F016C020
:10DD80009F70906292839B016E3681E078072CF43D
:10DD900077FF05C020E030E002C02DE631E02683A9
:10DDA000878130FB80F9878381E0089580E00895C2
:10DDB0006F927F928F929F92AF92BF92CF92DF929B
:10DDC000EF92FF920F931F93CF93DF93CDB7DEB700
:10DDD000E2970FB6F894DEBF0FBECDBF78AB6FA74A
:10DDE0005AAB49AB672B09F46FC2FA01309719F0AF
:10DDF0002081211109C0FC012385222329F09C01E7
:10DE0000255F3F4F3AAB29AB5C01E9A9FAA93097EE
:10DE100021F4F501E588F6880AC080818823C9F3DA
:10DE2000CE01C1960E945A687C01892B91F300E0D3
:10DE300010E08FA498A83401600E711EF301808158
:10DE4000882351F0082E000C990B0E947FD9F30112
:10DE500080830F5F1F4FEDCF8114910441F1F401D6
:10DE60008081882321F18D3229F190ED980F9A302D
:10DE700008F1853211F18B3719F1833221F12BE74B
:10DE8000622E25E1722E01E010E0C3010E947ACDDE
:10DE9000AC01B301C4010E9493CD892BB1F00F5F97
:10DEA0001F4FF9E06F0E711C0931110571F70FEF6B
:10DEB0001FEF0BC000E010E008C008E010E005C054
:10DEC0000EEF1FEF02C007E110E063E576E189EF96
:10DED0009EE00E9422B64AE050E0B80189EF9EE041
:10DEE0000E9442B789EF9EE00E9449B719A21AA288
:10DEF0001BA21CA21DA21EA21FA218A68BA18F707E
:10DF00008BA309A325E0E216F10439F086E0E816B8
:10DF1000F10429F407E110E002C008E110E0DE2C72
:10DF20006E2DCE0181960E94859A29873A874B876C
:10DF30005C876D877E878F87988B0A3011058CF4FC
:10DF40000830110524F50E3F9FEF19070CF4ACC102
:10DF50000F3FEFEF1E0709F00CF4B6C1012B81F162
:10DF6000A3C10731110509F45DC10831110509F09C
:10DF70009BC160E0CE0181960E94AD9A298B3A8BBD
:10DF80004B8B5C8B6D8B7E8B8F8B988F19C0CE01EA
:10DF90008F960E94454A2BA12F70206A2BA3092E31
:10DFA000000CAA0BBB0B482F8DA39EA3AFA3B8A751
:10DFB000E9A8FAA8CC24C39409A11AA13CA17DC167
:10DFC00019821A821B821C828B818F7080668B83E0
:10DFD0001982EFA5F8A9309709F463C080818823DE
:10DFE00009F45FC06FA478A8F3018081882359F0F9
:10DFF0008D3249F080538A3030F0FFEF6F1A7F0A7C
:10E0000078AA6FA6EFCFC3010E9443CD8C016EE2C8
:10E0100070E0C3010E94DED9009771F0FC0181819C
:10E02000803354F08A335CF4082E000C990B4C01B9
:10E03000F0E38F1A910806C0812C912C03C099E05F
:10E04000892E912C6CE270E0C3010E94DED900970A
:10E0500019F418AA1FA603C0019698AB8FA78114C4
:10E060009104B1F08AE0809F9001819F300D1124CE
:10E07000101611062CF0882799278819990901C0D4
:10E08000C401820F931F092E000CAA0BBB0B0CC0FE
:10E09000C801110FAA0BBB0B2B812F70206A2B8399
:10E0A00003C080E090E0DC0149815A816B817C8172
:10E0B000498F5A8F6B8F7C8F8D8F9E8FAF8FB8A3B8
:10E0C0006D2DCE0149960E94859A29833A834B8310
:10E0D0005C836D837E838F839887DB8CD2948FE003
:10E0E000D8224E0129E2820E911C00E010E08FA59B
:10E0F00098A9892B71F00330110559F00F5F1F4F5C
:10E10000CE018F960E94454AF401819391934F016D
:10E11000EECFFAE0EF16F10489F02BE0E216F104FD
:10E1200011F189E0E816F10419F5CE0149960E9433
:10E13000D29BCE0181960E94B76EB6C0CE014996A1
:10E140000E94D29B8BA1982F92959F7019F09230CC
:10E1500021F0AAC08F7080628BA3653610F064E650
:10E1600070E06EA3A1C0CE0149960E94D29B55C01B
:10E1700081E090E0D11002C080E090E0800F911F1C
:10E180008230910541F16CF4019709F08DC088E06F
:10E19000FE017996DE01919601900D928A95E1F744
:10E1A00083C08330910539F1049709F07DC01BA528
:10E1B00009A5CE0149960E94D29B8BA18F708062E7
:10E1C0008BA36FA388A570FB80F988A70EA31DA35E
:10E1D0006DA57EA522C019A5CE0149960E94D29BAD
:10E1E0008BA18F7080638BA36FA388A570FB80F9D0
:10E1F00088A71EA359C01BA509A5CE0149960E9458
:10E20000D29B8BA18F7080628BA36FA388A570FBBC
:10E2100080F988A70EA31DA347C0CE0181960E9456
:10E220009C8542C060E0CE0181960E94AD9A298F04
:10E230003A8F4B8F5C8F6D8F7E8F8F8F98A3FE01EF
:10E2400031967F0100E010E08FA598A9892B71F02D
:10E2500004301105E9F00F5F1F4FCE018F960E9429
:10E26000454AF701819391937F01EECF0330110569
:10E2700021F004301105C1F40BC09D812B8139813F
:10E280008BA18F7080648BA33FA32EA39DA30CC092
:10E290009F812D813B8149818BA18F7080658BA3EC
:10E2A0004FA33EA32DA398A7E9A8FAA8CC24C39412
:10E2B00009A11AA12BA13CA14DA15EA16FA178A536
:10E2C000C5010E942F2502C080E090E0E2960FB6C3
:10E2D000F894DEBF0FBECDBFDF91CF911F910F919C
:10E2E000FF90EF90DF90CF90BF90AF909F908F9076
:10E2F0007F906F9008950F931F93CF93DF93EC015E
:10E300000E9446B68C01CE010E9449B7800F911F32
:10E31000DF91CF911F910F9108951F93CF93DF93BA
:10E32000182F6091030D80EE9CE00E944347612FFF
:10E3300080EE9CE00E94584480EE9CE00E943C47A6
:10E3400069E070E080E090E00E94CDAB42E0609137
:10E35000030D80EE9CE00E946A4780EE9CE00E94E4
:10E360000F44182F80EE9CE00E940F44D12F20E034
:10E37000C22F9E01282BC901DF91CF911F910895D3
:10E380000F931F93CF93DF93182FEB016091EE0C47
:10E390008091EC0C9091ED0C0E9443478091EC0C25
:10E3A0009091ED0CDC01ED91FC910190F081E02D5C
:10E3B000612F19958E010C5F1F4F8091EC0C90918D
:10E3C000ED0CDC01ED91FC910190F081E02D699163
:10E3D00019950C171D0789F78091EC0C9091ED0CA5
:10E3E0000E943C47882319F082E090E002C080E060
:10E3F00090E0DF91CF911F910F9108950F931F939C
:10E40000CF93DF93082FEB01142F6091EE0C8091D6
:10E41000EC0C9091ED0C0E9443478091EC0C909194
:10E42000ED0CDC01ED91FC910190F081E02D602F6D
:10E4300019958091EC0C9091ED0C0E943C47811154
:10E440001EC0412F6091EE0C8091EC0C9091ED0C70
:10E450000E946A47CE01810F911D8C018091EC0CC6
:10E460009091ED0CDC01ED91FC910084F185E02DA3
:10E470001995892B39F0C017D10739F403C082E010
:10E4800090E010C080E090E00DC08091EC0C909185
:10E49000ED0CDC01ED91FC910284F385E02D1995E2
:10E4A0008993DCCFDF91CF911F910F910895823036
:10E4B000910599F038F4009769F00197A1F46DEE99
:10E4C00077E013C08330910559F0049761F46FE051
:10E4D00078E00BC065EE77E008C066EF77E005C036
:10E4E00060E078E002C06DE178E08CE59EE00C949D
:10E4F0005FB7EF92FF921F93CF93DF93C82F7B01FB
:10E500006091EE0C8091EC0C9091ED0C0E944347D1
:10E510008091EC0C9091ED0CDC01ED91FC9101905F
:10E52000F081E02D6C2F19958091EC0C9091ED0C01
:10E530000E943C47882319F0C2E0D0E002C0C0E04E
:10E54000D0E041E06091EE0C8091EC0C9091ED0CEC
:10E550000E946A4711E08091EC0C9091ED0CDC0177
:10E56000ED91FC910084F185E02D1995892B69F0DE
:10E570008091EC0C9091ED0CDC01ED91FC9102840A
:10E58000F385E02D1995182FE6CFF7011083CE0102
:10E59000DF91CF911F91FF90EF9008951092171087
:10E5A0001092161010921510109214100E94A74489
:10E5B0008EEF93E490931310809312108FEF93E4F7
:10E5C000909311108093101008950F931F93CF9381
:10E5D000DF93FC01818592850097C9F08B01EF01E3
:10E5E000DC01ED91FC910484F585E02D1995892BD2
:10E5F00071F089859A85DC01ED91FC910480F581AB
:10E60000E02DB801DF91CF911F910F91199480E017
:10E6100090E0DF91CF911F910F910895CF92EF92EB
:10E62000FF920F931F93CF93DF93CDB7DEB7289759
:10E630000FB6F894DEBF0FBECDBF19821A821B82BF
:10E640001C821D821E821F8218862B812F70CC2473
:10E65000C394E12CF12C02E01A813C8140E05E8100
:10E660006F8178850E942F2528960FB6F894DEBF1B
:10E670000FBECDBFDF91CF911F910F91FF90EF9013
:10E68000CF9008950F931F93CF93DF93EC012097C2
:10E6900031F10A811B8188858295807F85958595DA
:10E6A0008595859583FD06C08E819F81009711F029
:10E6B0000E94427388858F70843031F489859A85F1
:10E6C000009711F00E940BCB88819981009711F07F
:10E6D0000E940BCBCE010E940BCBE801D8CFDF917B
:10E6E000CF911F910F9108958F929F92AF92BF92F9
:10E6F000EF92FF920F931F93CF93DF938C017B01D7
:10E7000049015A010E942ABBEC01892B09F1888535
:10E71000807F8360888789869A86AB86BC8688815D
:10E720009981009711F00E940BCBC7010E9487D9F5
:10E7300099838883BE01C801DF91CF911F910F910A
:10E74000FF90EF90BF90AF909F908F900C94BC9FE4
:10E75000DF91CF911F910F91FF90EF90BF90AF90FD
:10E760009F908F900895CF92DF92EF92FF920F9338
:10E770001F93CF93DF93CDB7DEB728970FB6F894EA
:10E78000DEBF0FBECDBF6C018B0162E070E00E9466
:10E7900057697C0119821A821B821C821D821E828B
:10E7A0001F8218868B818F708B831982F7FC92C031
:10E7B00040E0B601CE0101960E94EE9963E070E060
:10E7C000C6010E945769AC011816190614F04FE3F0
:10E7D00050E081E0E816F10421F4012F110F110B34
:10E7E00004C082E0E816F1040CF411272FEF30E0AA
:10E7F000D8010E947DD69A01550F440B550B0E94FB
:10E8000011D68901C6010E94366AE82EF12C60E01B
:10E81000CE0101960E94D19A0817190771F40115CB
:10E82000110509F45AC082E0E816F10489F085E088
:10E83000E816F10409F051C00BC001151105C1F132
:10E8400086E0E816F10441F081E0E816F10421F0D9
:10E8500061E0C6010E940B6A17FD07C00F3F11055A
:10E8600031F02CF00FEF10E002C000E010E08B81DF
:10E87000982F92959F709150923018F08F70806110
:10E880008B830D8340E0B601CE0101960E949699DC
:10E8900082E0E816F10421F085E0E816F10429F49D
:10E8A00060E071E0C6010E942A4F60E072E00EC095
:10E8B00085E0E816F10489F082E0E816F10469F0D9
:10E8C00062E0C6010E940B6A60E071E0C6010E942E
:10E8D0002A4F03C080E090E002C081E090E02896DB
:10E8E0000FB6F894DEBF0FBECDBFDF91CF911F9161
:10E8F0000F91FF90EF90DF90CF900895CF93DF932B
:10E900001F92CDB7DEB76983DC01ED91FC910280E7
:10E91000F381E02D41E050E0BE016F5F7F4F19951C
:10E920000F90DF91CF910895DC01ED91FC91068C61
:10E93000F78DE02D199591E089270895862F089588
:10E9400081E086270895CF93DF931F92CDB7DEB77E
:10E950008983209119103981E0911A10F0911B10D0
:10E96000822F90E080959095F89400800822008294
:10E970004BE000C05DE000005A95E9F700800822F6
:10E980000894379508F4022A00824A9599F77894FA
:10E990000F90DF91CF9108950F931F93CF93DF9343
:10E9A0001F92CDB7DEB78C01DC01ED91FC910084A4
:10E9B000F185E02D1995892B51F0BE016F5F7F4FD6
:10E9C000F80184850E94A282898190E002C08FEFC5
:10E9D0009FEF0F90DF91CF911F910F910895FC0150
:10E9E00084850C94F382CF93DF931F92CDB7DEB76B
:10E9F00041E050E0BE016F5F7F4FFC0184850E94C3
:10EA0000F382181619061CF4898190E002C08FEF7A
:10EA10009FEF0F90DF91CF910895FC0184858430A2
:10EA200011F00C94F98080E090E0089544E050E00B
:10EA3000BC018FE090E00C9452BC44E050E0BC017B
:10EA400085E090E00C9452BC44E050E0BC0181E0D1
:10EA500090E00C9452BC08958CBD9DBD08956F92BA
:10EA60007F928F929F92AF92BF92CF92DF92EF925E
:10EA7000FF921F93CF93DF931F921F92CDB7DEB704
:10EA80005C013B016A01FC011485143041F481E012
:10EA900090E0F5019383828380E090E05BC07A018F
:10EAA0004130584018F0E12C88E0F82ECE01019654
:10EAB0000E9488C589819A810E942C75812F0E94AD
:10EAC000E5B24C0163E070E0812F0E9484828731BF
:10EAD00011F08C3121F48E149F0440F302C0E12C1C
:10EAE000F12CCE0101960E9488C589819A810E94ED
:10EAF0002C759701A30160E070E0812F0E9480B225
:10EB000060E270E0812F0E9478C562E070E0812FA2
:10EB10000E94848284FD14C063E070E0812F0E9413
:10EB20008482811104C0812F0E94B881B0CFCE01B0
:10EB300001960E9488C589819A810E942C75E5CF33
:10EB400040E162E070E0812F0E94AE81EF2809F47D
:10EB50009ECFC6010F900F90DF91CF911F91FF9034
:10EB6000EF90DF90CF90BF90AF909F908F907F906D
:10EB70006F9008958F929F92AF92BF92DF92EF9223
:10EB8000FF920F931F93CF93DF931F921F92CDB7E6
:10EB9000DEB7FC012485243009F082C05A018B01C4
:10EBA0007C01D12C8D2D0E941484811103C0F701AA
:10EBB000D48607C08B7F8831D1F3D394F4E0DF1281
:10EBC000F1CFF7018485843009F46AC020912B02CB
:10EBD00030912C022F5F3F4F11F420E030EC309346
:10EBE0002C0220932B0240912B0250912C0220E00A
:10EBF00061E00E94DB81F80182818F3F51F48381C3
:10EC00008F3F99F484818F3F81F485818F3F69F430
:10EC100044C081110AC0F8018381811106C084813A
:10EC2000811103C085818823C1F1A114B104A9F128
:10EC3000F701D484CE0101960E9488C589819A810A
:10EC40000E942C75B8016E5F7F4F8D2D0E94BB8492
:10EC5000B5018D2D0E94AA8464E070E08D2D0E9484
:10EC600078C50E9407AC4B015C01F4E98F0EF1E11D
:10EC70009F1EA11CB11CC7010E948DC5873141F1A7
:10EC800061E070E080E090E00E94CDAB0E94947C57
:10EC9000C7010E948DC5811106C084E0F7018487F9
:10ECA00080E090E01DC00E9407AC86169706A8067B
:10ECB000B90608F7F70184850E94B88184E0F7015E
:10ECC000848767E677E18CE59EE00E944DB7E8CF48
:10ECD0006CE577E18CE59EE00E944DB781E090E025
:10ECE0000F900F90DF91CF911F910F91FF90EF90B8
:10ECF000DF90BF90AF909F908F90089578941F926F
:10ED00000F920FB60F9211240BB60F92CF92DF9293
:10ED1000EF92FF920F931F932F933F934F935F9325
:10ED20006F937F938F939F93AF93BF93CF93DF9313
:10ED3000EF93FF93809170008E7F809370000FE3BC
:10ED400010E08BE1E82EF12C9BE2C92ED12CC09172
:10ED50001C10D0911D102097F9F40332110508F40E
:10ED60003BC003521109E0911A10F0911B109081E1
:10ED700020911910822F8095982390839BE0D701D2
:10ED80001197F1F79150D9F78081822B8083C601CA
:10ED90000197F1F780E00DC00B301105E8F00B5042
:10EDA0001109E0911E10F0911F10EC0FFD1F31971B
:10EDB00080810E94A3742196D0931D10C0931C10D3
:10EDC0008091290290912A028C179D0708F0BFCFED
:10EDD00010921D1010921C10809170008160809321
:10EDE0007000FF91EF91DF91CF91BF91AF919F9113
:10EDF0008F917F916F915F914F913F912F911F91D3
:10EE00000F91FF90EF90DF90CF900F900BBE0F907F
:10EE10000FBE0F901F90189581E08093181080917D
:10EE20002802282F30E0F901E053FF4EE491F0E092
:10EE3000EE0FFF1FE456F14E4591549150931B1075
:10EE400040931A10F901E657FF4EE491E093191030
:10EE500061E00E9484AA83E08093B100E0E7F0E0E3
:10EE60008081816080830895CF93DF9318161906FF
:10EE700044F0809170008E7F809370001092181083
:10EE800019C0EC0180911E1090911F100E940BCBB5
:10EE9000CE01C130D24014F080E092E090932A027B
:10EEA000809329020E9473CA90931F1080931E10B2
:10EEB000892B29F410922A021092290208C080910D
:10EEC0001810811104C0DF91CF910C940C77DF9161
:10EED000CF910895FF920F931F93CF93DF938C01EF
:10EEE000F62E80911810811102C00E940C77E80163
:10EEF0002197C11582E0D80798F48091290290915A
:10EF00002A028017910718F4C8010E943477809173
:10EF10001E1090911F10009719F0C80FD91FF8828A
:10EF2000DF91CF911F910F91FF900895DC0180E058
:10EF3000615040F09D91E82FE927F0E0E45AF94E46
:10EF40008491F6CF0895AF92BF92CF92DF92EF9265
:10EF5000FF921F93CF93DF93EC010E9407AC6B01EC
:10EF60007C0128EEC20E23E0D21EE11CF11C8BE4D2
:10EF7000A82EB12C0E9407AC6C157D058E059F054F
:10EF800098F460EFCE010E945347CE010E94494899
:10EF9000182F80FF11C0EF85F889309709F0199577
:10EFA000C5010197F1F7E6CF81E08A8360E378E05D
:10EFB0008CE59EE00E947B71812FDF91CF911F91A4
:10EFC000FF90EF90DF90CF90BF90AF9008950F9398
:10EFD0001F93CF93DF93EC01162F042F0E94A3778A
:10EFE000002319F0CE010E946048CE010E944D47D7
:10EFF00065EA80EE9CE00E945844612F80EE9CE020
:10F000000E945844CE01DF91CF911F910F910C9433
:10F010003F47EF92FF920F931F93CF93DF938C01A3
:10F020007B0140E065E50E94E777E70188E0E80EB4
:10F03000F11C699140E0C8010E94E777CE15DF0519
:10F04000C1F7DF91CF911F910F91FF90EF9008953D
:10F050001F93CF93DF93EC01162F0E94A377CE016D
:10F060000E944D4762ED80EE9CE00E945844612F63
:10F0700070E06095709584E0660F771F8A95E1F7E0
:10F08000612B80EE9CE00E945844CE010E943F47D5
:10F09000CE010E944948181711F084E08A83DF915D
:10F0A000CF911F9108951F93CF93DF93EC010E949E
:10F0B000A37780FD31C0CE010E94554860E0CE01AB
:10F0C0000E942878CE010E94A377CE010E944D476E
:10F0D00064EB80EE9CE00E945844CE010E943F47C2
:10F0E000CE010E94A377182F82FF03C082E08A839B
:10F0F00004C08A81823009F41A828881882341F011
:10F10000CE010E945548682F6160CE010E94287888
:10F1100011FB882780F901C080E0DF91CF911F911A
:10F120000895CF92DF92EF92FF920F931F93CF93A8
:10F13000DF937C01EB018A01FC01858196810E94AD
:10F1400053788823C9F1BE01F701858196810E9419
:10F15000097840E06EEBF701858196810E94E777A0
:10F16000E8016801F9E0CF0ED11CF7010581168195
:10F17000C8010E94A377C8010E944D4766E980EE4E
:10F180009CE00E945844C8010E943F47C8010E9469
:10F19000A37761EEC8010E945347C8010E94494805
:10F1A0008993CC16DD0609F7F701858196810E94C7
:10F1B000537891E0813009F090E0892FDF91CF9171
:10F1C0001F910F91FF90EF90DF90CF900895CF9314
:10F1D000DF93EA010E949178882339F068E0CE013C
:10F1E0000E94967791E02885281390E0892FDF917F
:10F1F000CF910895CF93DF93CDB7DEB729970FB6A0
:10F20000F894DEBF0FBECDBFAE014F5F5F4F0E94CF
:10F21000E778882389F08D818F3361F020F48F3176
:10F2200059F489E00CC08F3519F08F3739F004C0DC
:10F230008BE005C08AE003C080E001C08CE0299625
:10F240000FB6F894DEBF0FBECDBFDF91CF9108950A
:10F250006F927F928F929F92AF92BF92CF92DF92E6
:10F26000EF92FF920F931F93CF93DF93FC012485BE
:10F2700021119EC0872E762EEC010E9453788111B9
:10F2800008C06BE378E08CE59EE00E947B718FEF15
:10F2900090C0CE010E94A37740E060EFCE010E94B3
:10F2A000E777C12CD12C66246A94EE24E394F12CE8
:10F2B0000C2D06950695069510E08C2D877057014C
:10F2C00001C0AA0C8A95EAF78B85082E000C990BD1
:10F2D000C816D90634F4FE01E00FF11F93809A207E
:10F2E00006C099249394C816D90609F0912CCE0132
:10F2F0000E94A377CE010E944D4768E780EE9CE014
:10F300000E945844911002C060E001C060E880EEA5
:10F310009CE00E945844CE010E943F47CE010E94CB
:10F32000A377282F2074982F907885FF11C022236F
:10F33000A9F042E050E0682F8CE59EE00E94B1B653
:10F3400067E478E08CE59EE00E947B718EEF31C02F
:10F35000211104C0911104C06C2C08C0992331F014
:10F36000FE01E00FF11F83818A2907C0FE01E00F33
:10F37000F11F8A2D8095938189238383FFEFCF1A14
:10F38000DF0A80E4C816D10409F092CF6B86EFEF54
:10F390006E1202C081E08C87DE011396E72DF82DF6
:10F3A0002B968D918193CA17DB07D9F781E001C0B5
:10F3B00080E0DF91CF911F910F91FF90EF90DF9050
:10F3C000CF90BF90AF909F908F907F906F90089557
:10F3D000AF92BF92CF92DF92EF92FF920F931F9363
:10F3E000CF93DF93CDB7DEB7AF970FB6F894DEBFFC
:10F3F0000FBECDBF7C015B016A010AEE13E01A83E8
:10F4000009831B821C821D821E82CE0109960E94E6
:10F4100029811BA70AA71CA61DA61EA61FA68091B0
:10F42000DA0C9091DB0CA091DC0CB091DD0C8EA37A
:10F430009FA3A8A7B9A78B839C83AD83BE8318869F
:10F440001F82AE01465D5F4FB501CE0101960E945D
:10F4500013AC81309105B1F4D701ED91FC91068494
:10F46000F785E02D1DA30CA38CA59DA5AEA5BFA57A
:10F470008EA39FA3A8A7B9A7A601BE016C5D7F4F6D
:10F48000C7011995AF960FB6F894DEBF0FBECDBF7A
:10F49000DF91CF911F910F91FF90EF90DF90CF9070
:10F4A000BF90AF900895A8950895E5E0F1E08081C0
:10F4B0008F7980830895E5E0F1E080818066808324
:10F4C00008950E94C2A7A8950E940F1B039724F0DD
:10F4D0000E94E6AF0E94493D0C940314CF92DF9244
:10F4E000EF92FF920F931F93CF93DF936C01EB0189
:10F4F00009900020E9F72197C61BD70BC032D10530
:10F5000014F0CFE1D0E08B01E12CF12CEC16FD06DC
:10F5100064F4F80161918F01C7018C0D9D1D0E945B
:10F52000D1D5FFEFEF1AFF0AF1CF60E0C6018C0FD3
:10F530009D1FDF91CF911F910F91FF90EF90DF9072
:10F54000CF900C94D1D5CF93DF931F92CDB7DEB778
:10F550001982892B21F0FB016281738103C0BE01F6
:10F560006F5F7F4F86E390E00E946E7A6AE178E1F8
:10F570008CE49EE00E9422B60F90DF91CF91089517
:10F58000CF93DF93C0E0D0E060E0CE010E94D1D500
:10F590002196CD34D105C1F76CE486E490E00E9459
:10F5A000D1D568E487E490E00E94D1D563E488E493
:10F5B00090E00E94D1D566E489E490E00E94D1D524
:10F5C0006AE078E18CE49EE0DF91CF910C9422B662
:10F5D000EF92FF920F931F93CF93DF931F92CDB7BC
:10F5E000DEB78B01CE0101969F938F9385E99BE057
:10F5F0009F938F9384E99BE09F938F9383E99BE094
:10F600009F938F9382E99BE09F938F9381E99BE087
:10F610009F938F9380E99BE09F938F9381E598E080
:10F620009F938F93FB0183818F9382818F930E949D
:10F630009DDA0FB6F894DEBF0FBECDBF06977CF4FF
:10F64000F801028113816CE278E184E59EE00E947A
:10F6500022B6B80184E59EE00E945FB719C00E94FF
:10F66000359780E9E82E8BE0F82E00E010E0F701F6
:10F6700061917F01C8010E94D1D50F5F1F4F0630F5
:10F680001105A9F76EE378E18CE49EE00E9422B6B2
:10F690000F90DF91CF911F910F91FF90EF90089500
:10F6A000EF92FF920F931F93CF93DF93CDB7DEB707
:10F6B0002C970FB6F894DEBF0FBECDBF8C017B0137
:10F6C0008AEE93E09A8389831B821C821D821E82AC
:10F6D00098878F8319861A861B861C86053011052C
:10F6E0005CF0BE01695F7F4FF701808591850E94C4
:10F6F0006A58892B09F052C0BE016F5F7F4F82E1CB
:10F7000090E00E944B58043011050CF44FC0BE012C
:10F71000695F7F4FF701868197810E946A58892B24
:10F7200009F444C0BE01695F7F4F8EE090E00E9403
:10F730004B58BE01695F7F4FF701848195810E941C
:10F740006A58892BF1F1BE01695F7F4F8AE090E032
:10F750000E944B58BE01695F7F4FF7018281938100
:10F760000E946A58892BC1F1BE01695F7F4F86E014
:10F7700090E00E944B5863EF77E18CE49EE00E949A
:10F7800022B62C960FB6F894DEBF0FBECDBFDF9128
:10F79000CF911F910F91FF90EF900895BE01695F87
:10F7A0007F4F82E190E00E944B58B1CFBE016F5F66
:10F7B0007F4F8EE090E00E944B58033011050CF013
:10F7C000B8CFBE016F5F7F4F8AE090E00E944B5838
:10F7D000023011050CF0BECFBE016F5F7F4F86E097
:10F7E00090E00E944B580130110529F6BE016F5F71
:10F7F0007F4F86E090E00E944B586AEF77E18CE4FF
:10F800009EE00E9422B6B7CFCF93DF93CDB7DEB78D
:10F810002C970FB6F894DEBF0FBECDBF1C821B82A3
:10F820001E821D828FEF9FEF98878F8386E494E07E
:10F830009A8389838CE490E09A8789871C861B864B
:10F8400069ED77E18CE49EE00E9422B66091201081
:10F8500070912110CE0101960E941EA86FEFCE017B
:10F8600001960E9451B969EC77E18CE49EE00E9418
:10F8700022B62C960FB6F894DEBF0FBECDBFDF9137
:10F88000CF910895CF93DF93CDB7DEB769970FB6C9
:10F89000F894DEBF0FBECDBF8FE290E09A838983DC
:10F8A000FE01339687E1DF011D928A95E9F764EB4B
:10F8B00077E18CE49EE00E9422B6AE014E5F5F4F7E
:10F8C00066E080E99BE00E94984A1E8665E678E043
:10F8D000CE0101960E94D3D9BE016F5F7F4F89EFA1
:10F8E0009EE00E945FB7CE0101960E94FF551E86E2
:10F8F0006DE678E0CE0101960E94D3D9BE016F5F1C
:10F900007F4F89EF9EE00E945FB767E778E0CE0106
:10F9100001960E949B6E69960FB6F894DEBF0FBEEB
:10F92000CDBFDF91CF9108958091DC0A8F5F8093E6
:10F93000DC0AA8950E94493D8091DC0A81508093A1
:10F94000DC0A089566EE7AE18CE49EE00E9422B61D
:10F9500063ED7AE18CE49EE00E9422B665EC7AE1E8
:10F960008CE49EE00E9422B66DEB7AE18CE49EE08E
:10F970000E9422B68CE49EE00E9449B76DEA7AE1CB
:10F980008CE49EE00E9422B660EA7AE18CE49EE07C
:10F990000E9422B660E97AE18CE49EE00E9422B6E1
:10F9A00064E87AE18CE49EE00E9422B66DE67AE19A
:10F9B0008CE49EE00E9422B66BE57AE18CE49EE046
:10F9C0000E9422B666E47AE18CE49EE00E9422B6B0
:10F9D00067E37AE18CE49EE00E9422B668E27AE175
:10F9E0008CE49EE00E9422B660E27AE18CE49EE024
:10F9F0000E9422B66FE07AE18CE49EE00E9422B67B
:10FA000064E07AE18CE49EE00E9422B66AEF79E13C
:10FA10008CE49EE00E9422B662EF79E18CE49EE0E5
:10FA20000E9422B666EE79E18CE49EE00E9422B646
:10FA30006CEC79E18CE49EE00E9422B66DEA79E1FB
:10FA40008CE49EE00E9422B668E979E18CE49EE0B5
:10FA50000E9422B66BE879E18CE49EE00E9422B617
:10FA60006DE779E18CE49EE00E9422B661E779E1DE
:10FA70008CE49EE00E9422B669E679E18CE49EE087
:10FA80000E9422B66EE579E18CE49EE00E9422B6E7
:10FA900061E579E18CE49EE00E9422B669E479E1B7
:10FAA0008CE49EE00E9422B66EE379E18CE49EE055
:10FAB0000E9422B68CE49EE00C9449B7AF92BF92AC
:10FAC000CF92DF92EF92FF920F931F93CF93DF932A
:10FAD0006C017B018A010E94C9D581508E3FA0F440
:10FAE0005701C0E0D0E001501109C017D1077CF4E4
:10FAF000C6018C0F9D1F0E94C9D5F50181935F013E
:10FB0000882329F02196F1CF80E090E005C0CE0D4A
:10FB1000DF1D188281E090E0DF91CF911F910F915E
:10FB2000FF90EF90DF90CF90BF90AF900895882323
:10FB300019F067E478E102C069E478E18CE49EE0C2
:10FB40000C9422B6CF93DF93CDB7DEB72C970FB6C8
:10FB5000F894DEBF0FBECDBF69E977E18CE49EE08B
:10FB60000E9422B68CE49EE00E9449B78CE490E0AB
:10FB70000E94C9D58B37D1F51C821B821E821D8243
:10FB80008FEF9FEF98878F8386E494E09A83898331
:10FB90008CE490E09A8789871C861B860E94E89CEB
:10FBA000CE0101960E9457C590932110809320109A
:10FBB000892B49F46CE777E184E59EE00E9422B648
:10FBC00084E59EE01BC065E777E18CE49EE00E943F
:10FBD00022B68CE49EE00E9449B70E94A85B81E0B7
:10FBE0009FE00E94358281E090E00CC068E877E1F8
:10FBF0008CE49EE00E9422B68CE49EE00E9449B70D
:10FC000080E090E02C960FB6F894DEBF0FBECDBF1B
:10FC1000DF91CF910895AF92BF92CF92DF92EF9292
:10FC2000FF920F931F93CF93DF93CDB7DEB7C058EA
:10FC3000D1090FB6F894DEBF0FBECDBF8E010F5BAA
:10FC40001F4FD8011D921C92FE01ED5BFF4F2EE16C
:10FC5000DF011D922A95E9F70297CCF0FB01628142
:10FC600073814FE150E0C8010E9417DAB80186E1C4
:10FC700090E00E946E7AB8018CE49EE00E945FB72B
:10FC800067E379E18CE49EE00E9422B61BC040E26B
:10FC900050E0B80186E190E00E945E7D892BB1F4CE
:10FCA00040E250E06BE279E1C8010E94A1CD6DE035
:10FCB00079E18CE49EE00E9422B6B8018CE49EE0DB
:10FCC0000E945FB78CE49EE00E9449B78091950B3B
:10FCD0001F928F938091940B1F928F938091930B1F
:10FCE0001F928F938091920B1F928F938091910B13
:10FCF0001F928F938091900B1F928F9389E798E0CA
:10FD00009F938F931F9280E48F93CE0101966C0195
:10FD10009F938F930E9431DA69EF78E18CE49EE043
:10FD20000E9422B6B8018CE49EE00E945FB7B60143
:10FD30008CE49EE00E945FB78CE49EE00E9449B78D
:10FD40007E0191E6E90EF11CD70113961C921E92DA
:10FD5000129788EE93E0A0E0B0E0F70184839583EA
:10FD6000A683B78384E0848784EC93E091838083C7
:10FD700016870587108A178680E590E0928B818B25
:10FD8000158A6CED79EB8DE59BEB0E9405CE8C011D
:10FD90000FB6F894DEBF0FBECDBF892BE1F183E033
:10FDA00090E00E9473CAD8011D969C938E931C9775
:10FDB000FC01F182E0821282C7010E94CE8088237A
:10FDC00019F0C7010E943582D7011F966D917C9171
:10FDD00050975196AD90BC9052976115710569F09E
:10FDE000CE0189589F4F0E9461B7A501BE01695895
:10FDF0007F4FC7010E94BA7507C0F70165857685F8
:10FE0000A501C7010E94E879181619060CF478C0FC
:10FE1000C8010E9436BB00E010E0F701E388F488D7
:10FE20000115110509F463C0F8ECEF16F10409F0AF
:10FE30004CC06DEE78E18CE49EE00E9422B6EB9619
:10FE40001FAE1EAEEB97ED961FAE1EAEED978FEF79
:10FE50009FEFEF969FAF8EAFEF978CE594E0E9961A
:10FE60009FAF8EAFE997C158DF4F19830883CF57F3
:10FE7000D040F8940E94E89CCE0189589F4F0E9480
:10FE800057C590932110809320107894C8010E9448
:10FE900036BB8091201090912110892B29F466EDBA
:10FEA00078E184E59EE027C06BEC78E18CE49EE08D
:10FEB0000E9422B60E94A85B64EC78E18CE49EE08C
:10FEC0000E9422B684E090E0BBC06CEA78E184E551
:10FED0009EE00E9422B64AE050E0B70184E59EE031
:10FEE0000E9442B784E59EE00E9449B706C069E9D6
:10FEF00078E189EF9EE00E9422B68EE090E0A0C0FB
:10FF0000D7011D96BC901D971E96AC90DF92CF92A4
:10FF100085E998E19F938F931F930F930E948ECE54
:10FF2000DF92CF9280E998E19F938F931F930F9375
:10FF30000E948ECED8011C96ED91FC911D9781E018
:10FF40008283DF92CF928DE898E19F938F931F93E6
:10FF50000F930E948ECED8011C96ED91FC911D97B7
:10FF60001282AF92BF9287E598E19F938F931F9380
:10FF70000F930E948ECE82E998E19F938F931F93F7
:10FF80000F930E948ECEF701148A138AD8011C9613
:10FF9000ED91FC911D97A080B1800FB6F894DEBF63
:10FFA0000FBECDBF83E3C82ED12CD501ED91FC91BE
:10FFB0000084F185E02DC501199541975CF4B1E00D
:10FFC000CB1AD10839F064E170E080E090E00E9443
:10FFD000CDABEBCF6E01F7E7CF0ED11CDF92CF9206
:10FFE0008BE498E19F938F931F930F930E94ABCE66
:10FFF0000F900F900F900F900F900F90019709F0B6
:020000021000EC
:100000000CCFF60180819181D70154969C938E93F9
:100010005397D12C80E08A3039F4BAE0DB1609F42A
:10002000FCCE9AE0D92E03C08D3009F0D82EC8013D
:100030000E9450CE8F3F79F7C8010E9436BBEDCEAB
:10004000C058DF4F0FB6F894DEBF0FBECDBFDF91B3
:10005000CF911F910F91FF90EF90DF90CF90BF90C5
:10006000AF9008950E940B7E90939510809394100A
:1000700081E09FE00C9435820895CF93DF931F9227
:10008000CDB7DEB76983DC01ED91FC910280F3818D
:10009000E02D41E050E0BE016F5F7F4F19950F905A
:1000A000DF91CF910895FC01818D928D0895FC011F
:1000B0008489958908952AEE33E0FC0131832083F9
:1000C000FB014089518962897389FC014283538312
:1000D000648375830895DC01ED91FC91048CF58DAA
:1000E000E02D199480E00895FC019485FB0184853E
:1000F000981303C081E0943009F480E0089521E072
:10010000FC018485843009F420E0822F089508954D
:100110008F929F92AF92BF92DF92EF92FF920F93D6
:100120001F93CF93DF931F921F92CDB7DEB77C0151
:100130004B018A01FC01A688B788D08CCE010196BC
:100140000E9488C589819A810E942C758D2D0E94FC
:10015000E5B28017910720F48D2D0E94E5B28C0145
:100160009801A401B5018D2D0E9480B20E942B75CB
:10017000F70186899789800F911F978B868BC8011D
:100180000F900F90DF91CF911F910F91FF90EF9003
:10019000DF90BF90AF909F908F900895CF93DF93A3
:1001A000FC0124852430D1F0EC010E948DC58431FE
:1001B00081F0882371F0883161F08C3161F4E8813D
:1001C000F9810084F185E02DCE01199521E0892B7C
:1001D00019F420E001C021E0822F01C080E0DF910E
:1001E000CF9108958EBD00000DB407FEFDCF8EB5F2
:1001F0000895DF92EF92FF920F931F93CF93DF93B7
:100200001F921F92CDB7DEB7D82ECE0101960E9465
:1002100088C589819A810E942C75E12CF12C8D2D45
:100220000E949CBC8C01892B21F08D2D0E949CBCCE
:100230007C010E151F0599F70E942B75C8010F90C0
:100240000F90DF91CF911F910F91FF90EF90DF9072
:100250000895FC011382128288EE93E0A0E0B0E0E2
:1002600084839583A683B78388E794E09183808312
:100270008AEE93E097878687108A118A128A138AFA
:1002800084E0808F0895AF92BF92CF92DF92EF9279
:10029000FF920F931F93CF93DF93CDB7DEB7AF9746
:1002A0000FB6F894DEBF0FBECDBF7C015B016A01C3
:1002B0000AEE13E01A8309831B821C821D821E82B0
:1002C000CE0109960E9429811BA70AA71CA61DA67C
:1002D0001EA61FA68091DA0C9091DB0CA091DC0C7D
:1002E000B091DD0C8EA39FA3A8A7B9A78B839C8395
:1002F000AD83BE8318861F82AE01465D5F4FB50198
:10030000CE0101960E9413AC81309105B1F4D70162
:10031000ED91FC910488F589E02D1DA30CA38CA51B
:100320009DA5AEA5BFA58EA39FA3A8A7B9A7A6010B
:10033000BE016C5D7F4FC7011995AF960FB6F8945B
:10034000DEBF0FBECDBFDF91CF911F910F91FF9008
:10035000EF90DF90CF90BF90AF9008959B0190E019
:100360000496982F8827642F820F931F0C9481BCCA
:100370001F93CF93DF931F921F92CDB7DEB7182F35
:10038000CE0101960E9488C589819A810E942C75B0
:1003900060E170E0812F0E9478C54FEF62E070E06D
:1003A000812F0E94AE810E942B750F900F90DF91DC
:1003B000CF911F910895DF92EF92FF920F931F93B9
:1003C000CF93DF931F921F92CDB7DEB7182FD62E93
:1003D0007A01022F0E94B881CE0101960E9488C541
:1003E00089819A810E942C754D2D402B60E070E030
:1003F000812F0E94AE81E114F10459F4E0902A109B
:10040000F0902B108FEFE81AF80AF0922B10E09280
:100410002A104F2D64E070E0812F0E94AE814E2D96
:1004200065E070E0812F0E94AE8161E070E0812F75
:100430000E9478C50E942B7581E00F900F90DF918C
:10044000CF911F910F91FF90EF90DF900895CF9380
:10045000DF93FC01808D843029F0EF010E94B88188
:1004600084E0888FDF91CF910895CF92DF92EF9251
:10047000FF920F931F93CF93DF931F921F92CDB7DD
:10048000DEB7FC01F484F4E0FF1699F18C01CE0193
:1004900001960E9488C589819A810E942C7568E026
:1004A00070E08F2D0E9478C50E942B750E9407ACCA
:1004B0006B017C01C8010E948DC58823B9F062E3FD
:1004C00070E080E090E00E94CDAB0E9407ACDC01C0
:1004D000CB018C199D09AE09BF09883E9340A10547
:1004E000B10540F3F80184850E94B88184E0F801E9
:1004F00084870F900F90DF91CF911F910F91FF9004
:10050000EF90DF90CF900895CF93DF9390E0049623
:10051000982F8827EC01C60FD71F0E941CBC8FE0C4
:100520000E94F2808D2F0E94F2808C2F0E94F28018
:1005300080E00E94F280C82F0E9416BC8C2FDF91B1
:10054000CF910895CF92DF92FF920F931F93CF9395
:10055000DF931F921F92CDB7DEB7F82E6B01CE014D
:1005600001960E9488C589819A810E942C7568E253
:1005700070E08F2D0E948482082F10E069E270E005
:100580008F2D0E948482702F6627682B21E030E037
:10059000A6018F2D0E9438B20E942B7581E090E059
:1005A0000F900F90DF91CF911F910F91FF90DF90EF
:1005B000CF900895CF93DF931F92CDB7DEB7FC01A4
:1005C000218D328D232B49F0BE016F5F7F4F808DCF
:1005D0000E94A282898190E002C08FEF9FEF0F906E
:1005E000DF91CF9108958F929F92BF92CF92DF9229
:1005F000EF92FF920F931F93CF93DF931F921F925F
:10060000CDB7DEB7B82E6B017A01CE0101960E94FC
:1006100088C589819A810E942C75812C912C8B2D03
:100620000E949CBC8C01892B21F08B2D0E949CBCCC
:100630004C010815190599F70115110599F463E0A6
:1006400070E08B2D0E9484828431D9F18823C9F116
:1006500001E010E08C3111F400E010E011950195FB
:1006600011092FC0E016F1060CF4870110161106CF
:1006700044F568E270E08B2D0E948482E82EF12C14
:1006800069E270E08B2D0E948482FE2CEE24E82A21
:100690009801A601B7018B2D0E9438B2E00EF11E21
:1006A0004F2D68E270E08B2D0E94AE814E2D69E2E5
:1006B00070E08B2D0E94AE8160E470E08B2D0E9473
:1006C00078C50E942B75C8010F900F90DF91CF91D4
:1006D0001F910F91FF90EF90DF90CF90BF909F9070
:1006E0008F900895CF93DF93FC01218D328D2115DA
:1006F000310519F48FEF9FEF11C0EC01421753073A
:1007000008F0A901888D0E94F3821816190694F743
:10071000298D3A8D281B390B3A8F298FDF91CF9184
:1007200008950F931F93CF93DF931F92CDB7DEB73A
:10073000FC01218D328D232B61F08C0141E050E0D2
:10074000BE016F5F7F4F808D0E94F38218161906DD
:100750001CF08FEF9FEF08C0F801818D928D0197FB
:10076000928F818F898190E00F90DF91CF911F91BF
:100770000F9108950F931F93CF93DF93CDB7DEB7FB
:1007800028970FB6F894DEBF0FBECDBF8C01D801FD
:1007900059968D919C915A97892B41F0ED91FC913E
:1007A0000284F385E02DC8011995F1CFF801808D01
:1007B0000E94F9801816190654F548E050E0BE0171
:1007C0006F5F7F4FD80158968C910E94F382181664
:1007D0001906FCF4D801509684E0FE013196019090
:1007E0000D928A95E1F78D8190E0982F88272E81D0
:1007F000820F911DF801958B848B8F8190E0982F4B
:1008000088272885820F911D928F818F02C080E0FA
:1008100090E028960FB6F894DEBF0FBECDBFDF91F3
:10082000CF911F910F9108951F93CF93DF931F9244
:100830001F92CDB7DEB7182FCE0101960E9488C552
:1008400089819A810E942C7563E070E0812F0E945B
:100850008482182F0E942B75812F0F900F90DF91AB
:10086000CF911F910895EF92FF921F93CF93DF9343
:10087000FC01208D243011F080E01CC07B01EC01D4
:1008800010E0812F0E941484811102C0188F05C0CE
:100890008831E1F31F5F1430A1F7888D843061F354
:1008A000FD86EC861A8E198E20E0A70162E00E9478
:1008B000DB8181E0DF91CF911F91FF90EF90089550
:1008C0001F93CF93DF931F921F92CDB7DEB7FC012A
:1008D000108DCE0101960E9488C589819A810E945F
:1008E0002C7560E270E0812F0E9478C562E070E0B4
:1008F000812F0E94848284FD1DC062E070E0812F00
:100900000E94848283FF0BC048E162E070E0812F87
:100910000E94AE810E942B7580E090E015C00E947D
:100920002B75CE0101960E9488C589819A810E940B
:100930002C75DCCF40E162E070E0812F0E94AE8137
:100940000E942B7581E090E00F900F90DF91CF9186
:100950001F910895CF93DF93C82FD62F472F60E1C3
:1009600070E00E94AE814D2F61E170E08C2FDF912D
:10097000CF910C94AE8190E0982F882744E050E00E
:10098000845F9B4F0C9452BCBF92CF92DF92EF9248
:10099000FF920F931F93CF93DF9300D000D0CDB77A
:1009A000DEB7FC01208D243009F04CC06A017B01C8
:1009B0008C01B12C63E070E08B2D0E948482811148
:1009C00003C0F801B08E06C08831D9F3B394F4E0C7
:1009D000BF12F0CFF801808D8430A1F196E0EEE6F1
:1009E000F4E0DE01119601900D929A95E1F7F7017E
:1009F00093819F779C8394819D8395819E83B7018A
:100A00006E5F7F4F0E94BB84B601F801808D0E940B
:100A1000AA84F801808D90E0982F882746E050E066
:100A2000BE016F5F7F4F8A5F9B4F0E9452BCF801EF
:100A3000128E118E20E8A60162E0808D0E94DB817B
:100A400081E001C080E026960FB6F894DEBF0FBEAD
:100A5000CDBFDF91CF911F910F91FF90EF90DF906D
:100A6000CF90BF900895DF92EF92FF920F931F9364
:100A7000CF93DF931F921F92CDB7DEB7FB01DC014E
:100A800057961C921E9256972281211109C02381EC
:100A9000211106C02481211103C025812223F1F0F8
:100AA00041155105D9F07A018F01FC01D08CCE019E
:100AB00001960E9488C589819A810E942C75B8018F
:100AC0006E5F7F4F8D2D0E94BB84B7018D2D0E94DC
:100AD000AA840E942B7581E090E002C080E090E043
:100AE0000F900F90DF91CF911F910F91FF90EF909A
:100AF000DF900895FC01A7812A2F2E7FD1F08281FB
:100B000082958F7081508330A0F4A695B0E0119744
:100B10002BE531E00E947DD624E630E040E050E055
:100B20000E9411D6DA01C90187569F4FAF4FBF4FC0
:100B300008958FEF9FEF0895CF93DF93EC018A81A3
:100B4000982F92959F7019F0943050F503C08F70D4
:100B500080628A83CB01770FAA0BBB0B9C01AD018E
:100B60002959310941095109A4E6B0E00E9430D663
:100B70002BE531E040E050E00E9411D625363105EA
:100B80002CF437FF05C020E030E002C024E630E05E
:100B90002F5F220F8F818170282B2F8381E001C06E
:100BA00080E0DF91CF9108956F927F928F929F9214
:100BB000AF92BF92CF92DF92EF92FF920F931F936B
:100BC000CF93DF93CDB7DEB72C970FB6F894DEBF87
:100BD0000FBECDBF4C01762E672E6A01590181E010
:100BE00090E09093301080932F1026E040E855E27B
:100BF00060E070E088E99BE00E94DEA270922F0D19
:100C000088E99BE090932E0D80932D0D10923A0E63
:100C100010923C0E10923B0E0115110541F001306F
:100C2000110539F4FE2CEE24EE24EA9402C0FF24D0
:100C3000FA94C701A0E0B0E089839A83AB83BC83B8
:100C400080E190E09E838D83A60160E070E04F8399
:100C5000588769877A879C878B874AE050E0672DA1
:100C6000762D89EF9EE00E9442B767E27BE189EF33
:100C70009EE00E9422B6BE01695F7F4F89EF9EE031
:100C80000E94D86B8C0163E27BE10E9422B64AE0AD
:100C900050E0B501C8010E9442B760E27BE1C801A3
:100CA0000E9422B6BE016F5F7F4FC8010E94D86BC1
:100CB0000E9449B7A114B10491F082E0A816B104D2
:100CC00009F5D092B50DC092B40D1092B70D1092E7
:100CD000B60DF092B90DE092B80D86E010C0D0923A
:100CE000B50DC092B40DE11003C080E090E002C0E9
:100CF00080E09FEF9093B70D8093B60D85E00E9442
:100D000027A007C068E07BE189EF9EE00E9422B641
:100D100080E01092301010922F10882331F0C4011F
:100D20000E946F4D80E090E002C081E090E02C9640
:100D30000FB6F894DEBF0FBECDBFDF91CF911F91EC
:100D40000F91FF90EF90DF90CF90BF90AF909F906A
:100D50008F907F906F9008952F923F924F925F9265
:100D60006F927F928F929F92AF92BF92CF92DF92BB
:100D7000EF92FF920F931F93CF93DF93CDB7DEB720
:100D8000A4970FB6F894DEBF0FBECDBF6C010F8BDA
:100D9000188F298F3A8F4B8F5C8F6D8F7E8F2DE050
:100DA000E216F10428F4F701E456FB4F308001C04D
:100DB000312CCE0147960E947A8597FD04C0BC0174
:100DC000C6010E949C85198D812F8F70D6011296C5
:100DD0000C911297007F082B12960C9302950F70BE
:100DE000802F90E08C30910508F027C4FC01882703
:100DF000E25DFE4F8F4F0C9466D612951F70812FC7
:100E000090E0FC013197EB30F10508F090C08827A5
:100E1000E65CFE4F8F4F0C9466D68E8DF60187836D
:100E20008D8DD60116968C9316978C8D15968C9376
:100E300015978B8D14968C9314971295107F12969C
:100E40008C9112978F70182B12961C93F6C38D8D70
:100E50009E8DF6018683878190FB80F987838C8D38
:100E60008583EBC38B8D9C8DAD8DBE8DB7FD0BC087
:100E70008F3F9105A105B105A1F19CF18FEF90E0A5
:100E8000A0E0B0E02EC080E02CC06B8D7C8D8D8DFD
:100E90009E8D673FBFEF7B078B079B076CF061154B
:100EA000EAE07E07810591054CF42AE030E040E05D
:100EB00050E00E9411D603C020E001C02FEFD60100
:100EC00014962C93BAC38D8D9E8DF60186838781EF
:100ED00090FB80F987838C8D85838B8D8483ADC354
:100EE0008B8DD60114968C93A8C38B8C9C8CAD8C67
:100EF000BE8C20E030E0A901C501B4010E94A5D458
:100F000087FD0FC020E030E04FE753E4C501B40196
:100F10000E94ADD718163CF0C501B4010E947ED7DF
:100F200003C060E001C06FEFF601648386C36FEA1F
:100F30007BE189EF9EE00E9422B64AE050E0612FFB
:100F400089EF9EE00E94B1B66CEA7BE167C38B8DAE
:100F50009C8DAD8DBE8DF60184839583A683B7836A
:100F6000107F82818F70182B128367C360E0CE01DF
:100F700047960E94D19AD60114968C93149779C003
:100F800012951F70812F90E0FC013197EB30F10535
:100F900008F077C08827EB5BFE4F8F4F0C9466D626
:100FA0006B8D7C8D8D8D9E8D0E94ACD420E030E0C9
:100FB00040E251E40E9405D70BC06B8D70E080E0E9
:100FC00090E010C06B8D7C8D8D8D9E8D0E94ACD479
:100FD000F60164837583868397832FC36B8D7C8D25
:100FE0008D8D9E8D0E94AAD4D60114966D937D930B
:100FF0008D939C93179721C31295107FF6018281E0
:101000008F70182B12838B8D9C8DAD8DBE8D84833C
:101010009583A683B78311C31295107FD6011296CC
:101020008C9112978F70182B12961C938B8D9C8D20
:10103000AD8DBE8DF60184839583A683B783FDC2F3
:1010400060E0C6010E94D19AD60114968C93149741
:101050008D8D9E8D16968C93169717968C9117975B
:1010600090FB80F917968C9317978C8D15968C931F
:10107000159712968C9112978F70806212968C93AE
:10108000DCC26AE97BE189EF9EE00E9422B64AE079
:1010900050E0612F89EF9EE00E94B1B667E97BE1E5
:1010A000BDC2BB24B39401C0B12C12951F70812F17
:1010B00090E0FC013197EB30F10508F0A0C28827E1
:1010C000E05BFE4F8F4F0C9466D68B8D9C8DAD8D63
:1010D000BE8DF60184839583A683B7831295107F16
:1010E00082818F70182B128388E012C3163091F022
:1010F00038F4113069F0133001F56FEF70E01FC064
:101100001730A1F01A501230C0F46B8D7C8D17C0CF
:101110006B8D15C06B8D7C8D8D8D9E8D2AE030E0A2
:1011200040E050E00E9411D6B90109C06B8D7C8D62
:101130008D8D9E8D0E9477D702C060E070E084E6BE
:101140008D8F8E8D8E7F8E8F1C8E898D8F7080629D
:10115000898F6B8F2C8D30E0AFEFB0E00E9443D6CB
:101160006115F4E67F078105910544F424E630E03B
:1011700040E050E00E9411D6890102C00FEF10E05C
:101180002B8CE22CF12CBB2009F47BC1AE8CA694F5
:10119000B12CC501019798A38F8F019609F083C0E8
:1011A000003811050CF04AC08FE790E0801B910BCE
:1011B0008E9DD0018F9DB00D9E9DB00D11242FEFFF
:1011C00030E00E947DD621E83EE740E050E00E94FA
:1011D00011D6F60127832EEF31E0D8010E947DD68B
:1011E000EFE74E2E512C612C712CA30192010E942D
:1011F00011D6D7010E9430D62FEF30E040E050E00A
:101200000E9411D649015A012BE930E0D8010E9411
:101210007DD6A30192010E9411D6DA01C9018C5931
:101220009F4FAF4FBF4F8C017401FFEF8F1691049A
:1012300019F114F1EE24EA94F12C1EC0C801110F2B
:10124000AA0BBB0B9C01AD01205831094109510982
:10125000ABE9B0E00E9430D62FE730E040E050E04C
:101260000E9411D6DA01C9018C599F4FAF4FBF4F71
:101270008C01D60117961C926AE87BE189EF9EE00B
:101280000E9422B64AE050E0B80189EF9EE00E9439
:1012900042B76CE77BE189EF9EE00E9422B64AE00C
:1012A00050E0B701E6C02F8D38A1AAEBBFEF0E9436
:1012B00075D644E6842E912CA12CB12CA501940165
:1012C0000E9411D629013A01B4E64B0E511C611C53
:1012D000711C26E430E0AF8DB8A10E947DD6A50137
:1012E00094010E9411D649015A01EEE18E0E911C23
:1012F000A11CB11CC801012E000CAA0BBB0B8F8FC7
:1013000098A3A9A3BAA3003811050CF057C08FE722
:1013100090E0801B910B8E9DD0018F9DB00D9E9D06
:10132000B00D1124A50194010E943BD69B01AC0194
:10133000AFEFB0E00E9430D624E63AE640E050E05D
:101340000E9411D6D60117962C932F8D38A149A152
:101350005AA1240D351D461D571DAEEFB1E00E9468
:1013600030D623EE30E040E050E00E9411D63CA39E
:101370002BA3A22DB0E00E9430D62FEF30E040E04A
:1013800050E00E9411D62F8F38A349A35AA32FEF04
:1013900030E0D8010E947DD62FE730E040E050E0F9
:1013A0000E9411D68901EF8CF8A0BFEFEB16F10473
:1013B00001F1FCF0EE24EA94F12C1BC02F8D38A132
:1013C00049A15AA12058310941095109ABE9B0E0BE
:1013D0000E9430D62FE730E040E050E00E9411D666
:1013E000DA01C9018C599F4FAF4FBF4F8C01F601F5
:1013F000178266E77BE189EF9EE00E9422B62AE031
:1014000030E0B301A20189EF9EE00E94FAB660E7E6
:101410007BE189EF9EE00E9422B62AE030E0B50130
:10142000A40189EF9EE00E94FAB668E67BE189EFAD
:101430009EE00E9422B64AE050E0B80189EF9EE0AB
:101440000E9442B760E67BE189EF9EE00E9422B6EF
:101450004AE050E0B70189EF9EE00E9442B767E59D
:101460007BE189EF9EE00E9422B64AE050E06BA14A
:101470007CA189EF9EE00E9442B789EF9EE00E9426
:1014800049B720E030E040E050E060E070E0CE019D
:1014900001960E946FA5B02E2D8D3E8D3170AFEF5D
:1014A000BFEF0E9443D62DE631E040E050E00E94BD
:1014B00011D644275527AAEFB5E00E9430D6DC01AB
:1014C000CB019058AF4FBF4FCD01BB2797FDB095D3
:1014D000AB2F8E3FF1E09F0760F48F3F910518F42A
:1014E000682F80E029C06EEF962F981B80E06FEF89
:1014F00024C08C3F43E0940760F48D3FE2E09E07F8
:1015000018F48E5F6FEF03C06CEF681B8FEF90E0F5
:1015100014C08A3FF5E09F0769F08B3F44E09407D1
:1015200028F494E0980F8FEF60E007C06AEF681B23
:10153000862F01C080E060E09FEFAFEFEA1AFA0A61
:101540000F5F1F4FB094EB2DF0E0909FA001919F93
:10155000500D1124452F55274E0F5F1F609F90019E
:10156000619F300D1124232F33272E0F3F1F809FA3
:10157000B001819F700D1124872F9927E80FF91F63
:10158000D7010E947DD62B013C0144246624772498
:101590009F010E947DD6BB27A92F982F872F53012B
:1015A0004201882A992AAA2ABB2A9A01D7010E94B5
:1015B0007DD6DC01CB018827AA27BB27BA2FA92F0C
:1015C000982F882788299929AA29BB29F601A6835B
:1015D0009583848360E57BE189EF9EE00E9422B6DB
:1015E000C6010E9444998A859B850E940BCB8F81FE
:1015F000988597FD22C060E00E9484AA1EC06EE319
:101600007BE189EF9EE00E9422B64AE050E0612F24
:1016100089EF9EE00E94B1B66BE37BE189EF9EE02B
:101620000E9422B64AE050E0602F89EF9EE00E94BF
:10163000B1B689EF9EE00E9449B7332009F466C035
:10164000D60112961C9112951F70212F30E0832D28
:1016500090E02817390709F459C06FE27BE189EF60
:101660009EE00E9422B64AE050E0612F89EF9EE0A2
:101670000E94B1B66CE27BE189EF9EE00E9422B647
:101680004AE050E0632D89EF9EE00E94B1B66AE225
:101690007BE189EF9EE00E9422B6F601008119826B
:1016A0001A821B821C821D821E821F821886932D25
:1016B0009295907F8B818F70892B8B830983EE2489
:1016C000EA94FE2C11812281338144815581668107
:1016D0007781CE0101960E94AC86D6012C9311969B
:1016E0003C93119712964C93129713965C93139711
:1016F00014966C93149715967C93159716968C9365
:10170000169717969C93C6010E94449988E0F601AB
:10171000DE01119601900D928A95E1F729813A81B7
:101720004B815C816D817E818F819885A4960FB6F7
:10173000F894DEBF0FBECDBFDF91CF911F910F9107
:10174000FF90EF90DF90CF90BF90AF909F908F90E1
:101750007F906F905F904F903F902F9008950895E5
:1017600084E090E00895DC011496ED91FC911597CA
:10177000309729F08081082E000C990B089580E0A5
:1017800090E008950895DC011296ED91FC91139775
:10179000309779F016968D919C911797833091052B
:1017A00049F0049719F421E030E006C0208530E0CC
:1017B00003C0089522E030E0C901089580913110FE
:1017C0009091321008950C940BCB0C940BCB0C948D
:1017D0000BCB6EEC7BE189EF9EE00E9422B689EF95
:1017E0009EE00E9449B7109232101092311081E0B1
:1017F00090E008950E94771261EC7BE189EF9EE012
:101800000E9422B689EF9EE00E9449B781E090E0F5
:10181000909332108093311008958F929F92AF92DF
:10182000BF92CF92DF92EF92FF920F931F93CF93CD
:10183000DF93CDB7DEB728970FB6F894DEBF0FBEA3
:10184000CDBF09831A83122F2B833C834D835E8384
:101850006F837887B7011F70C12ED12CDC011496DD
:10186000ED90FC9015976115710569F0FB01808181
:10187000882349F0D7011F968D919C9150970E9423
:10188000565A892B51F5D7011F96ED91FC9150972F
:10189000E680F780812E912CA12CB12CE114F1046B
:1018A000E1F06CE977E0C7010E94565AFC0190858F
:1018B0009F70923049F481859285A385B4858815FF
:1018C0009905AA05BB0549F068EA78E0C7010E94BE
:1018D000565AF701E280F380E1CFF980FF20A1F1B1
:1018E000C114D10419F0113089F503C0CC24C3947C
:1018F000D12C8FEF8F0D823020F162E37DE189EFF3
:101900009EE00E9422B64AE050E06F2D89EF9EE0F3
:101910000E94B1B689EF9EE00E9449B762E27DE184
:1019200089EF9EE00E9422B64AE050E0B60189EFBE
:101930009EE00E9442B789EF9EE00E9449B780E096
:1019400001C081E090E014C01130B9F2113068F4A8
:101950006FE37DE189EF9EE00E9422B62B81207F1C
:1019600081E090E029F480E003C01230B9F3D6CFD3
:1019700028960FB6F894DEBF0FBECDBFDF91CF9192
:101980001F910F91FF90EF90DF90CF90BF90AF909D
:101990009F908F9008954F925F926F927F928F9257
:1019A0009F92AF92BF92CF92DF92EF92FF920F93EE
:1019B0001F93CF93DF93EC01EC81FD8183859485A8
:1019C000892B21F485859685892B89F180912F10AB
:1019D00090913010892B59F5E881F9810484F585BF
:1019E000E02DCE0119954C0181E088169104F9F49F
:1019F000EC81FD8145805680612C712C0E9407ACE2
:101A00009B01AC01EC81FD816781708581859285A8
:101A1000AA24AA94BA2C6501830172010E9482480B
:101A200081111AC004C01092301010922F10EC8156
:101A3000FD8185819681DF91CF911F910F91FF905C
:101A4000EF90DF90CF90BF90AF909F908F907F905E
:101A50006F905F904F900895EA81FB810190F08133
:101A6000E02D008111816CE17DE189EF9EE00E9413
:101A700022B6B80189EF9EE00E945FB789EF9EE031
:101A80000E9449B79092301080922F10EC81FD8116
:101A900041815281052E000C660B770B238188E96A
:101AA0009BE00E94DEA2EC81FD81038114816181B3
:101AB00072814AE050E089EF9EE00E9442B768E1FF
:101AC0007DE189EF9EE00E9422B6A80160E070E00F
:101AD0002AE089EF9EE00E945BB689EF9EE00E94BB
:101AE00049B760E070E08A819B810E9457698093CA
:101AF0002F0D88E99BE090932E0D80932D0D109271
:101B00003A0E10923C0E10923B0EEC81FD816385E3
:101B1000748542E050E0CE010E9464A9EC81FD8111
:101B20006585768543E050E0CE010E9464A90C8172
:101B30001D8180E00E946C48F8016783708781876F
:101B40009287EA81FB810190F081E02D0081118173
:101B50006FE07DE189EF9EE00E9422B6B80189EF37
:101B60009EE00E945FB789EF9EE00E9449B70E9405
:101B700007AC2B013C010E9407AC9B01AC01AA24DD
:101B8000AA94BA2C650112E3E12EF12C00E010E0DA
:101B9000C301B2010E948248811145CF0E94617A3F
:101BA000EACFCF93DF93EC016FEA78E08CE59EE01B
:101BB0000E947B718C819D810E940BCB60E070E064
:101BC0008A819B810E949C681D821C8281E090E03A
:101BD000DF91CF9108958F929F92AF92BF92CF9253
:101BE000DF92EF92FF920F931F93CF93DF93EC015D
:101BF0000E9477128C819D81892B59F481E190E0BC
:101C00000E9473CABC018A819B810E949C689D834B
